:020000040800F2
:10000000F0FF0010E9B8050859CD0008F584040890
:1000100089B9050889B9050889B9050800000000F3
:1000200000000000000000000000000055CD0008A6
:1000300051CD0008000000004DCD00085D7404089B
:1000400089B9050889B9050889B9050889B9050874
:1000500089B9050889B905080D940408399504087B
:10006000FD940408C194040885940408EDA10508D2
:10007000DDA10508CDA10508BDA10508A9A10508B8
:1000800095A1050881A1050889B9050889B9050860
:1000900089B9050889B9050889B90508499404088A
:1000A000755D0408FD5D0408655D0408255E0408AF
:1000B000ED5D0408DD5D0408CD5D040881A8050838
:1000C00089A8050875A805087DA8050889B9050847
:1000D00089B905086D780408B1770408F576040835
:1000E000D193040889B9050825060108555D04085F
:1000F000855D0408455D0408AD5D04086DA1050833
:1001000089B9050889B90508BD5D040889B90508DC
:10011000397604087D750408ED680308D96803087A
:1001200059A1050845A1050831A105081DA105082B
:1001300009A1050889B9050889B9050889B905081B
:1001400089B9050889B9050889B90508FDF40008C9
:10015000F5A00508E1A00508CDA00508C1740408B4
:1001600069A8050871A8050889B9050889B90508AD
:1001700089B9050889B9050889B9050889B9050843
:0801800089B9050889B90508D9
:0801880098B40500010000001D
:10019000030101000A000000643100202452002005
:1001A00000000000ED0A0108130201000400000035
:1001B0000C2200203052002000000000100900082E
:1001C0000D10010070000000D43F002034520020C8
:1001D0000000000041010408040008008000000045
:1001E000143F0020A4520020000000000000000086
:1001F0000902010001000000EC50002024530020FF
:100200000000000014090008FD01010024000000A6
:10021000CC3E002028530020000000009B3A040838
:10022000FB01010001000000883E00204C5300202B
:1002300000000000ADC50408FC0101000900000039
:10024000543D00205053002000000000BDC50408AC
:10025000F701010006000000483D00205C5300202B
:100260000000000016090008F90101000400000068
:10027000443D00206453002000000000413B04087E
:100280000A800100280000001C3D00206853002067
:1002900000000000F5080208160215003F000000EB
:1002A000302F00209053002000000000D9C5040822
:1002B0003400010010000000483C0020D053002012
:1002C00000000000A13C020811020100080000002B
:1002D000203C0020E0530020000000001C09000822
:1002E0001212010004000000183C0020E853002016
:1002F000000000002409000818200100320000005E
:10030000E43B0020EC53002000000000F5BF04088F
:10031000061001001C000000142F002020540020B3
:100320000000000041C50408122001001100000077
:10033000043B00203C540020000000002809000875
:10034000000201000B000000403800205054002043
:100350000000000000000000FA010100030000009E
:10036000C43700205C5400200000000019BF0408BE
:100370000202010003000000082700206054002052
:1003800000000000000000000C020100040000005A
:10039000E8260020645400200000000025BF040867
:1003A000FE01010014000000EC4100206854002010
:1003B0000000000085BF04081B1001000C000000B5
:1003C000D46900208C7C002000000000393D010829
:1003D00021020100F00000003C680020987C002011
:1003E000000000000927010823120100100000008E
:1003F0006C6B0020887D0020000000003C09000894
:10040000371001002E000000206F0020987D002092
:10041000000000004C0900080E020100020000006C
:10042000686B0020C87D0020000000007A090008E9
:100430001610010006000000606B0020CC7D00203B
:10044000000000007C0900082F10010022000000BD
:10045000687C0020D47D0020000000008209000894
:100460001E00010009000000046B0020F87D002040
:1004700000000000A40900080510010006000000AB
:10048000506B0020047E002000000000AE09000830
:10049000F581010068000000CC6700200C7E002080
:1004A00000000000DD3401082320010010000000DE
:1004B000AC6B0020747E002000000000090A0208D6
:1004C000FD070100760000000A670020847E0020FE
:1004D000000000003D100108261001000E00000081
:1004E0000C7F0020FC7E002000000000B90E0108F7
:1004F0000B3001001A000000F06600204C7F002045
:1005000000000000B40900081F30010024000000B2
:10051000EC690020687F002000000000D00900087E
:1005200005020100040000007C6B00208C7F00208D
:1005300000000000F409000814000100040000009D
:10054000049000203090002000000000F80900080E
:10055000012001000C00000064860020349000207F
:1005600000000000FC0900080EF003009E010000DE
:100570007C8300204090002000000000E91D02085C
:1005800013000100040000000C8D0020E091002009
:1005900000000000080A000801010100040000003A
:1005A000BC820020E4910020000000000000000058
:1005B0000001010004000000B4820020E891002046
:1005C000000000000C0A0008020101000300000006
:1005D000B0820020EC910020000000003D320308B2
:1005E000220201001C010000F48A0020F09100208A
:1005F0000000000019C204080C200600CC00000016
:10060000408500200C930020000000000132030808
:10061000010201000B000000C8820020D8930020D6
:100620000000000009BF04081B02010010000000C8
:10063000AC860020E4930020000000008DBE04087A
:10064000203201000A00000030A100203CA100205F
:1006500000000000C51D0208150010007000000019
:100660003C9F002048A10020000000000000000086
:100670002A000800600000004C9E0020B8A1002065
:10068000000000009D1D02082C0004001000000066
:1006900028A2002018A2002000000000751B0208FC
:1006A0002B001200240000005CA2002038A20020D1
:1006B00000000000491B02082920140078000000F7
:1006C0002C9C002080A20020000000000000000000
:1006D000F62101000C000000689A0020F8A200201A
:1006E00000000000100A00081C0202001C000000AC
:1006F000109A002048A300200000000049C104080F
:1007000028200100180000002C9A002064A300207B
:1007100000000000611F0208031201003D000000FC
:10072000B0A80020F4A80020000000001C0A000867
:1007300025201E002C01000014A6002034A9002052
:100740000000000000000000101001000200000086
:10075000FCA5002060AA0020000000005A0A000842
:10076000F821010006000000DCA5002064AA00209A
:10077000000000005C0A00081900010005000000EC
:1007800030A500206CAA002000000000620A0008CA
:100790001A0001000E00000084A3002074AA0020AB
:1007A00000000000680A0008290201004000000063
:1007B0002CAD0020ECB2002000000000760A0008FA
:1007C0000A0201001400000060B200204CB30020B7
:1007D000000000002D3903080300010001000000A3
:1007E000B0B2002060B30020000000000000000054
:1007F000020001000C00000080B6002010B70020AD
:1008000000000000000000002802040004000000B6
:1008100090B8002034BA002000000000ADBE0408EB
:1008200027020400040000008CB8002038BA002021
:1008300000000000A1BE04081F0208001000000014
:100840007CB800203CBA0020000000003DBF040836
:100850001A0201003C00000040B800204CBA002001
:100860000000000085C004083810010001000000ED
:1008700038B7002088BA002000000000B60A00083F
:10088000081203000F00000020BB002010BB002056
:1008900000000000B1BE0408060203000C000000C6
:1008A0003CBB002030BB002000000000C5C1040894
:1008B0002700010004000000B0BA002048BB00205F
:1008C00000000000B80A000810020100010000004A
:1008D000A8D90020A4D9002000000000BC0A00080C
:1008E00007020100020000008CD90020ACD90020D2
:1008F00000000000BE0A00081D0202000600000001
:1009000078D90020B0D900200000000000000000CD
:100910000000010029003D0100000000200000004F
:1009200001010101FFFFFFFF000000010000054D74
:1009300042463400000800020000000000000000F1
:100940000000000000000000000000002000320055
:10095000C800D00796001400320028004C0440065E
:100960000005500014000F000800640001000100A1
:1009700005000A000000F40196000000C409000010
:10098000190000000000000000000000000000004E
:100990000000000000000000000000000000000057
:1009A0000000000000050100000000000000200021
:1009B00001010000AE014A015E012C016401010049
:1009C000000001000A019A01001E0A000002000056
:1009D000000000000001000000050000010203000B
:1009E0000000000000000000000000000000000007
:1009F000008007000000000003000023E8036400FB
:100A0000040A000114001E00480444309001000054
:100A100000000000010000000202000000000000D1
:100A200000000000000000000000000000000000C6
:100A300000000000000000000000000000000000B6
:100A400000000000000000000000000000000000A6
:100A50000000000000000000010000050101F40199
:100A600014000000280100007E05EA05B4053200EC
:100A7000E803D007000000000000000000000000B4
:100A80000000000000000000000000000000000066
:100A90000000000000000000000000000000000056
:100AA0000000000000000000000000000000000046
:100AB0000000000000000000200300000000023CD5
:100AC0000403090412010002EF02014083045632BC
:100AD00000020102030100001201000202020040B4
:100AE00083044057000201020301000009022000B4
:100AF000010104C032090400000208065005070580
:100B00008102400000070501024000000902640064
:100B1000030100C0320904000001030000000921A4
:100B2000110100012226000705830308000A080BB3
:100B30000102020201000904010001020201000594
:100B400024001001052401000204240202052406E9
:100B50000102070582030800FF09040200020A00DF
:100B60000000070501024000000705810240000067
:100B700009024300020100C0320904000001020220
:100B800001000524001001052401000104240202D3
:100B90000524060001070582030800FF090401007F
:100BA000020A00000007050102400000070581025B
:100BB00040000000FF00000000FF000000000000F7
:100BC0000000AA55070100000800AA550501000011
:100BD000080000001CF00508FF1FFF1F7D0000003B
:100BE000010000000000803F05010905A101A100EE
:100BF0000501093009310932093309350934094041
:100C000009381581257F750895088102C0C000004C
:100C100009022200010100E0320904000001030181
:100C200002000921110100012226000705830308A3
:100C3000000A00005D820008598200085582000801
:100C40004982000845820008518200084D82000850
:100C5000000004010000000000000002100000007D
:100C60000700000000000000010203040102030469
:100C7000060708094DD800084DD700089DDB00087D
:100C8000598300087D8A000869830008858300086D
:100C900031830008218300080000000000000000EC
:100CA0002D202D2D202D2D2D2D202D2D2D2D0000F5
:100CB000000000000000000000000000000000AA8A
:100CC000550B010000AA5505010000AA55090200B4
:100CD0000000AA5503009F0001000000C0120000A0
:100CE00001010000000001FFFFFFFFFF7EFF000089
:100CF000FFFFFFFF447F0020000000001C7F00205A
:100D000000000000207E06089C7D06080000000010
:100D1000AD320308A08601000400000000000000BE
:100D200000000000000000000000000000000000C3
:100D300000000000000000000000000000000000B3
:100D400000000000207E0608287E06080000000043
:100D5000F5380408E803000004000000000000006B
:100D60000000000000000000000000000000000083
:100D70000000000000000000000000000000000073
:100D800000000000307E06080000000000000000A7
:100D9000C93303087D000000FF00000000000000D0
:100DA0000000000000000000000000000000000043
:100DB0000000000000000000000000000000000033
:100DC0000000000010E10608000000000000000024
:100DD000953E03087D000000FF00000000000000B9
:100DE0000000000000000000000000000000000003
:100DF00000000000000000000000000000000000F3
:100E0000000000009C8B06080000000000000000AD
:100E10000D7303087D000000FF00000000000000CB
:100E200000000000000000000000000000000000C2
:100E300000000000000000000000000000000000B2
:100E400000000000387E06080000000000000000DE
:100E50005D430408E80300000300000000000000F8
:100E60000000000000000000000000000000000082
:100E70000000000000000000000000000000000072
:100E8000000000003C7E060800000000000000009A
:100E900075C80208102700000300000000000000D1
:100EA0000000000000000000000000000000000042
:100EB0000000000000000000000000000000000032
:100EC0000000000018DD0608000000005D170208A1
:100ED000598504085F76000005000000000000004E
:100EE0000000000000000000000000000000000002
:100EF00000000000000000000000000000000000F2
:100F000000000000B4E0060800000000000000003F
:100F1000F5A80408102700000100000000000000F0
:100F200000000000000000000000000000000000C1
:100F300000000000000000000000000000000000B1
:100F400000000000487E06080000000000000000CD
:100F5000F9380408E8030000050000000000000064
:100F60000000000000000000000000000000000081
:100F70000000000000000000000000000000000071
:100F800000000000547E0608000000000000000081
:100F9000813B0308204E0000030000000000000019
:100FA0000000000000000000000000000000000041
:100FB0000000000000000000000000000000000031
:100FC00000000000647E0608000000000000000031
:100FD00069390308204E00000300000000000000F3
:100FE0000000000000000000000000000000000001
:100FF00000000000000000000000000000000000F1
:1010000000000000747E06080000000000000000E0
:1010100071490408400D03000300000000000000B7
:1010200000000000000000000000000000000000C0
:1010300000000000000000000000000000000000B0
:1010400000000000847E0608000000000000000090
:101050007D020408102700000100000000000000CD
:101060000000000000000000000000000000000080
:101070000000000000000000000000000000000070
:1010800000000000C87D060800000000000000000D
:1010900075BA0108102700000300000000000000DE
:1010A0000000000000000000000000000000000040
:1010B0000000000000000000000000000000000030
:1010C000000000008C7E0608000000000000000008
:1010D0002D460208A086010001000000000000006B
:1010E0000000000000000000000000000000000000
:1010F00000000000000000000000000000000000F0
:1011000000000000947E06080000000000000000BF
:10111000DD41040850C30000010000000000000091
:1011200000000000000000000000000000000000BF
:1011300000000000000000000000000000000000AF
:10114000000000009C7E0608000000000000000077
:10115000C13D0408A861000001000000000000007B
:10116000000000000000000000000000000000007F
:10117000000000000000000000000000000000006F
:1011800000000000A87E060800000000000000002B
:10119000DDE10108A0860100010000000000000060
:1011A000000000000000000000000000000000003F
:1011B000000000000000000000000000000000002F
:1011C00000000000B47E06080000000000000000DF
:1011D0001DB80308A00F000001000000000000007F
:1011E00000000000000000000000000000000000FF
:1011F00000000000000000000000000000000000EF
:1012000000000000C07E0608000000000000000092
:10121000B56E01081027000001000000000000006A
:1012200000000000000000000000000000000000BE
:1012300000000000000000000000000000000000AE
:1012400000000000CC7E0608000000000000000046
:10125000316701081A410000010000000000000091
:10126000000000000000000000000000000000007E
:10127000000000000000000000000000000000006E
:1012800000000000D07E0608000000000000000002
:101290001D0B0108102700000100000000000000E5
:1012A000000000000000000000000000000000003E
:1012B000000000000000000000000000000000002E
:1012C00000000000B07D06080000000000000000E3
:1012D0008DEB010850C30000010000000000000079
:1012E00000000000000000000000000000000000FE
:1012F00000000000000000000000000000000000EE
:1013000000000000DC7E0608000000000000000075
:10131000D5960008400D030000000000000000000A
:1013200000000000000000000000000000000000BD
:1013300000000000000000000000000000000000AD
:1013400000000000E47E060800000000000000002D
:10135000A1B70308400D03000000000000000000DA
:10136000000000000000000000000000000000007D
:10137000000000000000000000000000000000006D
:1013800000000000EC7E06080000000000000000E5
:10139000F1C8010850C30000030000000000000075
:1013A000000000000000000000000000000000003D
:1013B000000000000000000000000000000000002D
:1013C00000000000F87E0608000000000000000099
:1013D000216D030840420F000000000000000000E3
:1013E00000000000000000000000000000000000FD
:1013F00000000000000000000000000000000000ED
:1014000000000000047F060800000000000000004B
:10141000F5B7030850C30000000000000000000002
:1014200000000000000000000000000000000000BC
:1014300000000000000000000000000000000000AC
:101440000000000001FF0100E00101000D80010823
:101450000000000000000000CCFB050808000000B0
:1014600000000000000000000000000070150608E9
:101470000000000000000000000000002816060820
:10148000000000000000000000000000D415060865
:101490000000000000000000ED970108B587002063
:1014A000010100009DD401080000000000000000C0
:1014B000FC160608C5D70108000000000000000067
:1014C000B41606082D202D2D202D2D2D2D202D2D4F
:1014D0002D000000000000000000000000000000DF
:1014E00000000000FFFFFFFF75AA010800000000D8
:1014F000000000000015060801000000FA000000CE
:1015000001000000010000005C8600200000F401E2
:10151000010000005A8600200000F40101000000D4
:10152000588600200000F4010100000056860020CB
:101530000000F40101000000548600200000F401C6
:1015400001000000528600200000F40101000000AC
:10155000508600200000F401010000000988010805
:10156000CD870108000000008001060840860020A9
:10157000053201004E8600206400F40101000000E5
:101580004C8600206400C409010000003E86002053
:10159000E803D007010000003C860020E803D007E4
:1015A000010000003A860020E803D0070100000097
:1015B000388600201E00B80B01000000468600207F
:1015C00005000F00010000004886002003000A000B
:1015D00001000000368600201E00F401010000001A
:1015E0004A860020020000000C0206083486002013
:1015F0001400640001000000428600203200E8036D
:1016000001000000328600200000C8000100000038
:101610003D85002000C801003C85002000500100ED
:101620003B850020005A010039850020020000009F
:1016300018020608D8820608E08206086A400020E0
:101640000100C40900000000684000200100C40936
:1016500000000000664000200100C40900000000F6
:10166000644000200100C409000000006040002028
:101670000100C40900000000624000200100C4090C
:10168000000000005E4000200100C40900000000CE
:101690005C4000200100C40900000000E782002037
:1016A00000C80100E682002000C80100E48200209A
:1016B0000000FFFF0A000000E28200200100C800D5
:1016C00001000000E082002032003075320000008E
:1016D000DE82002005820500DC82002005002C014E
:1016E00005000000DB820020055A0500D88200209A
:1016F00000FF0100DA82002002000000FC0C002044
:10170000D682002003000000B4F60508D78200202E
:1017100000FF0100D982002002000000FC0C002024
:10172000D582002003000000B4F605085D8701089B
:10173000ED860108000000002402060874860020DF
:10174000EE02CA08010000007286002000C80100F5
:10175000640000007186002000C8010064000000E1
:10176000708600200200000030030608C2820020BC
:101770000000803E05000000C082002080C1803E45
:1017800005000000BA8200200083007D05000000F3
:10179000B882002080C1803E05000000B382002096
:1017A00000FF0100AC8200206400F4010100000091
:1017B000AA820020040000003C030608A982002041
:1017C00002000000500306086D8300200D00000099
:1017D0005C0306086A83002000640100688300201F
:1017E000320010270A000000668300200D00000070
:1017F0005C030608658300200D0000005C030608FA
:10180000648300200200000094030608000000002A
:101810000000000000000000A00306087A860020F7
:101820003E000000D8030608788600200100FF7FF4
:10183000010000007786002002000000D4040608A2
:101840006F83002003000000E40406086E8300207C
:1018500003000000E40406082A850020000A0100B5
:10186000288500200000E8030100000026850020F4
:101870000000E80301000000248500200000E803C8
:1018800001000000228500200000E80301000000A4
:101890001A8500200000E8030100000020850020D8
:1018A0000000E803010000001E8500200000E8039E
:1018B000010000001C850020001401003885002074
:1018C00002000000F4040608368500200000F40140
:1018D00001000000348500200000F4010100000038
:1018E000328500200000F401010000003085002056
:1018F0000000F401010000002E8500200000A00F70
:10190000010000002C8500200000A00F0100000055
:101910001F860020196401001E86002002000000BE
:10192000000506081C860020E803D0070A00000016
:101930001A860020006401000A0000000F860020C3
:10194000006401000E86002000640100168600205D
:10195000006401000A0000001586002000640100F8
:101960000A00000014860020006401000A00000044
:101970001986002000FF01000A00000018860020E0
:1019800000FF01000A0000001786002000FF010090
:101990000A0000001386002001FF01000A00000079
:1019A0001286002001FF01000A00000011860020BD
:1019B00001FF01000A000000788300200000F4010C
:1019C00001000000768300200000A00F010000004D
:1019D000748300200000A00F01000000728300202B
:1019E0000000A00F01000000708300200000A00F85
:1019F00001000000FD87002000C80100FC870020D6
:101A000000640100FB87002000640100FA870020C9
:101A100000640100F987002000640100F8870020BD
:101A2000FF080100F78700200164010055860108C6
:101A300019860108000000000C0506080088002037
:101A400001320100FF870020010000007C0506082C
:101A5000FE8700200400000084050608F6870020A9
:101A600000640100F48700201400E8030100000076
:101A7000F2870020E80330750A000000F18700209B
:101A800000C80100F087002000C80100EF87002097
:101A900000C80100EE87002000320100028800200B
:101AA000004B010001880020040000009805060892
:101AB000ED870020006401000A000000108800206B
:101AC0000000D007010000000B88002000C80100C2
:101AD0000A88002000C801000988002000C8010011
:101AE0000E8800200000D0070100000008880020B8
:101AF00000C801000788002000C8010006880020F7
:101B000000C801000C8800200000D0070100000080
:101B10000588002000C801000488002000C80100DA
:101B20000388002000C801000D840108F583010826
:101B300000000000AC05060861830020005A010087
:101B40006083002000C801005E830020E803D00706
:101B50000100000000000000000000002D980108B6
:101B6000480606084D414D42414634303555530034
:101B7000D482002000030100D38200200003010072
:101B800031830108E5820108000000009C06060878
:101B9000A58201085D8201080000000038070608E0
:101BA0007D83010859AA010800000000B807060853
:101BB000C482002001030100E5880108B9880108FA
:101BC00000000000100B0608E18101089581010862
:101BD00000000000800B06081D8401080DE10108CB
:101BE000000000001C0C060861AE01081189010804
:101BF00000000000C40C06086D840108000000000D
:101C000000000000500D060849850108F184010814
:101C100000000000B40D0608DD850108A18501085B
:101C2000000000005C0E06083107020891860108DA
:101C300000000000E80E06083186002001060100C1
:101C4000B58401088184010800000000E40F060843
:101C500065060208F5AB01080000000054100608F4
:101C60007D070208BDAC010800000000A4110608B1
:101C70003086002001030100C58301089583010817
:101C80000000000078120608D907020800000000D2
:101C900000000000DC1206082D82010841AA01089C
:101CA000000000005C1306080000000000000000B7
:101CB00000000000E8130608C586010835AD0108DC
:101CC000000000005814060800000000000000009A
:101CD0000000000070160608745100209CFF2C01C3
:101CE00000000000A48C0020E0150C17000000008C
:101CF0004987002002000000A8160608A4820020E0
:101D000088136F1701000000A682002088136F1748
:101D1000000000005631002000000000000000001C
:101D2000543100200000000000000000523100206B
:101D30000000000000000000503100200000000002
:101D4000000000004E3100200000000000000000F4
:101D50004C3100200000000000000000A40300201F
:101D600000000000000000002C82002003000000A2
:101D7000981706089C82002088136F170100000046
:101D8000BE51002088136F1700000000D5800108A5
:101D90000000000000000000A81706084A87002085
:101DA00001000000FC170608C051002001000000DF
:101DB00008180608B6510020020000001018060896
:101DC0000000000000000000000000001C180608D1
:101DD000BD8001080000000000000000B8180608DF
:101DE0000000000000000000000000000C190608C0
:101DF0000000000000000000000000007C19060840
:101E0000A882002002000000B4190608BA51002080
:101E1000E0150C17000000007C950020D0950020F4
:101E200001D601FF010000000001010100000000D7
:101E30000000803F000000000000000000000000E3
:101E40000000000000000000000000000000000092
:101E500000000000000000000000803F00000000C3
:101E600000000000000000000000803F00000000B3
:101E700000000000000000000000803F00000000A3
:101E80000000000000000000010000000000FA4314
:101E90000000FA430000803FFFFFFFFFFF0000004B
:101EA0008D04040800000000000000000000000095
:101EB000000000003CB3002008000000000000000B
:101EC0002CB3002008000000FFFFFFFF010000000E
:101ED000A00F0000B80B00000102FFFF010000008E
:101EE000618A0008CD8800087DDB00080000000042
:101EF0001D83000839D7000819880008ADD60008EE
:101F00000000000000000000D98200086D82000877
:101F100061820008FDCD000819CE0008E1CD00085F
:101F2000C5CD0008A9CD0008198A0008A9880008B5
:101F3000C9DA000800000000F1820008B1D60008EC
:101F4000ED87000809D6000800000000000000002E
:101F5000E5820008685E0C0002FFFF00006002409E
:101F6000106002400000000000000000000B0000B4
:101F700000000000000000000000000000600240BF
:101F8000286002400100000000000000060C000074
:101F9000000000000000000000000000006002409F
:101FA000406002400200000000000000100D000030
:101FB000000000000000000000000000006002407F
:101FC000586002400300000000000000160E0000F0
:101FD000000000000000000000000000006002405F
:101FE000706002400400000000000000200F0000AC
:101FF000000000000000000000000000006002403F
:10200000886002400500000000000000261000006B
:10201000000000000000000000000000006002401E
:10202000A060024006000000000000003011000027
:1020300000000000000000000000000000600240FE
:10204000B86002400700000000000000362F0000CA
:1020500000000000000000000000000000640240DA
:102060001064024000000000000000000038000082
:1020700000000000000000000000000000640240BA
:102080002864024001000000000000000639000042
:10209000000000000000000000000000006402409A
:1020A000406402400200000000000000103A0000FE
:1020B000000000000000000000000000006402407A
:1020C000586402400300000000000000163B0000BE
:1020D000000000000000000000000000006402405A
:1020E000706402400400000000000000203C00007A
:1020F000000000000000000000000000006402403A
:102100008864024005000000000000002644000032
:102110000000000000000000000000000064024019
:10212000A0640240060000000000000030450000EE
:1021300000000000000000000000000000640240F9
:10214000B8640240070000000000000036460000AE
:102150000000000000000000000000000CDD060888
:1021600000000802050303000000000014DD06085B
:10217000010008020504030000000000E8A20608B0
:102180000200FE0101100300000000004C8606085A
:102190000300140200030000000000001CDD06081C
:1021A00004001F02020008000000000024DD0608F1
:1021B00005001F020201080000000000FFFFFFFFF2
:1021C0001A030000000000000000000000000000F2
:1021D00000000000000000000000000004030904EB
:1021E0001201000200000040830420570002010297
:1021F00003010000C13205084525050841250508F1
:102200003D250508E9340508392505083525050863
:102210004C6D0608BD89000889880008E5D80008CB
:102220000000000000000000E1D50008FDD4000817
:10223000000000000000000000000000958200087F
:10224000DD250508D1250508093A0508253A0508C0
:1022500089250508ED390508D13905081F0000005A
:102260001C0000001F0000001E0000001F000000F6
:102270001E0000001F0000001F0000001E000000E4
:102280001F0000001E0000001F0000000068214C1D
:10229000FF010000F4010000FF000000EC760608DA
:1022A0000000000000000000010203040607080906
:1022B0000100000080190020000000000000000064
:1022C000000000000000000000000000000000000E
:1022D00000000000000000000000000000000000FE
:1022E00000000000000000000000000000000000EE
:1022F00000000000000000000000000000000000DE
:1023000000000000000000000000000000000000CD
:082310000000000000000000C5
:082800000000000000000000D0
:108000002DE9F04700230F6801264FF0030C02E032
:108010000133102B41D006FA03F232EA0704F7D1FC
:10802000D0F800E05C000CFA04F52EEA050EC0F86A
:1080300000E091F80490D0F800A009FA04FE09F1DC
:10804000FF394EEA0A0EB9F1010FA846C0F800E068
:108050006FEA050515D8D0F808E005EA0E05856039
:108060004D79D0F808E0A54045EA0E0585604568E1
:1080700025EA020242608A7945689A4092B22A4310
:108080004260C26822EA0802C260CA79C568A2409A
:1080900001332A43102BC260BDD1BDE8F08700BF79
:1080A000074AD2E9003199421FBFD1180133097A3A
:1080B00001701DBFC3F30A03012013600020704745
:1080C000E0190020064AD2F80838D2F80C2893426A
:1080D00094BF4FF400600020013B9B1A1844704786
:1080E000E0190020012380F85130704707B501A83E
:1080F000FFF7D6FF0028FAD09DF8040003B05DF822
:1081000004FB044BD3E90003984288BF03F50063E6
:10811000181A7047E019002001207047024BC3F87D
:108120001028C3F814187047E0190020024BC3F858
:108130001828C3F81C187047E019002070477047D2
:1081400030B4124DD5E900239A4286BF03F500648E
:10815000A21A9A1A0A44B2F5006F11D899B10144D3
:108160004A1E013810F8014FE918824203F1010359
:108170000C72C3F30A03F5D16B60002030BC70476A
:10818000022030BC70470846F8E700BFE019002025
:10819000212838B50C4605D022282ED0202813D00F
:1081A000002038BD0029FBD0072AF9D11A4BD3F89B
:1081B000200893F8241893F8252893F8263820608F
:1081C00021716271A371EBE70029E9D0072AE7D199
:1081D000114DD5F814381BB10968D5F81008984727
:1081E000206821796279A379C5F8200885F82418D8
:1081F00085F8252885F82638D2E70029D0D0022A2C
:10820000CED1054AD2F81C38002BC9D00988D2F843
:1082100018089847C4E700BFE0190020024B00206F
:10822000C3F82808704700BFE0190020044B002065
:108230000522C3F82828C3F81C08C3F8140870479F
:10824000E0190020704700BF704700BF704700BFB3
:10825000704700BF704700BF704700BF704700BF46
:10826000042301480B8070478801002010B4074A9E
:10827000074B92F82C08122403F114020C800128F9
:108280000CBF184610465DF8044B7047E0190020FB
:108290008C010020202301480B807047B40100208E
:1082A00010B40C4A92F8303802EBC3010133DBB250
:1082B000042B4FF0050408BF00234FF4045081F84D
:1082C000344882F83038C1F838085DF8044B4FF074
:1082D000FF307047E0190020642301480B8070478D
:1082E000D4010020432301480B807047380200204E
:1082F00010B5084CD4F8F400FF2809D00649D1F88D
:10830000542801F65801FFF743FFFF23C4F8F43067
:10831000002010BD88010020E0190020E8E700BF20
:1083200008B5D0F8E4355B6A9847002008BD00BF67
:1083300008B5D0F8E4351B6A9847002008BD00BF97
:10834000D0F8E43510B504461B689847D4F8E835F2
:108350009B689847002010BD08B5D0F8E435DB696C
:1083600003B19847002008BD08B5042290F8121107
:10837000D0F8E83580F8131180F81221DB689847AF
:10838000002008BD10B5D0F8E83504461B699847B1
:10839000032384F81231002010BD00BF82B00023F7
:1083A000016801930B6901930E4B03E00A69019286
:1083B000013B13D0019A002AF8DA019A094B42F0E6
:1083C00001020192019A0A610A69019203E00A69B5
:1083D0000192013B02D0019AD207F8D4002002B0EA
:1083E000704700BF400D0300436D064A1A61C27812
:1083F000012A06D100F2CC5058614FF08022196852
:108400001A6070471800086070B44B78012B26D0B2
:108410000B784A6900EB83035C6D25682369D2B150
:108420008A684A6102F07F0223F4002323F07F036D
:1084300042F4002213432361C378012B04BF0B696C
:108440006361C5F3076363F07B0363F31F65256016
:10845000002070BC70478A6802F07F02E4E78269FE
:108460004C691568136944B38E68B4428CBF06F03A
:108470007F0404F07F0423F4002323F07F0344F4FB
:10848000002443EA040388BF4E611361C378012BC3
:108490001DD0C5F3076464F07B0464F31F651560A9
:1084A000002BD5D14B69002BD2D002690878516BD3
:1084B000012383400B435363CAE723F4002323F0D3
:1084C0007F0343F400231361C378012BE1D10B78C0
:1084D0000C6900EB8300C5F30763816963F07B03DC
:1084E00063F31F654C610020156070BC704700BFCE
:1084F0002DE9F0434B78012B30D00B784C6900EB21
:1085000083035E6D356837691CB38B681C44013C7E
:10851000B4FBF3F4C4F3090203FB02F3C3F3120345
:108520004B61144643EAC44363F31C073761C378C5
:10853000012B04BF0B697361CB78012B44D0C5F3C9
:10854000076363F07B0363F31F6535600020BDE8BC
:10855000F0838A680124C2F31203E3E791F80080F4
:108560004E6900EB880EDEF818C0DCF80050DCF82D
:10857000107076B3D1F80890384A06EB0904013C34
:10858000B4FBF9F402EAC444C6F312022243CC78E5
:1085900007F060473A43012C174649D0CCF8102029
:1085A000C278012A55D00269516B03FA08F30B43D4
:1085B0005363C5F3076363F07B0363F31F65CCF874
:1085C00000500020BDE8F0834B7973B345F00055AF
:1085D000B5E707F0604747F40027CC78CCF8107077
:1085E000C378012B2FD0012CE3D102699268D20508
:1085F00054BF45F0005545F08055C5F3076262F061
:108600007B0262F31F65CCF80050002B9ED1B0B204
:1086100003308010DEF8D04098D0CA6852F8041BAE
:10862000216001339842F9D190E745F0805586E703
:1086300064F35E77CCF81070C378012BD5D10A694A
:10864000CCF81420D1E70A69CCF81420012CB0D161
:10865000CBE70B69CCF81430ABE700BF0000F81F84
:1086600082B000230193019A094B42F0100201925B
:10867000C168019A0A610A69019203E00A690192DC
:10868000013B02D0019AD206F8D4002002B0704714
:10869000400D030082B000230193019A0B4B42F07E
:1086A00020020192019A61F38A120192C168019A33
:1086B0000A610A69019203E00A690192013B02D052
:1086C000019A9206F8D4002002B07047400D0300D2
:1086D0000B0617D401EB810300EBC30310B400EBCE
:1086E00081000124002283F8764383F8741383F811
:1086F0007523426D5DF8044B136843F400130020AA
:108700001360704701F07F0101EB810300EBC303AD
:10871000012200EB810083F81C1183F81E2183F8ED
:108720001D2182691368002B01DA43F0804343F472
:10873000001313600020704710B580210446FFF736
:10874000C7FF20460021FFF7C3FF2046BDE81040C9
:108750004AE600BF38B501EB810400EBC4040D46C6
:10876000002184F87453C4F88C1384F87513C4F88A
:108770008833C4F88023C3782821012B01FB05012D
:1087800008BFEDB201F55D7108BFC4F884231DB9BF
:10879000FFF73AFE002038BDFFF7AAFE002038BDE3
:1087A00070B5104BD3F8682893F8805804461AB176
:1087B00093F86C382B430DD081212046FFF788FFBA
:1087C000022D00D070BD2046074ABDE870401F232F
:1087D0000121BFE70121FFF77BFF20468121BDE892
:1087E000704075E7E01900204022002010B501EB31
:1087F0008101084A00EBC1010446B1F88C13104610
:10880000FFF79EFC034A204640230121FFF7A2FF09
:10881000002010BD64220020E8E700BF0B0630B442
:108820001CD401EB810200EBC202002300EB8105A6
:1088300082F8741382F8753301241A4604FA01F1A0
:108840006D6D61F31F4201696FF3CF332B60CB690C
:1088500023EA0203002030BCCB61704701F07F01A6
:1088600001EB810400EBC404012200EB810500232D
:1088700084F81C1184F81D2102FA01F11A46AD6931
:1088800061F30F02DFE700BF10B581210446FFF757
:10889000C5FF20460121FFF7C1FF024B002083F8EE
:1088A000C40810BDE019002010B581210446FFF76F
:1088B000B5FF20460121FFF7B1FF82212046FFF7D7
:1088C000ADFFFFF7ABFC002010BD00BF38B50D4673
:1088D00004468321FFF7A2FF29462046FFF7E4FF65
:1088E000002038BDF0B416460A063AD401EB8105E3
:1088F00000EBC5052824002204FB0104022B85F8A7
:108900007413C5F87C6385F8773385F8752304F50F
:108910005D7448D0154600EB8107012202FA01F18F
:108920007F6D61F31F45D7F800C01CF4004F11D1D3
:10893000E488204946F0805242F4004242EA8342F1
:1089400004F00F041C4B42EA845211400CEA03036A
:10895000194339600269D3692B430020F0BCD3610D
:10896000704701F07F0101EB810500EBC50528246C
:10897000012204FB0104022B85F81C11C5F82461B7
:1089800085F81F31A5F8221185F81D2104F58E7494
:108990000CD0002500EB8107012202FA01F1BF692A
:1089A00061F30F05BFE722711546B4E70025257175
:1089B000F0E700BFFF87CC13007833EC70B50446B6
:1089C000144EFFF761FF2046022340228121FFF76A
:1089D00089FF4022012120460223FFF783FFD6F8BA
:1089E000C83800251B6886F8C458284686F8805881
:1089F00098472046FFF734FE20460121FFF74AFE44
:108A0000204606F506621F230121FFF7A3FE284634
:108A100070BD00BFE019002010B5022304464022BB
:108A20008121FFF75FFF2046022340220121FFF74B
:108A300059FF8221204603230822FFF753FF064BEC
:108A400002229A83FFF7F2FB044A204640230121C9
:108A5000FFF780FE002010BD880100206422002066
:108A600038B508220D46044603238321FFF73AFF59
:108A700029462046FFF7D0FF002038BD002310B55F
:108A8000194604464022FFF72DFF8021204600238F
:108A90004022FFF727FFD4F8E835A078012284F8B8
:108AA00012215B689847002010BD00BF0E4BDA68AA
:108AB000D20310D4DA68D1060FD4DA68D20510D404
:108AC000DA6812F0E00F0AD1DB6813F0020F14BF6E
:108AD00008200920704701207047062070470720B2
:108AE00070470220704700BF003C0240024A536AB0
:108AF00023EA0000506270470038024000207047AF
:108B0000704730B1034B93F9CC080028D4BF002044
:108B100001207047E019002008B5FFF7F2FF60B1AF
:108B2000064A92F8CD3892F8CE285B0003F0020393
:108B3000002A18BF43F001030B6008BDE0190020B4
:108B400008B5FFF7DEFF18B1024BD3F8D0380B8021
:108B500008BD00BFE019002070B5FFF7D2FF90B14B
:108B6000094AB2F8D45875B1D2F8D8680023B34294
:108B70001C4608DA02EB44040133B4F8DC48AC428A
:108B8000DBB2F4D30B7070BDE019002008B5FFF71D
:108B9000B8FF10B100230B70137008BD042070479C
:108BA00028B1034B93F9F800003818BF0120704733
:108BB0008801002008B5FFF7F3FF50B1054B93F98A
:108BC000F820012AC3BF93F8FB30C3F340030B60C6
:108BD000002008BD8801002008B5FFF7E1FF18B1AB
:108BE000024B93F8FA300B7008BD00BF88010020DB
:108BF00070B5FFF7D5FF38B10E4C94F8FB30DB07AA
:108C000003D500230B70137070BD0B4D94F9F93030
:108C100095F8EC6893FBF6F301330B7094F9F94087
:108C200095F8EC1894FBF1F301FB13430133137037
:108C3000EAE700BF88010020E01900200320704708
:108C400070B50B4A92F8F03806255E1CB6FBF5F4B9
:108C500005FB146492F8F158AC421FBF02EBC3034A
:108C600082F8F048C3F8F408C3F8F81870BD00BFE4
:108C7000E0190020002230B504461046914200DC85
:108C800030BDA35C0825584010F0800F4FEA400328
:108C900018BF83F0D503013DD8B2F5D10132EDE71D
:108CA00010B5E9B10F4BD3F82409814218DCBAB1F1
:108CB000D3F8EC389A4213DC0B4C013A013903FB30
:108CC000012184F8061104F581700521FFF7D2FF18
:108CD000062184F8070104F58170BDE81040AFE774
:108CE00010BD00BFE019002088010020134B10B414
:108CF00000220F2483F82A19090A83F8290983F826
:108D00002B19C3F82C29C3F83029C3F8342983F868
:108D1000284903F62810012110F8014F013122449F
:108D20000E29D2B2F8D183F836290549D3F838098B
:108D30005DF8044B10223EF0F9BF00BFE01900209F
:108D400008230020054B002183F83C19C3F8401983
:108D5000D3F8383903B1C9E7704700BFE0190020E4
:108D60002DE9F0416C4C00234FF4F07220210646AF
:108D700004F6481084F8443955F0F1FE04F6283022
:108D80004FF4F072202155F0EAFE94F8090D10B16D
:108D900094F80A2D1AB900252846BDE8F0813FF065
:108DA0009BF80746C4F8140D3FF06AFB05460028FF
:108DB000F1D00FB12323FB80092138463DF05CFD43
:108DC000D4F8140D554F3FF06DFB94F80A0D01389F
:108DD00040B241F081FB0223102184F80C3DC4F81D
:108DE000100D4DF081FFB7F808114D4841F02AFAF7
:108DF000D4F8140D3FF050FBFF218C204EF0C2F848
:108E00008046D4F8140D3FF04DFBD4F8100D04212A
:108E10004DF06AFFB8F11B0F05D0D4F8140D2021D6
:108E20003DF02AFDB7E7D4F8143D012284F8442927
:108E30000BB12322DA80B7F80811394841F002FA61
:108E4000D4F8140D3FF028FB40210A204EF09AF888
:108E5000FF218A204EF096F8C0F38013D4F8140D49
:108E600084F8183D3FF01EFBD4F8100D04214DF09E
:108E70003BFF94F8083D012B44D0022B3AD0EBB3D2
:108E800094F8193D182B09D194F8182DB7F808312A
:108E9000A4F81C6DA4F81E2DA4F8203DB7F8081105
:108EA0001F4841F0CFF9B7F808111D4841F0CAF941
:108EB000D4F8140D3FF0F0FA022100204EF062F8D1
:108EC000D4F8140D3FF0EEFA0421D4F8100D4DF053
:108ED0000BFF94F8292D94F82A3D94F8281D84F866
:108EE000241DC2F12002C3F1100384F82B2D84F855
:108EF0002C3D51E70823A7F80831C1E71023A7F854
:108F00000831BDE7002EF5D094F8183D002B14BFB2
:108F100008231023EFE700BFE0190020880100209C
:108F2000EC260020F8B51A4C94F82D3D002BFBD10F
:108F300059B301444E1E451ED4F80C28D4F8081825
:108F400015F8017F531CC3F30A038B422CBF4FF467
:108F500000600020C91A224401440129C4F80C38D9
:108F600082F8307D0FD101203EF0D4F9D4F80838D2
:108F7000D4F80C188B4294BF4FF4006200225B1AA5
:108F80001344012BEFD0B542D6D10020F8BD00BF6D
:108F9000E01900200A4B0846D3F8281810B569B12B
:108FA000D3F82838052B09D1064C002AD4F83834D8
:108FB00004DD1146FFF7B6FFD4F8383410BD00BF0A
:108FC000E0190020D82A002010B590F85010002396
:108FD00080F8503089B10C4CD4F828287AB1D4F8F4
:108FE0002828052A0DD1094C3C30D4F83834FFF735
:108FF00099FFD4F83834012010BD0120FCE7104659
:10900000FAE71846F8E700BFE0190020D82A002048
:10901000002280F85120D7E790F85020531C0244DA
:10902000DBB280F8503082F83C1090F851200AB141
:10903000132B00D9C8E770472DE9F04FCD4DDFF86D
:109040006483DFF86C9384460F4616460FCD444682
:109050002DED068B0FC40FCD0FC495E807008BB024
:1090600099F83E34029684E80700CDE906C7042B40
:1090700000F26881DFE813F0B801660161010500C4
:10908000C8019FEDBD8ADFEDBD8ABD49C8F81C103F
:10909000BC49BD4BBD4AC8F818100299002918BF39
:1090A000134638EE887AF5EE006A86EE87AAC8F88D
:1090B0002430B74FB74B03930026DFEDB77A9FED0F
:1090C000B79A28EE278AF0EE679A079BB34200F022
:1090D0002E81039B13F8014B039306F1010B5FFAFA
:1090E0008BF2002C00F09381DFF8C8C2002303E06C
:1090F0000133152B00F08B8103EB43015D001CF85D
:109100000100A042F4D14944049291F85914002975
:1091100000F0858120463DF08FF803680593824674
:1091200018463DF075F89AF805103DF0C9F990F829
:1091300000E0BEF1000F40F06A8109EB050025094F
:109140000321013D049A059B80F899248D4280F803
:10915000981404F00F0C00F23381864800EB4500B0
:10916000808D40FA0CF414F0010400F03B810124DE
:1091700004FA0CF3013B1840049252F03DFA7D4B87
:10918000DFF834C2049A1D44032195F83430794D38
:1091900018440CEBC0037B619971DA715CF8300004
:1091A0009AF8082000F13F4101F57E0105EB91217D
:1091B00091F8381001F01F054909032904FA05F454
:1091C00000F00B81042900F00381022900F0FB80EC
:1091D0009B880893B3FA83F3C3F11F03C3F3CC0155
:1091E00000EB810103F007030C6A9B000F259D40F3
:1091F00024EA05040C620C6A02FA03F323430B62AF
:10920000022308A90993FEF7FBFEDAF80030029A60
:10921000002A00F0A180B9F83C2400EE102AB8EE34
:10922000C00AFCEEC07A17EE901A5D4A934200F035
:109230008E80A2F58062934200F0898002F5804220
:10924000934200F0848002F5806293427FD002F561
:10925000806293427BD0D9F84C2650084FF6FF73BA
:10926000B0FBF1F21A44120CB0FBF2F202980028A3
:1092700070D0B2FBF1F18BB299F83E0404280BBF19
:1092800007EE901A07EE902AF8EE677AF8EE676A12
:1092900005BF07EE102A67EEA97A66EE887AF8EE27
:1092A000476A29EE677A99F83F0406990091A6EE7D
:1092B000A87A019051463846C7ED027A87ED037AC5
:1092C0002CF0FCFF002E52DD7B68D8F8382093424A
:1092D00074D0012E4BD0D8F8502093426ED0022E7D
:1092E00045D0D8F86820934268D0032E3FD0D8F8F4
:1092F0008020934262D0042E39D0D8F8982093422F
:109300005CD0052E33D0D8F8B020934256D0062E2C
:109310002DD0D8F8C820D31A18BF01235E460122E9
:10932000082E3B747A7407F118077FF4CEAE1D48FF
:109330000BB0BDEC068BBDE8F08F9FED1B8AF0EE05
:10934000488AA2E69FED198AF0EE488A9DE6D9F890
:109350004C0683E719468FE7B0EE4A0A049353F0B0
:1093600053F8FCEEC07A049B17EE901A5DE70123D8
:10937000D4E700BF00EC0508ACC5A737ACC5A736DD
:109380009D330308313B0408DD2D0308253B040809
:10939000480000101B2F00206F12833A00007A440F
:1093A0000004014014000010282930386F120339DE
:1093B000D82A0020302F00209C2F00200023ADE76A
:1093C000C7F814E023E717494D6C2C434C64FFE6C3
:1093D00014490D6B2C430C63FAE612490D6C2C43B7
:1093E0000C64F5E67C6112E79FED0F8A0F4BC8F81D
:1093F000183000230E4A069301230293C8F81C205C
:109400000C4BF0EE488A4CE69FED0B8AEEE70B4AD8
:10941000084BC8F81C20C8F82430002088E70B68E7
:10942000FFDE00BF003802406F12833A313B040870
:109430009D330308253B040800000000D5300308D5
:10944000F8B50546262022F0C9FA134C0146F0B9BA
:10945000D4F8500690F838301E3B012B01D93EF06D
:1094600099FC0E4F0026AE4209DBB4F87436013386
:10947000A4F87436D4F83834C4F88436F8BD17F834
:10948000011BD4F850063EF085FC0136EBE70023C3
:1094900084F88236EEE700BFD82A00202C31002065
:1094A00038B5154C94F8F13894F8F0289A421CD04D
:1094B00004EBC303114AD3F8F418D3F8F8080023D7
:1094C000984213DC8B780E4A5B0882F88236C2F829
:1094D0008806FFF7B5FF94F8F13806210133B3FB96
:1094E000F1F201FB123384F8F13838BDCD5C02F89B
:1094F000015B0133E4E700BFE01900202C310020BC
:10950000D82A00202DE9F84F1B4C05461E2094F860
:109510008CA694F88DB694F88E66B4F89096B4F84C
:10952000928694F8947622F059FA30B1B8F1000F8F
:109530001EBFC14601264FF0000A94F89636DA079E
:109540000AD494F89B263AB9012F12D0022F03D1E6
:1095500013F0020F08BF012685F800A085F801B0BE
:10956000AE70A5F80490A5F806802F722846BDE8D5
:10957000F88F3E46F0E700BFD82A002013B5044616
:10958000FFF70EFB08B300230DF106022046ADF8ED
:10959000063013F09FFEC0B10D4C9DF8062094F9E3
:1095A000F81084F80E21032908BF62F07F024FF003
:1095B0000501084808BF84F80E21FFF75BFB062170
:1095C00084F80F010348FFF73BFB02B010BD00BF5A
:1095D00088010020920200202DE9F84F2DED028B2A
:1095E000FFF7DEFA002844D0254B93F9F800012854
:1095F0003FDD93F81041DFF890809FED228A0FF253
:10960000780BDBE900AB15468E1E02EB44094D4595
:1096100004D1BDEC028B2046BDE8F88F38F8027B00
:1096200026F8027F07EE907AF8EEE77A67EE887AFE
:1096300017EE900A51F0F0FB52465B4651F044FCA5
:1096400041EC100B54F0BCFF51EC100B51F064FFD7
:109650000E2F80B20AD919303223B0FBF3F080B25A
:1096600000EB800000EB8000400080B225F8020B88
:10967000CDE70024CDE700BF1655B5BBB16B024066
:1096800088010020CDCCCC3D9831002038B50D4666
:10969000FFF786FA044638B10C4890F8FB30DB0738
:1096A00004D5B0F8FC002880204638BD084A90F95F
:1096B000F93092F8EC2893FBF2F102FB11320132FF
:1096C000013100F58A7013F019FEECE788010020E3
:1096D000E01900202DE9F04FA94D95F8D0368BB058
:1096E0008146002B40F0B580D5F8D466002E00F0FE
:1096F000B080A44AD2F8184104F0F021B1F1E02F73
:109700006ED1C2F81831D5F8D826944268D00493A7
:109710000593ADF81830B5F8903695F88CE6ADF8AD
:10972000143095F88DC695F8943695F88EA68DF878
:1097300018300DF110088DF810E08DF811C08DF87B
:1097400012A098E8070007AB03C38F4F1A80C4F339
:1097500042533B44C4F3034293F83E10C5F8D84645
:109760008E4502F1010201D1944508D030468DF8B2
:109770001C108DF81D2013F0C1FDADF820003046FF
:1097800013F0F2FF032804F0070B34D0042836D07E
:1097900000239A4501A9304618BF8DF81E3013F0FA
:1097A00027FE48B1019BC4F3001103F001038B4273
:1097B00002D0304613F0CAFE0A2207A9404655F0EF
:1097C000A6F968B19DF81E30BDF81C2085F88E36CC
:1097D000BDF82030A5F88C26A5F8903643F0F4FEAD
:1097E00095F8DCA604AF95F8DC36032B7BD8DFE8D0
:1097F00003F00A3376A35F4497F84330C9E75F4428
:1098000097F84B30C5E73946304613F0F7FD04466C
:1098100058B107A8FFF776FE9DF81E109DF810308E
:109820008B4260D0304613F007FF95F8DC360133E9
:1098300003F0030385F8DC360CB99A45D3D195F8CB
:109840009636DB0700D524B1336849461B6830469D
:1098500098470BB0BDE8F08F01A8FFF753FE95F8CD
:1098600096869DF8044008F00108ECB1B8F1000FAD
:1098700039D13A460DF10301304613F0C2FD0446DA
:1098800088B307A8FFF73EFE9DF81C109DF8033033
:109890009DF81D208B4203D19DF81030934222D0B9
:1098A000304613F0D3FEC0E7B8F1000FBDD1394602
:1098B000304613F0A0FD0446A8B107A8FFF722FE2A
:1098C000BDF82010BDF810308B420CD085F8DD8635
:1098D00085F8DE86336830469B699847A5E795F89A
:1098E0009636D80701D500249FE707A9304613F024
:1098F0007FFD04460028F6D01E2022F06FF895F870
:10990000DF3683428046EED085F8DF0660B1B5F8D9
:109910009236002BE7D1079BD907E4D401213046CA
:1099200013F014FE444680E7079BDA07DBD50146B7
:10993000304613F00BFE78E73846FFF7E3FD97E873
:10994000070007AB03C31A809DF810309BB10DF1DF
:109950001D0207A9304613F054FD0DF11E013046DB
:1099600013F04CFD0A2207A9384655F0D0F8041E22
:1099700018BF012459E708A9304613F03CFDECE775
:10998000D82A00208801002000EC050800F01F0202
:1099900040090123032803FA02F304D004280CD061
:1099A000022805D07047074A116C0B4313647047B7
:1099B000044A516C0B4353647047024A116B0B43CA
:1099C000136370470038024000487047FC2F0020A6
:1099D00000285FD00368374A2DE9F04103F13F4486
:1099E00004F57E0402EB9422012492F8382002F060
:1099F0001F055209032A04FA05F456D0042A4FD051
:109A0000022A48D08588B5FA85F0C0F11F00C0F35E
:109A1000CC0603EB860600F0070082000F24306AB4
:109A2000944020EA04003062306A01FA02F20243F4
:109A3000002132624FF0010E0A464FF0030C02275C
:109A40000EFA02F838EA050002F101021CD118688A
:109A50000CFA01F420EA04001860186807FA01F60D
:109A600006431E609E6826EA04069E609868986019
:109A7000586820EA0800586058685860D86820EA9A
:109A80000400D860D868D860102A01F10201D7D14B
:109A9000BDE8F0817047084A556C2C435464B1E727
:109AA000054A156B2C431463ACE7034A156C2C4331
:109AB0001464A7E700EC0508003802402DE9F047E0
:109AC000C94C94F8E0160546C1F34001D4F8E80605
:109AD0003EF0EEFC94F8E016D4F8E406C94301F039
:109AE00001013EF0E5FC002D00F0E58005F1FF38B6
:109AF000BE4EBF4D5FFA88F81027D4F8E83633B170
:109B00001A689B8851690B4214BF53831383D4F89E
:109B1000E43633B11A689B8851690B4214BF5383F2
:109B20001383B4F8F036002B40F0558194F8F21608
:109B3000D4F8F4063EF0BCFC4FF0FA0C4FF47A7007
:109B40004FF0010E7368C3F30803002B40F0178138
:109B5000EFF31183002B40F01281D4F83824A96868
:109B6000D4F838349A42F8D1D4F818379942F4D856
:109B7000D4F8149700FB09F35B1AB3FBF9F300FB6D
:109B800002327368C3F30803002B40F0B780EFF391
:109B90001183002B40F0B280D4F83834D5F808A0F7
:109BA000D4F838148B42F7D1D4F818178A45F3D873
:109BB000D4F8149700FB09F1A1EB0A01B1FBF9F10C
:109BC00000FB03139B1AB3F57A7FDAD3BCF1010CC7
:109BD000B8D1D4F8E83633B11A689B8851690B4282
:109BE00014BF53831383D4F8E43633B11A689B88C7
:109BF00051690B4214BF53831383B4F8F036002B22
:109C000040F0DD8094F8F216D4F8F40681F00101FA
:109C10003EF04EFC4FF0FA0C4FF47A704FF0010E0C
:109C20007368C3F30803002B40F08980EFF31183BE
:109C3000002B40F08480D4F83824A968D4F8383454
:109C40009A42F8D1D4F818379942F4D8D4F8149736
:109C500000FB09F35B1AB3FBF9F300FB02327368F4
:109C6000C3F308034BBBEFF3118333BBD4F8383491
:109C7000D5F808A0D4F838148B42F7D1D4F81817C7
:109C80008A45F3D8D4F8149700FB09F1A1EB0A0137
:109C9000B1FBF9F100FB03139B1AB3F57A7FDED316
:109CA000BCF1010CBCD108F1FF385FFA88F8B8F1BB
:109CB000FF0F7FF422AFBDE8F087EFF3118987F340
:109CC0001288D5F808A02B68DB0344BFC4F810E75E
:109CD000D5F808A0D4F83834D4F810175FFA89F909
:109CE00089F31188D4F814970B4400FB09F1A1EB18
:109CF0000A01B1FBF9F100FB0313CDE7EFF3118982
:109D000087F31288D5F808A02B68D90344BFC4F89C
:109D100010E7D5F808A0D4F83834D4F810175FFA53
:109D200089F989F31188D4F814970B4400FB09F1E1
:109D3000A1EB0A01B1FBF9F100FB031342E7EFF3DA
:109D4000118187F31288D5F808902B68DA0344BF95
:109D5000C4F810E7D5F80890D4F83834D4F81027B0
:109D6000C9B281F31188D4F814171A4400FB01F327
:109D7000A3EB0903B3FBF1F300FB02326FE7EFF350
:109D8000118187F31288D5F808902B68DB0344BF54
:109D9000C4F810E7D5F80890D4F83834D4F8102770
:109DA000C9B281F31188D4F814171A4400FB01F3E7
:109DB000A3EB0903B3FBF1F300FB0232E1E6D4F8B5
:109DC0000C37002B3FF426AFD4F8F826002313609D
:109DD00084F809371EE7D4F80C37002B3FF4ACAEFB
:109DE0003DF05CFBA8E600BFD82A002000ED00E0B3
:109DF00010E000E02DE9F84FC44CC54F94F8E01690
:109E0000D4F8E806C34DC1F340013EF051FB94F88D
:109E1000E016D4F8E406C94301F001013EF048FB26
:109E20004FF0050B4FF01008D4F8E83633B11A683C
:109E30009B8851690B4214BF53831383D4F8E436D3
:109E400033B11A689B8851690B4214BF5383138343
:109E5000B4F8F036002B40F0518194F8F216D4F8A3
:109E6000F4063EF025FB4FF0320C4FF47A700126D9
:109E70007B68C3F30803002B40F01481EFF31183D8
:109E8000002B40F00F81D4F83824A968D4F8383476
:109E90009A42F8D1D4F818379942F4D8D4F81497E4
:109EA00000FB09F35B1AB3FBF9F300FB02327B689A
:109EB000C3F30803002B40F0B480EFF31183002BB1
:109EC00040F0AF80D4F83834D5F808A0D4F838146E
:109ED0008B42F7D1D4F818178A45F3D8D4F81497E1
:109EE00000FB09F1A1EB0A01B1FBF9F100FB03133F
:109EF0009B1AB3F57A7FDAD3BCF1010CB8D1D4F850
:109F0000E83633B11A689B8851690B4214BF5383FA
:109F10001383D4F8E43633B11A689B8851690B4235
:109F200014BF53831383B4F8F036002B40F0DA806B
:109F300094F8F216D4F8F40681F001013EF0B8FA74
:109F40004FF0320C4FF47A7001267B68C3F308039C
:109F5000002B40F08780EFF31183002B40F08280CC
:109F6000D4F83824A968D4F838349A42F8D1D4F80F
:109F700018379942F4D8D4F8149700FB09F35B1A08
:109F8000B3FBF9F300FB02327B68C3F308033BBB6E
:109F9000EFF3118323BBD4F83834D5F808A0D4F8F4
:109FA00038148B42F7D1D4F818178A45F3D8D4F86F
:109FB000149700FB09F1A1EB0A01B1FBF9F100FBD9
:109FC00003139B1AB3F57A7FDED3BCF1010CBCD12D
:109FD0000BF1FF3616F0FF0B7FF426AFBDE8F88FCC
:109FE000EFF3118988F31288D5F808A02B68DB03FA
:109FF00044BFC4F81067D5F808A0D4F83834D4F8B2
:10A0000010175FFA89F989F31188D4F814970B4473
:10A0100000FB09F1A1EB0A01B1FBF9F100FB03130D
:10A02000CFE7EFF3118988F31288D5F808A02B68E1
:10A03000D90344BFC4F81067D5F808A0D4F8383461
:10A04000D4F810175FFA89F989F31188D4F81497B6
:10A050000B4400FB09F1A1EB0A01B1FBF9F100FB94
:10A06000031345E7EFF3118188F31288D5F80890C0
:10A070002B68DA0344BFC4F81067D5F80890D4F809
:10A080003834D4F81027C9B281F31188D4F81417E2
:10A090001A4400FB01F3A3EB0903B3FBF1F300FB4C
:10A0A000023271E7EFF3118188F31288D5F8089036
:10A0B0002B68DB0344BFC4F81067D5F80890D4F8C8
:10A0C0003834D4F81027C9B281F31188D4F81417A2
:10A0D0001A4400FB01F3A3EB0903B3FBF1F300FB0C
:10A0E0000232E4E6D4F80C37002B3FF429AFD4F861
:10A0F000F8260023136084F8093721E7D4F80C37D9
:10A10000002B3FF4B0AE3DF0C9F9ACE6D82A0020F0
:10A1100000ED00E010E000E010B4B8B10D4CD4F850
:10A120001C37102B05D15DF8044B052100203CF0B5
:10A130008BBE03EB4302224482F8211701210B441A
:10A1400082F8200782F82217C4F81C375DF8044B08
:10A15000704700BFD82A0020F8B5274E00EBC00496
:10A1600006EB8404D4F85457002D38D094F865C712
:10A170000CF0FF07BCF1000F31D149004FF0010C8A
:10A18000C9B284F8661784F8672784F869C784F829
:10A190006A7784F868C784F865C784F86477AA8802
:10A1A000C4F86C37C4F87037940502D501273846D7
:10A1B000F8BD2B88D9050CD44FF4805301E0013B46
:10A1C00010D02A889205FAD42B889BB243F480736E
:10A1D0002B80AB889BB243F44073AB80E6E700274B
:10A1E0003846F8BDB6F8BC3701339BB2A6F8BC3789
:10A1F00050F004F8DBE700BFD82A002070B44E4AC4
:10A2000092F8BE3703EB430002EBC000590090F810
:10A21000C00703281ED8DFE800F00E200250C8183F
:10A2200002EBC000D0F8C4470CB3013CC0F8C447EF
:10A23000002070BC7047414890F82061002E63D028
:10A240003F4C002001E086425ED0258801308C34EE
:10A25000002DF8D0012070BC7047C81802EBC00078
:10A26000D0F8C447002CE0D1022480F8C04719443C
:10A2700002EBC10191F8CC070138C0B281F8CC07DC
:10A28000B0BB304892F8805CD0F81C01D1F8C847C8
:10A29000013303F00303421E0326AB42224481F83C
:10A2A000C067B2FBF0F4C1F8C447D3D090429CBF62
:10A2B00004F1FF34C1F8C447CCE7194402EBC101F3
:10A2C000D1F8C40790BB92F8801C8B42C2D00133F6
:10A2D00003F00304A14282F8BE47BBD004EB440361
:10A2E00002EBC3020223C2F8C40782F8C037B2E708
:10A2F000144BD3F81C21012002F2E73370BCB3FBEE
:10A30000F2F3C1F8C43770470E480B44D0F81C1163
:10A3100002EBC302012001F51C530F3370BCB3FBE9
:10A32000F1F382F8C007C2F8C43770470138C1F8AA
:10A33000C40700208FE700BFD82A002014000010B7
:10A34000F83200208801002070B5244D95F8844C27
:10A35000022C134682B00A4607D0014605F6844017
:10A3600002B0BDE8704040F0C3B8D5F88C1C11B104
:10A370000C6889886183D5F8881C8E8940F2E9349D
:10A380000E89013C16F0020FA4B223D084B28C8156
:10A3900040F2E9340889013C10F0010FA4B20DD05D
:10A3A0008889084600214DF0DDFFD5F88C3C13B1BB
:10A3B0001A689B881383012002B070BD002CE9D17C
:10A3C0000846CDE900233FF089FFDDE90023D5F8F9
:10A3D000881CE6E7002CD3D1F2E700BFD82A002082
:10A3E00030B40578022D14D0012D02D0002030BCED
:10A3F0007047044690F90400084B421C83F8C45C83
:10A40000F4D00328F2DC0A4603F6C443617930BC79
:10A41000A2E630BC012240F00DB800BFD82A0020CF
:10A420002DE9F04F2DED108B034697B004331593B3
:10A43000DFEDCACA149002238A4613928B46129308
:10A44000149C4FEADB0604EB461202EB06103101C6
:10A45000A6EB86034FEAC60806EB4605CDE90001E8
:10A4600000EBC303043108F1040011962044214499
:10A470002C01C6EBC60C0394EC00119D04944FEA2A
:10A48000CC0405946C0106EB860E0294159D009C8D
:10A4900003EB46174FEACE0E02EBC6064FEACB0996
:10A4A0004FF0000C51ED01AAD3ED001A92ED007AA5
:10A4B00094ED005A96ED004AD7ED007A15ED012A89
:10A4C00050ED016A32EE07BA76EE840A7AEE855ACA
:10A4D00031EEA70A3BEE256A70EE804A76EEC46A3A
:10A4E00036EE244A36EE646A05ED014A82ED006AD2
:10A4F000D0ED00BAD6ED012AD3ED019A95ED00AA70
:10A5000092ED016A97ED013A91ED00CAD4ED014A4E
:10A510007BEEE23A36EEE19A32EE472A73EEE98AB2
:10A520003AEE464A39EE279A78EE838AB0EE428AAE
:10A53000A9EE6C8ADC44E24573EEC33AB0EE441AED
:10A54000A8EEEC1A76EEE77A33EEA97A7CEE643A5E
:10A5500077EEA17A3AEE066A7AEEC51A3CEE24AAA4
:10A5600074EECC4A39EE833A35EE6A5AF0EE639ACD
:10A57000F0EE48AAE7EE2C9AA8EEAC4AE7EE2C4A99
:10A58000E7EE6CAAF0EE418AB0EE427AB0EE612AB4
:10A590007BEE656A7BEEA22A76EE4A5AA9EE2C7A09
:10A5A000A7EEAC2AA7EEAC5AE7EEEC8A32EE83BAFD
:10A5B00076EEC3BA35EEE09A75EEC07A36EE0A6AE8
:10A5C00076EEE26A36EE0BAA76EE836A77EEA07A32
:10A5D00034EE423A77EE290A36EE4B6A7BEEA22A37
:10A5E00039EE000A73EEAA3A78EE244A37EE697A19
:10A5F00031EE055A71EEA85A32EE044A85ED00AAF2
:10A6000082ED016A4D4441ED012A4A44C4ED006ADD
:10A6100081ED000AC4ED017A494440ED010A4C4441
:10A6200087ED007AC6ED003AC3ED004A80ED003AAE
:10A6300087ED014A484486ED015A4F44C3ED015A63
:10A640004E444B443FF62EAF119B072B40F2C7817F
:10A65000029D149E019B03980499059A083575196B
:10A660000C330E95354608F108080EF10804EB1876
:10A6700008300831083246442C1928186918AA18DD
:10A68000079305F10C030D960C940B900A91099217
:10A6900008934FF001084FF0000E129B9E44139B4D
:10A6A00003EBCE0303EBCE02109302EBCE0303EBDE
:10A6B000CE01029101EBCE0101EBCE0505EBCE06FA
:10A6C000D6ED007A0F93AEEB8E03019106EB0313E8
:10A6D00003EBCE07D3ED01AACDED067A019BD5EDB4
:10A6E000007A97ED01BACDED057AD3ED007A029BA1
:10A6F000CDED047AD3ED007A0F9BCDED037A07EB15
:10A70000CE0CD3ED007ADCED01BACDED027A0CEB84
:10A71000CE01D2ED007A109A009101EBCE000146F5
:10A7200091ED01DACDED017A0099D2ED007A91ED4B
:10A7300001CA00EBCE0000EBCE0494ED01EAD0EDAF
:10A7400001DACDED007ADDE90776DDE90954DDE9CE
:10A750000B01DDE90D23C44602E000BFF304353FE1
:10A7600094ED009A90ED00FA91ED006AD5ED007A33
:10A77000D3ED006A57ED014A92ED005A56ED013AC9
:10A7800096ED00AA35EE060A73EEA65A39EE278A30
:10A7900034EE8F7A70EE082A75EE87EA35EE465A67
:10A7A0003EEEA26A73EEE63A06ED016AD1ED019A39
:10A7B000D2ED01FAD4ED016AD3ED011A95ED013A1B
:10A7C000D0ED018A97ED004A3FEEE96A35EE491A6D
:10A7D00076EE660A31EE271A3AEE612A75EE677A4E
:10A7E00070EE830A3FEEA95A74EECF9A77EE897A1B
:10A7F0007AEE211AB0EE42AA74EE68FAA0EEECAA44
:10A80000DC44E24535EEC77AB0EE639A74EE285A1E
:10A8100038EEC44AF0EE698AA1EE6C9AE7EEAC8A93
:10A8200036EE436A7FEE644A36EE266AA0EEAC2A24
:10A83000F0EE4A0AE7EEEC0AE7EEAC4AF0EE687A90
:10A84000F0EE498A36EE833AE6EE6C8AE1EE2C3A77
:10A85000B0EE6F1AA6EE2C1A71EEE56AA6EE2C4A3F
:10A8600071EEA55A75EE031A7EEEE22A37EE43FA30
:10A8700075EEE1EAB0EE686A76EEC08A39EE044A17
:10A880007FEE86FA76EEC86A33EE816A38EE888A01
:10A8900073EEC13A37EE457A2CEE2E1A3FEE055A8A
:10A8A00022EECC9A9DED03FA70EE266A33EE077A1B
:10A8B000AFEE221AAFEE2E9A7AEE244A9DED01FAFF
:10A8C00079EEA09A25EE4BAA72EE670A37EE822A3D
:10A8D0006BEE087AAFEE08AAEFEE057A2DEEA63AF7
:10A8E0009DED05FA67EE6D8AAFEE073AEFEE268A28
:10A8F00066EE6A2A9DED00FA2AEEA00AEFEE202A03
:10A900006EEE02EADDED060A23EECE5AE0EEA3EA91
:10A910002BEEA98ADDED023AAFEE060AA3EE848A99
:10A9200024EE6B7A6DEE246A9DED044A2FEECD6A1B
:10A93000A0EE825AA3EEA97AE4EE2F6AA4EE246A6E
:10A9400075EEA15AC6ED005A83ED001A83ED019A07
:10A950004E4447ED017A87ED00AA4B4480ED003A62
:10A96000C0ED018A4F4482ED000A4844C2ED012A3D
:10A97000C5ED00EA85ED015A4A44C1ED006A81ED5A
:10A98000016A4D4484ED008A84ED017A49444C44C7
:10A990003FF6E6AE0E9B08330E930D9B08330D93E6
:10A9A0000C9B08330C930B9B08330B930A9B0833C7
:10A9B0000A93099B08330993089B08330893079B64
:10A9C00008330793119B08F1010843457FF465AEF6
:10A9D000129BDDF844B0DB009BB2129330E517B058
:10A9E000BDEC108BBDE8F08F0848002302461178BB
:10A9F000022902F1060204D00133062BF7D1002010
:10AA0000704703EB430300EB43007047A03700207F
:10AA1000F0B59F4C85B0242204F6C840002154F0C4
:10AA20009EF894F8ED6C002E3CD13546D4F8003DEC
:10AA30006BB39B6A5BB39748984783683BB30388C3
:10AA4000DFF878C2013B9BB260466646002137784A
:10AA5000032F06F106061DD001310629F7D1002289
:10AA60000178022900F1060000F0A6800132062AD2
:10AA7000F6D1D4F8281D052909D0481C02FB01C2D3
:10AA8000C4F8280D022000219380107051802846C0
:10AA900005B0F0BD062303FB0141B1F8CA3C013B00
:10AAA0009BB2DCE794F8EC0C04F6F443C4F8F03CF9
:10AAB00008B90025BAE73DF00FFA0746C4F8FC0CC8
:10AAC0003DF0DEFC05460028F3D0013E022370B2C3
:10AAD00084F8F43C3FF000FD0028EAD0C4F8F80CFC
:10AAE0000FB12023FB80092138463BF0C5FED4F886
:10AAF000F03C98683DF0D6FCD4F8F03C1021586842
:10AB00004CF0F2F8644BD4F8F02CC4F8202D93E804
:10AB100003000123009032208DF8041084F8243DB6
:10AB200000263CF0F7FB052302AA6946D4F8F00C96
:10AB30008DF80A608DF809603FF0BCFB9DF80A2093
:10AB40009DF809009DF80B10544B120242EA004296
:10AB50000A439A4200F0938032DCA3F5F1139A4243
:10AB60005FD043DD4E4B9A4253D002339A4263D1B9
:10AB70004FF400724FF48073A4F8042DA4F8103D34
:10AB8000B4F8102DB4F8043D120202FB03F30020C8
:10AB90004FF48071B3F1807FC4F8082DC4F80C3DE8
:10ABA00084F8120DA4F8061D58D83E4BC4F8003D99
:10ABB000012284F8192D39E7062101FB02C261E761
:10ABC000394B9A4235DC053B9A4235DD374B13440D
:10ABD000032B4CD801A252F823F000BF23AC00088D
:10ABE00013AC000805AC000871AB0008A3F5220304
:10ABF000013B9A423BD02DDD2D4B9A4209D00133C7
:10AC00009A4219D14FF48073A4F8043DA4F8103D82
:10AC1000B6E780224FF48073A4F8042DA4F8103D09
:10AC2000AEE740224FF48073A4F8042DA4F8103D41
:10AC3000A6E7204B9A42E5D0002594F8EC0CA4F846
:10AC4000045DA4F8105DC4F8085DC4F80C5D3FF025
:10AC5000D7FAEBE6184B9A42D4D0EDE70123D4F8AB
:10AC6000200D84F8183DB7214BF022FB9DE72022F0
:10AC70004FF48073A4F8042DA4F8103D80E74FF43E
:10AC800080621023A4F8042DA4F8103D78E700BFDB
:10AC9000D82A0020D837002054EC05081640E000E0
:10ACA0001720C2005CEC05081940EF00EABF10FF56
:10ACB00017BA20001870EF0018600100A0370020BC
:10ACC00099B10A6B824216D9154BD3F85C2D91428B
:10ACD00021D34C3991421ED30B6B9842F9D38B6B25
:10ACE0009842F6D80B46184670470D4BD3F85C1DBA
:10ACF0000A6B904212D30B680BB9F4E70A6B9042CF
:10AD00000B4602D38A6B9042EDD951F84C3F002B91
:10AD1000F4D1184670470023184670470A46D8E712
:10AD2000D82A00202DE9F047CC0143D10346224A1E
:10AD300043F8082B4FF0FF324260022418467E266B
:10AD4000DFF87880D8F8609D2644013E051D49460D
:10AD50006FF070474FF0010A08E0A3421CD0631C5B
:10AD600045F8043C321B1C460435CAB10B6BA342A8
:10AD700002D88B6BA34204D22046FFF7A1FF014605
:10AD800090B10A794B6B002AE7D1A34204D0E6D2F6
:10AD900045F8042C631CE5E745F8047C631CE1E7F7
:10ADA000C8F8601DBDE8F08745F804AC321B631C91
:10ADB0004946D8E78026C3E7F8FFFF0FD82A0020CE
:10ADC000F0B40D6800240CE0BCF1050F18D8A0F118
:10ADD00037030A2B14D104EB840415F8010B03EBA1
:10ADE0004404A0F13003DEB2092EA0F16107A0F106
:10ADF000410CF0D9052FE7D8A0F157030A2BEAD070
:10AE00000D601460F0BC7047036870B55E6A26B1CF
:10AE100033460522BDE87040184704460D464E1DD6
:10AE200000E023689B68204698470028F9D02368F3
:10AE300015F8011B1B6820469847B542F1D170BD3B
:10AE40002DE9F047154B054603F67454002093F99D
:10AE50006D8D84B06F1804F5287A06464FF0B60958
:10AE60002368ABB193F83830142B11D0B8F1FF3F01
:10AE700001D043450CD1002269462046CDE9026647
:10AE8000CDE90057ADF808908DF80E602CF0FAF877
:10AE9000E034A245E4D104B0BDE8F087D82A002010
:10AEA0002DE9F743124E0124A02318255FFA84F8F8
:10AEB000FF2B14DC56F8E40CE9B2C1F11C028272DB
:10AEC0005F1C026880F80B80DBB20093C1F11B01AC
:10AED000D2F8189000234246C9B2C8473B46013D0C
:10AEE000E6D10134052CE0D103B0BDE8F08300BF0A
:10AEF000D03B002010B50A4C14F8C70C003818BF1E
:10AF00000120FDF72DFF50B10649A4F1E0003FF00C
:10AF100007F9A4F1E0000EF011FFA4F1E00010BD6C
:10AF2000D03B002088EC050870B4447941BB03682D
:10AF30004FF400524FF40076202502213CBB1A8CBE
:10AF400022F001021204120C1A841A8B188C22F0BF
:10AF5000F30280B2120420F00A00120C014342F006
:10AF6000010241F001011A8319841A8B22F00C02AC
:10AF70001204120C1A831A8B92B270BC1A83704797
:10AF800000220368164615461146002CD7D0042C23
:10AF900021D0082C38D0198C21F480510904090CD7
:10AFA00019849C8B1D8C45F6FF7040F6FF412840AC
:10AFB0002140024342F4805241F4807199831A8403
:10AFC0009A8B22F440621204120C9A839A8B92B2EA
:10AFD00070BC9A8370471A8C22F010021204120C73
:10AFE0001A84188B198C89B240F6FF4221F0A00117
:10AFF00002400D4342F4807245F010051A831D840F
:10B000001A8B22F44062B3E71A8C22F48072120485
:10B01000120C1A84998B1A8C21F0F30192B2090454
:10B0200022F42062090C324342F4807241F00101A3
:10B0300099831A849A8B22F00C02C4E70B88F0B42F
:10B0400033BB028C4C880E898B88C98822F00102A0
:10B050001204120C0284058B028CADB225F0F305AC
:10B0600092B22B4322F00A0243EA061322439BB218
:10B0700042F0010203830284038B23F00C031B04C0
:10B080001B0C0383038B9BB21943F0BC01837047F5
:10B09000042B048C2CD0082B4E888A880D89C988F3
:10B0A00051D024F480542404240C0484838B078C12
:10B0B0002C0344EA022440F6FF421A4045F6FF738F
:10B0C0003B4043EA063322439BB292B243F480539F
:10B0D00082830384828B22F440621204120C8283E6
:10B0E000838B9BB243EA01239BB2F0BC83837047FE
:10B0F00024F010042404240C4D880F898A88C98800
:10B100000484068B038C12029BB242EA073423F0BC
:10B11000A00340F6FF42324043EA051322439BB2AC
:10B1200092B243F0100302830384028B22F4406244
:10B130001204120C0283038B9BB243EA01239BB2DD
:10B14000F0BC0383704724F480742404240C04842A
:10B15000848B038CA4B29BB224F0F30423F4206309
:10B16000224343EA062342EA05129BB243F480736A
:10B1700092B282830384838B23F00C031B041B0C89
:10B180008383838B9BB21943F0BC8183704700BFDC
:10B19000094B93F83E34042B08D9053B032B08D800
:10B1A00001231A4600B103701046704700230122A4
:10B1B000F8E700231A46F5E7D82A00202DE9F047E2
:10B1C0009AB0DDE9226ADDF8909004460D461746F4
:10B1D000984602E020683CF0D1FD20683CF0D6FDA6
:10B1E0000028F7D10146642201A853F0B8FC264B91
:10B1F0008DF80450CDF85CA00293002D3FD0AB1E1B
:10B20000012B3ED9042D14BF002203221F4B0396AD
:10B21000D3F838348DF805201E440123CDE9059478
:10B2200004968DF85B3037B14246394607A853F093
:10B2300035FC8DF85A80164E16F8769C002318932C
:10B24000B9F1000F18D116F8770C642202FB0060E8
:10B2500001A9743853F022FC012306F8779C06F804
:10B26000763C236843B143463A46294620461AB005
:10B27000BDE8F04711F01ABB1AB0BDE8F08705220F
:10B28000C4E70222C2E700BF183B0020D82A0020F2
:10B29000D03B00209FED737A07EE901A20EE070A4C
:10B2A000F8EE677A27EE800AFDEEC07A17EE903A44
:10B2B0002033402B00F2C780DFED6B7AB4EEE70A53
:10B2C000F1EE10FAF0EE407A0CDD9FED686ADFEDEA
:10B2D000686AB0EE677AB4EEE67AF1EE10FA77EECD
:10B2E000C67AF6DC9FED637AF4EEC77AF1EE10FAD7
:10B2F0000CD59FED5E6ADFED606AB0EE677AB4EE62
:10B30000E67AF1EE10FA77EE867AF6D49FED5B7A64
:10B31000F4EEC77AF1EE10FA00F38D809FED587AC3
:10B32000F4EEC77AF1EE10FA44BF9FED527A77EE51
:10B33000677A27EEA76ADFED535A9FED537ADFED68
:10B34000536AA6EE257A67EE865AE6EE076AB6EEEF
:10B35000007AE5EEA67A27EE877ADFED486A70EE8E
:10B36000267ABDEEE76A16EE103A2033402B67D8F6
:10B37000B4EEE60AF1EE10FA0CDDDFED3C5A9FED7B
:10B380003C6AF0EE676AF4EEC66AF1EE10FA77EE08
:10B39000E57AF6DCDFED376AF4EEE67AF1EE10FAE4
:10B3A0000CD5DFED325A9FED346AF0EE676AF4EEA9
:10B3B000C66AF1EE10FA77EEA57AF6D4DFED2F6AC1
:10B3C000F4EEE67AF1EE10FA40DDDFED276A76EE74
:10B3D000E77A67EEA75A9FED2B5A9FED2B6ADFEDB8
:10B3E0002B6AA5EE856A27EEA55AE5EE866AB8EEC9
:10B3F000006AE5EE267A67EE867AC7EE206A0023B9
:10B40000836143610362C361B7EE006A76EE865AD8
:10B4100076EE666A86EE257A67EE277A66EE876AAA
:10B42000C0ED017AC0ED037A80ED007A80ED027AFA
:10B43000C0ED046A70479FED0C7A77EE677A78E783
:10B44000DFED137AD9E79FED127A86E7DFED0C6A1C
:10B45000F4EEE67AF1EE10FA44BFDFED066A76EE1E
:10B46000E77AB6E727D4D236DB0F4940DB0FC94075
:10B47000E4CB1641DB0F49C0E4CB16C1DB0FC93F5B
:10B48000DB0FC9BF92E741B99730083C15A82ABE27
:10B49000000000000B480C4BC16810B40B4C40F886
:10B4A000043C8A1E2231C38C1B01A4FB03C3DB08AE
:10B4B000A3F5B06322F8023F9142F4D15DF8044B4A
:10B4C000704700BFD03B0020B5140208CDCCCCCCD7
:10B4D00070B5084C251D2E4614F8010B30F028F9E4
:10B4E00028B1037805F8013BB442F5D170BDFF23C4
:10B4F000F8E700BF183C00202DE9F0471D4F01265A
:10B5000007F10805B2464FF03C094FF0000817F864
:10B51000010B3CF0E1FC044690B180F80690C67146
:10B52000FB7803F07F02012A18D013F0800F204629
:10B530000DD185F804803CF0AFFF85F805802C60C4
:10B540000136052E05F10805E1D1BDE8F08785F843
:10B5500004A03CF0A7FF85F805A0F0E71B0605D482
:10B56000012120463BF088F9FB78DEE73CF09AFFAA
:10B57000F6E700BF203C00202DE9F04FDFF8E09116
:10B58000DFF8E0A183B009F10C05012419F8018B63
:10B59000B8F1000F00F0BF804FEA1817013F032FEA
:10B5A00008F00F0200F2BA800AEB4703988D40FAC8
:10B5B00002F616F0010600F0C38001239340013B20
:10B5C0001840574450F018F897F834305E4E18443D
:10B5D00006EBC00604236E61F471B371002303E02F
:10B5E0000133152B00F09780584903EB43025F00AD
:10B5F000895C4145F4D1564B1A4492F859140029FC
:10B6000000F0A08040463AF017FE804600683AF00D
:10B61000FFFD98F805103AF053FF0378002B7AD11C
:10B620004B4B3B44042283F8994483F89824002E22
:10B6300058D0336898F8080003F13F4202F57E02C3
:10B640000AEB9222012792F8382002F01F015209DA
:10B65000032A07FA01F169D0042A62D0022A6AD0CB
:10B66000B6F804C0BCFA8CF2C2F11F02C2F3CC01DE
:10B6700003EB810102F007020E6A92000F27974048
:10B6800026EA07060E620E6A9040304300220862E6
:10B690004FF0010B11460BFA01FE3EEA0C001CD1E3
:10B6A00018680326964020EA060018601F680220EA
:10B6B0009040384318609F6827EA06079F609868A3
:10B6C0009860586820EA0E00586058685860D8683A
:10B6D00020EA0600D860D868D8600131102902F14C
:10B6E0000202D8D11B4B1C4AB3F87810B3F87A3059
:10B6F0000091002001340190B2FBF3F328469BB285
:10B700004146E4B22AF0DAFD0123092C6B7405F1FD
:10B7100018057FF43BAF03B0BDE8F08F00266E61E3
:10B720005CE70E4F3A6B0A433A6399E70B4A176C92
:10B730003943116494E7094A576C394351648FE7E0
:10B740006E614BE70B68FFDE9C2F0020302F00203E
:10B75000D82A0020D03B002040420F000038024091
:10B760004C3C002000EC05082DE9F0418C4B82B0E8
:10B7700093F848210190002A40F00C8193F86C2145
:10B78000B3F86E11DFED876AB3F87081864D07EE6E
:10B79000102A07EE901AB8EEC76AB7EE007AB3F82F
:10B7A0006A11A5F83481F0EE475A4FEA4804E6EEF4
:10B7B000665A8C42B8BF0C46A6EE267AA6B2012184
:10B7C000F8EEE77AA5F8386167EEA67AC5ED4A5A31
:10B7D00085ED4B7AC5ED4C7A83F84811002A00F0CC
:10B7E000D680DDED017A9FED710AF8EE677AA4B29A
:10B7F00080EE270A50F04EFE6400B0FBF4F4012CFA
:10B80000B8BF0124E4B2B0FBF4F39BB2074685F85D
:10B810003C4100EE103ABBEEED0A85ED500A50F0C7
:10B8200039FE634BDFED636AB8FBF0F0A3FB07372B
:10B83000FF0807EE907AF8EEE77A022886EEA77AFC
:10B84000B8BF02205C4985F8440100239FED5B1AD4
:10B850009FED5B6ADFED5B1ADFED5B5A9FED5B2AC4
:10B86000DFED5B2A9FED5B3ADFED5B3A9FED5B4AD4
:10B8700085ED527A07EE903AB8EEE77AF0EE467A26
:10B88000E7EE017AFDEEE76A16EE902A2032402AB2
:10B890007AD8B4EEE17AF1EE10FA0CDDDFED506A01
:10B8A0009FED507AB0EE675AB4EEC75AF1EE10FA37
:10B8B00077EEE67AF6DCF4EEE57AF1EE10FA0CD5E6
:10B8C000DFED476A9FED487AB0EE675AB4EEC75A8B
:10B8D000F1EE10FA77EEA67AF6D4F4EEC67AF1EE2F
:10B8E00010FA49DD74EE677A67EEA76AF0EE624AF5
:10B8F000E6EE824AF0EE430AE6EEA40AB7EE007ADC
:10B9000027EEE65A77EE677AB6EE007AE5EE207A11
:10B9100067EE877A0133202BE1EC017AAAD107EE9A
:10B92000904AF8EEE77AF7EE006A86EEA77A2F4B98
:10B930002F4AC5F8E83703F12801A833C5F8E41702
:10B940001020C5F8F4372021142385F84546A5F8C2
:10B95000E007A5F8F01707EE906AF8EE677AA5F809
:10B96000EC3782ED007AC2EDAC7AC2EDAD7AC2ED71
:10B97000AE7A02B0BDE8F081F4EEE37AF1EE10FAAF
:10B9800048BF75EEE77AAFE7F6EE007AC2E7194BEB
:10B990001A7026E7044D95F83C41B5F83861BEE7CA
:10B9A000D03B00200AD7233C140000100024744927
:10B9B000ABAAAAAADB0FC941600100103C8C4F3E24
:10B9C000DB0FC93F0100F840DB0F49C092E741B9E6
:10B9D0009730083C15A82ABEDB0FC9BFDB0F4940D2
:10B9E000DB0FC940E4CB1641E4CB16C1D8EC050807
:10B9F0005C060010000000102DE9F041214E224F9E
:10BA000096F8773187F8E03606F5BA7607F2E465FE
:10BA100000244FF0050816F8010B20BB2860013404
:10BA2000032C05F10405F6D197F8E016D7F8E406E3
:10BA3000C94301F001013CF03BFD97F8E016D7F84F
:10BA4000E80681F00201C1F340013CF031FD97F8B6
:10BA5000E016D7F8EC0681F00401BDE8F041C1F32F
:10BA600080013CF025BD3CF037FA0134012128600B
:10BA7000E3B210B180F80680C37128683AF0FCFE8A
:10BA8000CEE700BFD03B0020D82A00202DE9F041AE
:10BA90002A4C2B4DB4F87C61A5F8F06682B0EEB963
:10BAA00094F878013CF018FA94F87921C5F8F40676
:10BAB000003A18BF012285F8F22648B194F87A11AD
:10BAC0002B22002914BF11210121C2803AF0D4FE9B
:10BAD000002002B0BDE8F0413DF03CBC94F8788114
:10BAE000002240462B213AF03BFD074640463CF001
:10BAF000F3F9F8B1F7B12B22C5F80C07C280397AF7
:10BB0000FDF766FF4FF000080E4AB2FBF6F3C3F3F1
:10BB10004F0000909BB23946CDF8048005F5DF60F8
:10BB2000A4F87E612AF0CAFBD5F8F836C3F8008085
:10BB300085F8098702B0BDE8F08100BFD03B002046
:10BB4000D82A002040420F002DE9F84F254C94F8E8
:10BB50008C3184F8803104F28317002604F5D07408
:10BB60005FFA86FB0BF101085FFA88F8012117F8EC
:10BB7000010F42460E448A463AF0F2FC4FF00009AB
:10BB8000054640B3387804F80E9C04F80D9C04F880
:10BB90000FBC04F810AC44F8045C3CF09DF918B1FB
:10BBA00080F806A080F80780297AFDF711FF0E4A79
:10BBB000002128463AF0BEF90C4B23600C4B221DA5
:10BBC00021462846C4E901393AF034F969792868F0
:10BBD0004A462AF02BFB082E04F11C04C0D1BDE814
:10BBE000F88F00BFD03B002040420F006562030881
:10BBF000B52B030870B52B4C2B4B94F8B802C4F846
:10BC0000B03200220221C4E99C22C4F87822C4F890
:10BC1000AC22A4F8B4223AF0A3FC002841D0234B74
:10BC20000668054603F1C0015A7C12B15A68964273
:10BC30002BD018338B42F7D1002394F8B802C4F804
:10BC40009C5184F890313CF047F908B10223C3803D
:10BC5000297AFDF7BDFE2846154A00213AF06AF917
:10BC6000144A1549C4F8A0110026111F2846134B89
:10BC7000C4F8A431C4F8A8613AF0DCF869792868FE
:10BC80003246BDE870402AF0D1BA30464CF0B8FDDB
:10BC9000328D0B4992B2531CB0FBF3F081F82001B6
:10BCA000CAE770BDD03B002000FFFF004800001035
:10BCB00040420F00743D0020DD2B03087D2D03085A
:10BCC000880100202DE9F04FC14DDFF8409385B089
:10BCD00088460446C02205F134000021CDF80480D6
:10BCE00052F03DFF99F8B932002B71D099F8BA3271
:10BCF000002B00F08C80DFF8F8A29AF84C34012B6E
:10BD000000F0AE80022B00F08F80B24BB24E029357
:10BD10001C460FCE0FC40FCE0FC49AF842749AF887
:10BD20003E3496E80700AD4EC5F80C613E1E18BFC4
:10BD30000126072B84E8070085F84C6900F20D8185
:10BD4000042B00F21781DFF8C892DFF8B0820026DA
:10BD5000019B5FFA86FB0BF10107FFB2B3423A4643
:10BD60004FF0030129DD18F8014B20463AF0F8FBAB
:10BD7000034620461C4613B33CF0AEF8C9F8140045
:10BD800018B14FF003038371C7719AF83F349AF8E2
:10BD90003E24002B00F0EC80E37983F00103594648
:10BDA000204601364DF0BAF848B14FF00103082E95
:10BDB00089F8113009F11809CAD1029B06E0884BB5
:10BDC000884AC5F81831C5F810210023C5F848394C
:10BDD000D5F8483963B10022019883F82C0001217D
:10BDE00083F82D101A6383F82E2005B0BDE8F08F7C
:10BDF0007D4E7E4C0FCE0FC40FCE0FC496E80700C9
:10BE0000A4F1200384E80700C5F84839EDE7784B32
:10BE1000019993F84024003A204618BF0122FDF70B
:10BE20000BF9C5F84809D3E79AF84234002B3FF4E0
:10BE30006CAF9AF83E34082B12D1674E674F0FCE85
:10BE400005F1F40402940FC40FCE0FC496E8070066
:10BE5000012384E8070085F84C39C5F80C717FE0B0
:10BE6000644C019BC5F850390FCC634F0FC70FCC02
:10BE70000FC794E807009AF842449AF83E3489F8CC
:10BE8000F432003CA7F510634FF0000618BF012400
:10BE900003935A4B85F84C4987E8070007F12808B7
:10BEA00089F8BC62B34602933EE0F27982F0010762
:10BEB00007F0010695F84C09013689F8BB6208B114
:10BEC00087F0010720463CF0DBFA002862D0002C06
:10BED0006DD0A088C8F80C407101B0FA80F041F034
:10BEE00009010BF1010BC0F11F004FF00303C8F86B
:10BEF0000400C8F8141088F8107084F807B0A37113
:10BF000020463AF0B9FCFB07204623D53CF0C4FAA2
:10BF1000039BD8F80C205A61BBF1080F03F11803FA
:10BF200008F1200803931FD0D5F850295A451BDD8E
:10BF3000029B13F8014B029320463AF045FB06465C
:10BF400020463BF0C9FF9AF83F240446002AACD1B2
:10BF5000F779ADE73CF0A6FADAE7082B7FF4F3AE09
:10BF6000274BC5F85439EEE62348C5F848092FE7B2
:10BF7000E37914E79AF84134224AC5F85429012B91
:10BF800005D0022B06BFB7FA87F35B09002385F8BB
:10BF90005839D8E6134A1C4BC5F83029C5F82C3956
:10BFA0000F4AC5F83829012389F8BC32DDE7710151
:10BFB00041F009014FF0FF33C8F81410C8F80430FD
:10BFC000C8F80C4088F810700BF1010B98E700BF1F
:10BFD00014000010080100102CEE0508C94E0508D9
:10BFE000253B04082D3B040800EE0508903E002088
:10BFF000D82A002058EE0508280900101B2F002021
:10C00000A13B0408D13B0408313B0408D03B00208D
:10C0100048000010F8B56D4F97F8200097F82150B0
:10C020003BF05AFF60B12D23C380202104463AF033
:10C0300023FC0A203BF050F820463DF0BFF918B928
:10C04000D7F8F832DA0000D5F8BD013D092DFBD84C
:10C05000FC7FCCB9402033F07BFF0028F4D090F96E
:10C06000043017F80B1C092BC8BF143B3B440A29AA
:10C0700093F8FC4200F09B8093F80833BA7F002AC3
:10C0800008BF1C46002CDFD020463BF025FF0546AC
:10C09000002800F084802D23C38001213AF0ECFBBE
:10C0A000012108463CF00CFA2B68AA881A833C2030
:10C0B0003BF030F9002101203CF002FA97F82130E2
:10C0C000002B4CD0424C00261FE02B68AA885A83D4
:10C0D0003BF002F894F8E016D4F8E40601F0010110
:10C0E0003CF0E6F994F8E016D4F8EC06C1F38001D0
:10C0F0003CF0DEF92B68AA881A8378203AF0ECFF2E
:10C1000097F8213001369E4229DA94F8E016D4F8E7
:10C11000E406C94301F001013CF0CAF994F8E016C5
:10C12000D4F8EC0681F00401C1F380013CF0C0F9C1
:10C130007820002DC9D178203AF0CEFF94F8E0168F
:10C14000D4F8E40601F001013CF0B2F994F8E016ED
:10C15000D4F8EC06C1F380013CF0AAF9CDE7FB7FEF
:10C16000ABB997F82030002B7FF46EAF97F82230F0
:10C17000012B7FF469AFD7F8F83213F080537FF4C6
:10C1800063AF87F82130BDE8F84041F01DBA322096
:10C190003BF0C0F8284600213AF06EFBE1E70121B0
:10C1A0003AF06AFB012108463CF08AF97FE7D7F8AC
:10C1B00020335B057FF548AF09F012FD00287FF4BE
:10C1C00043AF002C7FF460AF3EE700BFD03B0020C0
:10C1D000D82A002038B504460D460A460068FF21DB
:10C1E00052F0BDFC21682944216038BD70B4344848
:10C1F00090F82433A3F13001092958D800F5497487
:10C20000224600F2333012F8015FA5F1300109290E
:10C2100004D88242F7D1002070BC7047141B022C56
:10C220004BDD2848002101E010F8013B01EB8101C2
:10C2300003EB4103161A303B022E044603F0FF01C4
:10C24000F2DC214B03FB01F1A2424FF000030DD9B8
:10C2500003EB830314F8016B5B00303B3344A242D1
:10C2600003F0FF03F4D1194800FB03F32E2D06D091
:10C270001748A0FB032301EB930070BC7047013209
:10C2800004200024157804EB8404303D6400092D5B
:10C29000A4B298BF641900F1FF309CBFA4B2013270
:10C2A00010F0FF00EED1642202FB0433E0E700212E
:10C2B0001D4600F549720B46D8E7064C0021C3E73E
:10C2C000D03B0020F53E00208096980040420F00B1
:10C2D000ABAAAAAAF43E00202DE9F047041E0D46A1
:10C2E00012DB092C26DC824A0B468248A0FB041094
:10C2F000C00800EB8000A4EB40000021125C1A7023
:10C3000059702846BDE8F08764422D23092C01F8B6
:10C31000013B24D8764A774BA3FB0403DB0803EBED
:10C320008303A4EB43030020D35C48700B702846C2
:10C33000BDE8F0876F4B632CA3FB04264FEAD606BB
:10C3400021DC6B4A0B466B49A1FB0601C90801EBD6
:10C350008101A6EB4101515C03F8011BC5E7654A69
:10C36000632CA2FB04364FEAD60637D8604A614BED
:10C37000A3FB0603DB0803EB8303A6EB4303D35CB9
:10C3800001F8013BC7E7A3FB0627B4F57A7F4FEA24
:10C39000D7070DD2564A0B465649A1FB0701C908DB
:10C3A00001EB8101A7EB4101515C03F8011BCAE7D6
:10C3B000A3FB072842F20F7294424FEAD80836D8FE
:10C3C0004B4A0B464B49A1FB0801C90801EB81010F
:10C3D000A8EB4101515C03F8011BDDE7A2FB063726
:10C3E000B4F57A7F4FEAD7070CD2414A414BA3FB01
:10C3F0000703DB0803EB8303A7EB4303D35C01F8DC
:10C40000013BB4E7A2FB073842F20F739C424FEAAC
:10C41000D80821D8364A374BA3FB0803DB0803EBC7
:10C420008303A8EB4303D35C01F8013BDEE7324A08
:10C43000A3FB080994424FEAD90921D82C4A0B469C
:10C440002C49A1FB0901C90801EB8101A9EB4101BC
:10C45000515C03F8011BB5E7274BA2FB08099C427E
:10C460004FEAD90921D8224A224BA3FB0903DB0852
:10C4700003EB8303A9EB4303D35C01F8013BCAE759
:10C480001E4AA3FB090394424FEAD30A21D80B4664
:10C490001849174AA1FB0A01C90801EB8101AAEB5F
:10C4A0004101515C03F8011BCAE7144BA2FB0902CE
:10C4B0009C424FEAD20A13D80E4B0D4AA3FB0A0343
:10C4C000DB0803EB8303AAEB4303D35C01F8013BD6
:10C4D000CAE70A22BAFBF2F042F0CAFF0346D7E7E6
:10C4E0000A22BAFBF2F042F0C3FF0146E4E700BFC4
:10C4F0001C770608CDCCCCCC9F8601003F420F00B4
:10C50000084BD3E9CD029042D3F83C3302DC11460C
:10C5100002460846984204DD9A42B8BF1A461046C1
:10C5200070477047D03B00200B6810B414681B1B89
:10C53000036054684B681B1B43608B6892685DF80E
:10C54000044B9B1A8360704783B50C46164605461C
:10C5500032F03CF9204632F039F90021204B0846F0
:10C56000002E08BF1E463BF0ABFF002101203BF030
:10C57000A7FF28463BF00AFCB0B1012100203BF0A8
:10C580009FFF28463BF0FAFB074620463BF0FAFBAC
:10C590000028FAD0394620463BF0FCFB3846B0472D
:10C5A000002108463BF08CFF20463BF0EFFB0028C3
:10C5B000DFD0012100203BF083FF20463BF0DEFB73
:10C5C0000146284601913BF0DDFB01990028F8D097
:10C5D00028463BF0DFFB002108463BF071FFC8E72F
:10C5E0009DB70308F0B500230B604B608B60CB60F8
:10C5F0000B610268DFF894C089B004ADC2F38557BF
:10C600002E4647FA03F0C007344644BF13F80C0027
:10C6100004F8010B03F1010348BF2646062BF0D1B5
:10C620001848C2F303240444002394F88C42337066
:10C630008DF8184000F5257CC2F305370DF1190679
:10C6400047FA03F0C007344644BF13F80C0004F85F
:10C65000010B03F1010348BF2646062BF0D100234E
:10C660003370C2F3834406ABCDE90134084602F0CF
:10C670000F0305490095C2F3031242F00FFD09B004
:10C68000F0BD00BF00EC05084477060884EE0508FD
:10C6900070B5094CD4F84023054662B10026D4F8A1
:10C6A00040032D2101363DF09DFFAE42F7DBBDE892
:10C6B000704040F08BB870BDD03B0020164901306F
:10C6C00001EBC000F0B4D0F8A0C2144E0022C6F8AE
:10C6D0004423C6F85423C6F86423C6F87423C6F866
:10C6E0008423C6F89423C6F8A423C6F8B423BCF167
:10C6F000000F0FD090F89C7267B13F0106F551769C
:10C7000000240CEB04030FCB35191034A74285E845
:10C710000F00F6D1F0BC704700EC0508D03B0020BC
:10C7200038B50F4C94F8CB1301F03F018B1C024637
:10C7300001F10A0584F8C93384F8C65304F5717011
:10C7400084F8C723083119F033FE254485F8C20365
:10C7500094F8C6331C44000A84F8C30338BD00BFF4
:10C76000D03B002070B51D4C0968D4F8F0531C4E26
:10C77000D4F8EC43D6ED497ADFED1A6A491B00EE96
:10C78000901A0168F8EEE00A091B60EEA70A00EEB5
:10C79000101A20EEA07AB8EEC00A1C46A0EE007A6D
:10C7A000B1EE400AF1EEC77A67EEA67AFCEEE77AC0
:10C7B000C2ED007A40F0B8FF9FED0B7ADFED0B7A07
:10C7C000E0EE077AFDEEE77A17EE902A002ABCBF6A
:10C7D00002F50C42A032226070BD00BFD03B0020A9
:10C7E000880100202C7D8E3FA00CB34500A00C4694
:10C7F00038B50B4C002501228021204633F094FBF4
:10C8000030B194F9040033F0C1FB08B1006838BDC1
:10C810000135092D04F10C04EDD10020F7E700BF2C
:10C82000D43F002038B5041F00F1080554F8043F38
:10C83000D81780EA430013F011F8A542F6D138BDAD
:10C840002DE9F041D24CDFEDD37AD4F85C3A94F87C
:10C85000F50A07EE103A2DED028BB8EE478A28EE66
:10C86000278A002840F0CA80D4F8002B94F8F41AE4
:10C8700094F8113B002A19DD07EE902ADFEDC66A15
:10C88000F8EEE77AC3F1640386EEA77A00EE103A79
:10C89000B8EEC00A20EE070A29B920EE000ADFED43
:10C8A000BF7A20EE270A4FF0F5FD80B2B4F8F63AD1
:10C8B000A4F8F60A834200F0A18094F8607AB84E9A
:10C8C000DFEDB88A4FF00008002594F8143B2B41A7
:10C8D000DB0714D594F8F43A002B7FD1B4F8F63A7C
:10C8E00007EE103A002F00F00281B8EE477AC8EE4A
:10C8F000877A77EE887A88EE277A86ED027A013594
:10C90000042D06F12406E0D194F8F95AB4F8FC6A33
:10C91000002D40F0EF80002F5CD194F8103B84F89C
:10C920001C5B84F8183B002E54D0002D52D007EE2B
:10C93000906A0123B8EE678ADFED9A7A84F8203B8B
:10C940009D42C7EE888A28D0022D43D1D4F85C1AC4
:10C950009548B0EE480A45F0DDF994F81C3B012BF0
:10C9600000F01181022B35D1D4F85C1A8F48B0EE5B
:10C97000480A45F0CFF994F81C3B012B00F0FE80EB
:10C98000022B27D1B0EE480ABDEC028BD4F85C1A1A
:10C990008748BDE8F04145F0BDB9864AD2ED007A3E
:10C9A00078EEA76A134687EEA67A002143F8041FA3
:10C9B00083ED017A78EEA76A002187EEA67A996066
:10C9C00083ED037A77EEA88A002287EEA87A1A61AF
:10C9D00083ED057ABDEC028BBDE8F081B4F8F63A40
:10C9E000D4F85C1A00EE103A301DB8EE400A002F61
:10C9F00077D145F08FF994F8607A80E794F8607AFF
:10CA0000002F3FF45CAF94F8F95AB4F8FC6A002D9B
:10CA1000E0D0694A94F8FA3AD2F8742492F8832064
:10CA20001343D7D1D4F8002B94F8113B002A6CDDC6
:10CA300007EE902ADFED586AF8EEE77AC3F1640357
:10CA400086EEA77A012D00EE103AB8EEC00A08BFB4
:10CA5000DFED527A27EE000A04BF20EE000A20EE36
:10CA6000270A4FF017FD80B2A4F8FC0A002F7AD0F5
:10CA70008642AFD00028ADD094F81C3B002BA9D043
:10CA800007EE900AB8EE678ADFED467A012BC7EE13
:10CA9000888A47D0022B9DD1D4F85C1A4248B0EE68
:10CAA000480A45F021F894F81C3B012B58D0022B82
:10CAB00090D1D4F85C1A3D48B0EE480A45F014F81D
:10CAC00094F81C3B012B46D0022B83D1B0EE480AD0
:10CAD000BDEC028BD4F85C1A3548BDE8F04145F056
:10CAE00003B8301D45F000F894F8607A07E7C6F8FF
:10CAF0000480FAE6304A94F8FA3AD2F8742492F8AC
:10CB0000832013437FF407AF8CE70023A4F8FC3A9B
:10CB1000002F7FF45FAF94F8103B84F81C5B84F81F
:10CB2000183B57E7234A1346F3EC017A78EEA76ADD
:10CB300087EEA67A83ED017AD2ED007A78EEA76AC5
:10CB400087EEA67A83ED037A77EEA88A87EEA87A35
:10CB500083ED057A3EE7174AD2ED007A131DF3E71D
:10CB6000144A131DE8E794F8103B84F81C5B84F822
:10CB7000183B00283FF42EAF0646D8E60D4AD2ED0A
:10CB8000007A131D1EE70B4AD2ED007A131D11E740
:10CB900014000010BD37863500409C45CDCC4C3C80
:10CBA000740A001083F9223E380B00105C0B001051
:10CBB000800B0010A40B0010D03B0020F8B5214CD6
:10CBC0001D270E46054684F8787419F017FD0020DD
:10CBD00019F0B6FC082019F0B3FC0E2019F0B0FCD7
:10CBE000384619F0ADFC042019F0AAFC042019F015
:10CBF000A7FC002019F0A4FC302019F0A1FC0020B3
:10CC000019F09EFC304619F09BFC002019F098FCAE
:10CC100019F0E0FC04F2794019F0E6FB234670B10C
:10CC200094F8792462B994F87A24302A00D03AB979
:10CC300093F87B2422B993F87C342B700120F8BD43
:10CC40000120FCE7D03B0020104B034410B5044604
:10CC500093F8740310F054F90D4800EB44040A23D0
:10CC6000B4F98C14B1F5FA6FA8BF4FF4FA61B1F5BD
:10CC70007A7FB8BF4FF47A71A1F57A71BDE81040A0
:10CC8000B1FBF3F10920C9B210F068B900EC050856
:10CC9000D03B00201D4991F82423A2B3F0B4002614
:10CCA00005463346304637461BB991F824432D2CB0
:10CCB00023D02E2A19D0CA1800EB800092F8244302
:10CCC000A4F13002092A4FEA40009CBFA0F13002D3
:10CCD000A0180E2B14D80133CA1892F82423002A66
:10CCE000E2D106B14042F0BC70470133002DF8D0CC
:10CCF000CA182A4482F82473DDE701231E46EBE7B5
:10CD00000020F0BC70470020704700BFD03B0020DF
:10CD10001FB503AC8DF80C30009400238DF80D3056
:10CD200009F0AEFA04B010BD10B5FCF74DFE1121AC
:10CD3000044639F0A1FD20463BF0AEFBC8203AF096
:10CD4000E9FA2046BDE810403BF0ACBB704700BF9D
:10CD5000704700BF704700BF704700BF037870B4D2
:10CD6000FBB10446C0F10106A31914F8015FDBB260
:10CD7000002DF9D101335B00DCB2032513800C7068
:10CD80004D7004785CB1022300255A1CD2B2CC54F9
:10CD90008D5410F8014F0233DBB2002CF5D170BC7A
:10CDA000704702242346E8E710B5044C04480A46BD
:10CDB0002146FFF7D3FF204610BD00BF8040002072
:10CDC0005477060810B5044C04480A462146FFF77C
:10CDD000C5FF204610BD00BF8040002064770608D4
:10CDE00010B5044C04480A462146FFF7B7FF204619
:10CDF00010BD00BF804000207077060810B5044CBD
:10CE000004480A462146FFF7A9FF204610BD00BF8F
:10CE1000804000207C77060810B5044C04480A4680
:10CE20002146FFF79BFF204610BD00BF8040002039
:10CE30008877060870B501F07F0505EB850400EBE7
:10CE4000C404282101FB05010126C4F83031002368
:10CE5000C4E94A2284F81C5184F81D61C4F83431B5
:10CE600001F58E711DB9FBF7CFFA002070BDFBF7FD
:10CE70003FFB002070BD00BF70B50D4B0D4D0E4A3D
:10CE8000C3F8B025044603F5B66283F8BC15002646
:10CE90000D23812185F8C468FFF7CCFF204605F5F6
:10CEA00006621F23BDE870400121FBF753BC00BFA1
:10CEB000D03B0020E0190020555342532DE9F043A8
:10CEC000B04DB14C95F86F38C4F8C00585B08946AF
:10CED0005A2B00F2B780DFE813F0CA00B500B500A6
:10CEE000DA00B500B500B500B500B500B500B50075
:10CEF000B500B500B500B500B500B500B5000D0131
:10CF0000B500B500B500B500B500B500B5003101FC
:10CF10007400B500B5007400B500B500B500B500EB
:10CF2000B901B5006101B500B5007C00B5000B0288
:10CF3000B500B500B500B5005B00B500B500B500A3
:10CF4000B500B500B500B500B500B500B500B50039
:10CF5000B500B500B500B500B500B500B500B50029
:10CF6000B500B500B500B500B500B500B500B50019
:10CF7000B500B500B500B500B500B500B500B50009
:10CF8000B500B500B500B500B500B500B500E601C7
:10CF900095F870389B0700F16B82B5F87638D5F8B4
:10CFA0007128D4F8CC155BBA9BB212BAD01888425B
:10CFB000C4F8D435C4F8D02503D9FBF771F900289B
:10CFC00052DB0020A4F8C4050646304605B0BDE893
:10CFD000F08395F8C438002B40F0FE8095F96C384A
:10CFE000002B2FDAD5F8C83808469B6898470028E8
:10CFF00040F02082B5F87668D5F87128D4F8CC35A1
:10D0000076BAB6B212BA90199842C4F8D465C4F888
:10D01000D02505D90192FBF743F90028019A23DBBB
:10D02000D4F8C835D5F8687803FB06F603FB02F29E
:10D030000220BE42C4F8D025C4F8D46585F8C408DF
:10D0400000F0D08095F830385A1CD2B205EBC303FB
:10D0500005204FF40051042A85F8302883F834085D
:10D06000C3F8381800F0A4814FF0FF36ADE7D5F8CB
:10D070006838002BE6D1D5F8C83808469B68984731
:10D080000646002840F0D681A4F8C4059DE73F4B32
:10D09000002203F1120103F8012F8B42FBD13C491E
:10D0A00094F8C63595F8300870260E7098424FF007
:10D0B0000C06CE7110D005EBC300013390F8346834
:10D0C0008E70B0F83808DBB2042B40BA888114BFE8
:10D0D00084F8C63584F8C62595F873381222934231
:10D0E000A4F8C42598BFA4F8C4350026304605B07E
:10D0F000BDE8F08395F87038DA0700F14281D5F881
:10D10000C83895F87308DA6901EBC10102EB8101B7
:10D110000A79531D834228BF0346A4F8C435002B67
:10D12000E3D0013B1A489BB201331944034411F880
:10D13000012D03F8012D8342F9D1D6E7154F164989
:10D140003E460823073FC6F10700A4F8C435002275
:10D1500002E092F894231E463346BE4203F80129AA
:10D1600000EB030211FA82F2F3D1D5F8C838484631
:10D17000DB6898470028B8D0B37863F07F03B370BA
:10D18000002622E7E0190020D03B00207B5400203D
:10D190007C5400208354002000EC0508D5F8C838E2
:10D1A000C84A5B680846111D98470646002840F0AB
:10D1B0004181D4F8CC35C44AD4F8C815013B180EC7
:10D1C0001070180C09BAD37050701B0A08209370A5
:10D1D0005160A4F8C405F8E6D4F8D475D4F8D02585
:10D1E000D4F8C835D5F8C868B2FBF3F2B7F5805F5C
:10D1F00028BF4FF480574FF4805C3669B249B7FBC3
:10D20000F3F348469BB2A4F8C4C5B0470028C0F267
:10D21000BD803B46AC4AD4F8C0058121FFF70AFE29
:10D22000D4F8D025D4F8D405D4F8B8353A44C61B80
:10D23000DF1BC4F8D025C4F8D465C4F8B875002E37
:10D240007FF453AF032385F8C438BEE69E4F4FF0FA
:10D2500000083B4607F10C0203F8018B9A42FBD110
:10D26000D5F8C83848465B6802AA03A9984706461D
:10D27000002840F0E980039BBDF80820013B190E0F
:10D2800052BAFB713971190C1B0A79710820BB71F4
:10D2900002217A810C23BDF80A20F87039727A7263
:10D2A000A4F8C43591E6894F894938460823073FD9
:10D2B000C0F10706A4F8C435002202E092F89C23CE
:10D2C00018460346874203F8012906EB030211FAC8
:10D2D00082F2F3D1D5F8C8384846DB689847002871
:10D2E0003FF403AFFB7863F07F03FB7000266CE62E
:10D2F00095F8C438002B61D195F96C38002BFFF6F6
:10D30000A1AED5F8C83808469B689847002840F079
:10D310009180D5F8C8384846DB689847064600280B
:10D3200040F0B880B5F87638D5F87178D4F8CC25C7
:10D330005BBA99B23FBA7B189342C4F8D415C4F8CB
:10D34000D07500F29F80D4F8C835D5F8682803FB63
:10D3500007F703FB01F39342C4F8D075C4F8D43542
:10D360007FF470AEB3F5805F28BF4FF48053012186
:10D37000D4F8C005544A85F8C4189BB2FBF7EAF903
:10D3800023E607235349A4F8C435CAE695F8303894
:10D390005A1CD2B205EBC30304204FF488518242D9
:10D3A00085F8302883F83408C3F838187FF45CAE69
:10D3B000002385F830384FF0FF3606E6D4F8D475F0
:10D3C000D5F8C808D4F8C835D4F8D0254669B2FBDA
:10D3D000F3F2B7F5805F28BF4FF480570846B7FBDC
:10D3E000F3F339499BB2B047002860DBD4F8D0256D
:10D3F000D4F8D465D4F8B8353A44F61BDB1BC4F82E
:10D40000D025C4F8D465C4F8B8352EB9D4F8C00511
:10D410003146FFF731FDD8E5B6F5805F28BF4FF400
:10D420008056B3B2D4F8C005274A0121FBF792F920
:10D430000026CAE595F830385A1CD2B205EBC30372
:10D4400002204FF4685106E695F8303805EBC30228
:10D450000133DBB202204FF46851042B82F8340808
:10D46000C2F8381820D085F830384FF0FF36ACE5D8
:10D4700095F830385A1CD2B205EBC30305204FF49F
:10D480001051E8E50191FAF70BFF00280199BFF66A
:10D490005AAFE9E595F830385A1CD2B205EBC30310
:10D4A00002204FF41C51D6E585F83088DCE595F86C
:10D4B00030385A1CD2B205EBC30304204FF440713C
:10D4C0006DE700BF984100207C5400208354002069
:10D4D00000EC05088CEF050810B5074B93F86D18A4
:10D4E0000446FFF7EBFC002800DB10BD20460121BD
:10D4F000BDE81040C0E400BFE0190020F8B5344C8E
:10D5000094F8C4582DB1012D01D1FFF7E5FF00209B
:10D51000F8BD304FB0F8B433D4F86428C7F8B42558
:10D520001F2BD4F86828C7F8B825064608D12A4B1F
:10D53000D4F860289A4203D194F86D18012919D9BA
:10D5400094F8303804EBC3020133DBB2042B08BF7C
:10D5500000234FF40051052082F8340884F8303855
:10D5600030460223C2F8381884F88038FBF718F9DF
:10D570000020F8BD94F86E38013B0F2BE0D8FFF780
:10D580009DFC00281CDB94F8C438013B022BBED95B
:10D59000B7F8C415C1B1D4F86838D7F8B82587F8FA
:10D5A000BC558B4228BF0B46D21A0421C7F8B825B8
:10D5B00084F8C418094A30468121FFF73BFCA6E7EE
:10D5C0003046FBF7EDF8A2E73046FFF755FC9EE743
:10D5D000E0190020D03B0020555342437C540020EA
:10D5E00008B5084B93F8C438022B07D0033B012B36
:10D5F00002D80021FFF740FC002008BDFFF76CFFB8
:10D60000002008BDE01900202549D1F8D8350F2B9E
:10D6100004D05A1CC1F8D8250020704770B5214CA1
:10D6200094F82D5D0023C1F8D835F5B9D4F8082851
:10D63000D4F80C38B2F5006F19D09A422CD01AD910
:10D64000C2F50063402B18D9403B02F14005C1F8F8
:10D65000DC35012384F82D3DC4F8085892B24023EC
:10D6600011490A448121FFF7E5FB002070BDC4F891
:10D6700008588BB12A469B1AE4E74FF0000502EBED
:10D680000306C1F8DC550CBF02210121C4F808686B
:10D6900092B284F82D1DE3E7002384F82D3DE4E7E2
:10D6A000D03B0020E019002010270020ACE700BF8D
:10D6B00070B51E4C94F82D3D012B03D0022B0AD0DF
:10D6C000002070BD01461A48D0F8DC3553B984F803
:10D6D0002D3D002070BD00231A468121FFF7AAFBD3
:10D6E0000023F4E7402BD4F8082810D9403B02F17E
:10D6F0004005C0F8DC35C4F8085892B240230D4C00
:10D70000084622448121FFF795FB002070BD4FF0B1
:10D71000000503EB0206C0F8DC5508BF0220C4F880
:10D72000086892B208BF84F82D0DE8E7E0190020E0
:10D73000D03B002010270020012905D008B5032187
:10D74000FAF7A8FF002008BDB2E700BF70B5044695
:10D7500049B990F81131022B1BD094F81631012BE6
:10D760000DD0002070BDD0F8E4355B69002BF8D0F7
:10D7700090F81221032AF4D19847002070BD2A4A5C
:10D780002369D2F8E0255A60002384F8163100207E
:10D7900070BDD0F83831D0F82451AB4217D9C278D7
:10D7A000012AD0F82821A3EB050308BF5219C0F8BD
:10D7B000383108BFC0F828219BB20021FFF73AFB9F
:10D7C00000231A4619462046FAF7C4FFC5E7D0F8E9
:10D7D0003C31B3FBF5F605FB163666B99D420AD817
:10D7E000D0F84021934206D233463246FFF722FB5F
:10D7F000C4F84061E4E7D4F8E435DB681BB194F881
:10D800001221032A0CD00023052284F81121194685
:10D810001A462046FAF79EFF2046FAF7E5FD9CE7F8
:10D8200020469847EFE700BFD03B002010B500230B
:10D8300004220446194680F811211A46FFF7FAFA25
:10D840002046FAF7D1FD002010BD00BF10B50446F8
:10D8500029B990F81131032B0DD0002010BDD0F85C
:10D86000E4359B69002BF8D090F81221032AF4D1FB
:10D870009847002010BDD0F89013D0F87C3399421F
:10D8800014D9C078D4F880230128A1EB030104BF88
:10D89000D218C4F880238B4228BF0B46C4F89013DB
:10D8A0009BB220460021FAF755FFD6E7D0F8E435C1
:10D8B0001B691BB190F81221032A03D02046FFF701
:10D8C000B5FFCAE79847F9E738B5134602250A4677
:10D8D000C0E94E3380F811510021FFF7ABFA002068
:10D8E00038BD00BFF8B50B7813F060050C4606464E
:10D8F0001DD0202D18D14A78FE2A45D0FF2A3ED1CE
:10D900004A88002A58D1CD88002D55D11B0653D402
:10D91000384B012103F5066283F8C45883F8801858
:10D920001F23FAF717FF00E000252846F8BD4B78C3
:10D930000A2B4CD00B2B45D0012BF6D191F904309A
:10D940008988002B48DBFAF78BFE2179294F304676
:10D95000FAF764FF0223217940223046FAF7C2FF2A
:10D9600097F88038022B3CD094F90420002ADCDAA6
:10D97000012BDAD030460121FFF77EFAD5E70225E8
:10D98000FAF7DAFE2846F8BD4D88ADB9CC88012CEF
:10D9900012D11A0610D5174BD3F8C8389B6998478F
:10D9A0001549C0B281F8E40530B1224601F2E451D4
:10D9B0003046FFF789FFB8E730460225FAF7BCFE8C
:10D9C0002846F8BD0C4B4A8883F8E525ADE70B499E
:10D9D0000122FFF779FFA8E701F07F01FAF75AFE6D
:10D9E000B3E730468121FAF773FE002387F88038C9
:10D9F0009BE700BFE0190020D03B0020B54100208C
:10DA000010B50C7814F0600413D0202C0AD14B7898
:10DA1000023B092B18D8DFE803F01B211717171753
:10DA20001717272E22490122FFF74EFF0024204618
:10DA300010BD4B78062B24D00A2BF3D01D4B8A78CF
:10DA4000C3F8F025204610BDFAF776FE0224EEE773
:10DA500019490122FFF738FF0024E8E7174901229E
:10DA6000FFF732FF0024E2E74B88124A1B0AC2F894
:10DA7000EC350024DBE70F4B8A78C3F8E825002457
:10DA8000D5E74B881B0A222B0CD0212B04D0214632
:10DA90002246FFF719FFCAE7CA880949092A28BFA1
:10DAA0000922F6E7CA880749262A28BF2622F0E776
:10DAB000C0410020D03B0020BC410020B8410020E4
:10DAC000EA020020B0020020F8B50B7813F06005E0
:10DAD0000C46064611D0202D16D1CD88D5B11B0697
:10DAE0002AD52A4620496078FAF752FBE2881E4977
:10DAF0003046FFF7E9FE00250AE04B780A2B16D0E6
:10DB00000B2B0ED0062B03D13046FAF715FE02255B
:10DB10002846F8BD022260781144FAF739FB2846FE
:10DB2000F8BD8B78E3B9114BC3F8F455F0E7104911
:10DB30000122FFF7C9FEEBE70E4B4A780E4FC3F800
:10DB4000F42003230021C0E9E45580F8113107F6E1
:10DB500058022B46C7F854580D46FAF7FBFDD7E795
:10DB6000FAF7EAFDD4E700BF38220020D03B0020BE
:10DB7000C441002088010020E01900200B7803F048
:10DB80000303012B03D0022B04D0002070478B88A5
:10DB90001BB935E78B88832BFBD095E7F0B50121C6
:10DBA00090F8D17590F8D36590F8CFC590F8CE5520
:10DBB00090F8D03590F8D22580F8111190F8CC1556
:10DBC00085B005EB0C2503EB072302EB062201F0E1
:10DBD0001F06AFB292B290F8CD558DF808109BB2E7
:10DBE000012E0446ADF80A70ADF80C30ADF80E20E9
:10DBF000C0F840218DF8095017D0022E1FD036B141
:10DC000001F08001FAF764FD002005B0F0BD092D98
:10DC10000FD8DFE815F0BF00AC000E00D5000E00F5
:10DC2000EA0085000E007700540090F81221032AC4
:10DC30002FD02046FAF780FD002005B0F0BD01F09E
:10DC400060012029DAB234D0012D00F02081032DAB
:10DC500000F00681002DD7D190F81211022900F0B2
:10DC6000DF800329E5D11B0600F14B8102EB820224
:10DC700000EBC20393F87633002B00F04D81BF4BCD
:10DC80000122C3F80426BE4920460222FFF71CFEEB
:10DC9000BAE7DAB2012ACCD8D0F8E43502A99B68F9
:10DCA0009847BDF80E30002BAED12046FFF7BEFDE1
:10DCB000AAE7D0F8E43502A99B689847A4E7F9B22F
:10DCC000AE4D012985F8F815B3D890F81231022B22
:10DCD00000F02781032BACD1002900F0868190F859
:10DCE00010110129E1D0D0F8E4355B68984795F828
:10DCF000F81584F810112046FAF722FB2046FFF7AA
:10DD000095FD81E7012A94D190F81231022B00F0A1
:10DD10001781032B8DD100F58871FFF7D5FD73E7CF
:10DD20003D0A022DADF8062000F05081032D00F0D1
:10DD30000B81012D7FF47DAFD0F8EC3580781B6826
:10DD40000DF106019847BDF80620002A3FF45CAFAC
:10DD5000BDF80E30002B3FF457AF9A4228BF1A4649
:10DD600001462046ADF80620FFF7AEFD4CE790F8DF
:10DD70001231023B012B3FF65CAF012F7FF444AF21
:10DD8000D0F8E43500229B68C0F8182102A920468B
:10DD900098478AE790F81231023B012B3FF649AFD2
:10DDA000764BD0F818210021C3F8001612B10222D8
:10DDB000C3F80026734920460222FFF785FD23E7BA
:10DDC000012F00F09880022F7FF41EAF13F0FF0F99
:10DDD0007FF41AAF02691B0A023B5268032B00F260
:10DDE0001D81DFE803F0393531241A437FF421AF78
:10DDF00090F81231032B3FF41CAF036907F07F0545
:10DE000080F81451196867F30A120A431A60FFF781
:10DE10000DFD002D00F0E580022384F81231F3E6B9
:10DE200051063FF4F1AE1146FAF752FCECE6052339
:10DE300063F30612514B012184F816112046C3F8F2
:10DE4000E025FFF7F3FCDFE6042363F30612F1E7B6
:10DE5000032363F30612EDE7022363F30612E9E7F7
:10DE600090F81231022BDBD0032B7FF4E2AE27B9FE
:10DE7000550602D01146FAF72BFCD4F8E43502A976
:10DE80009B68204698472046FFF7D0FCBCE690F8F8
:10DE900012110229C4D003297FF4CBAE002F7FF4E6
:10DEA000B3AE12F07F013FF400AF180600F1A78077
:10DEB00002EB820304EBC30304EB810083F8767367
:10DEC00083F8741383F87573282303FB0243416DB1
:10DED00003F55D73DA780B68023A6FF35553012A44
:10DEE000D4F8E42598BF43F080530B602046936834
:10DEF00002A99847D9E6D0F8E435C0F818719B68B4
:10DF000044E702F07F0202EB820200EBC20393F8C7
:10DF10001E31002B7FF4B3AE184B0022C3F8042649
:10DF2000B1E600293FF4C1AE0121032380F81011AE
:10DF300080F81231FAF704FA2046FFF777FC63E61F
:10DF40001149FFF7C1FC5FE6FDB2052D3FF671AE4A
:10DF5000DFE805F0342C241C0B03D0F8EC35807876
:10DF60009B690DF106019847EDE6D0F8EC35807815
:10DF70005B690DF106019847E5E600BFD03B002044
:10DF8000D4410020D0410020CC410020D0F8EC3515
:10DF900080781B690DF106019847D4E6D0F8EC357E
:10DFA0008078DB680DF106019847CCE6D0F8EC35B7
:10DFB00080789B680DF106019847C4E6D0F8EC35EF
:10DFC00080785B680DF106019847BCE6D0F8E4352F
:10DFD00080789B6A0DF1060198474570C4F8F005FA
:10DFE000B1E6012384F812310EE60222D0F8E435BE
:10DFF00080F8101180F812215B68984755E62822B6
:10E0000002FB014304EB810083F81E7183F81C11AD
:10E0100083F81D51816903F58E735BE7012363F378
:10E02000061207E7214A038890429BB212D002F5FC
:10E03000806290420ED0B0F1804F0BD0A2F58032BA
:10E04000904207D002F58062904203D002F58062D0
:10E05000904203D14A8823F070031343144A90423C
:10E0600018D002F58062904214D030B423F440738B
:10E070000C894D6802F56C429BB2234390420C8898
:10E080000380C56204850DD18B7A0386012330BCE1
:10E090008382704703800B884A68C262038501232C
:10E0A00083827047034B9842EED0EFE700000140B7
:10E0B00000100040000401400023C0E90033C0E923
:10E0C0000233C0E90433C0E90633C0E90833C0E9CC
:10E0D0000A33C0E90C338363704700BF0B6870B428
:10E0E000D1E90524CD682B431343D1E90725234308
:10E0F0001343D1E909422B43D1E90D65234313436F
:10E1000004680B4A334322402B4313430360D1E995
:10E110000B3442690D6922F0070223431343D1E90E
:10E12000014243614560846070BCC260704700BFBB
:10E130003F801CF002683649002310B422F001022F
:10E14000212488420260036043608360C3600361EE
:10E15000446138D02F4B98422ED02F4B98423CD060
:10E160002E4B984240D02E4B984232D02D4B9842A5
:10E1700041D02D4B984246D02C4B984217D02C4B77
:10E1800098423CD02B4B984216D02B4B984224D02F
:10E190002A4B984228D02A4B98421AD0294B9842B1
:10E1A00029D0294B98422ED0284B984208D14FF0C5
:10E1B0003D5243F8AC2C03E04FF4746243F8202C3A
:10E1C0005DF8044B7047224B5DF8044B3D229A608A
:10E1D0007047204A43F8642CF2E74FF474125DF85C
:10E1E000044B43F8382C70474FF074625DF8044BD1
:10E1F00043F8502C7047184A43F87C2CE0E73D2246
:10E2000043F8082CDCE7154A43F8942CD8E700BF04
:10E2100010600240286002404060024058600240A6
:10E220007060024088600240A0600240B860024016
:10E230001064024028640240406402405864024076
:10E240007064024088640240A0640240B8640240E6
:10E25000006002403D000020400F002000003D20F3
:10E260002DE9F04FDFF884A32DED028B9AF81C16F0
:10E27000002297B0CAF80C26CAF81026CAF814264D
:10E28000CAF81826CAF8082619B19AF81D268AF87D
:10E2900008269AF81E261AB19AF81F268AF8172619
:10E2A0009AF822261AB19AF823268AF812269AF8A2
:10E2B00020261AB19AF821268AF80D269AF82436D3
:10E2C00005935A1ED3B257B204937B1C00F0AA8068
:10E2D000BC4ABD4E52F83780029602EBC7020023BB
:10E2E0001279019308EE102A1D4634469946267885
:10E2F000394630463CF082FA83463046BBF1000F87
:10E300001ED039F0E9FDEA1D1321D2B220B14FF041
:10E31000000E827180F807E038F0AEFA20783CF009
:10E320009FFA4FF0070309F1010223714FF0010337
:10E3300084F802906070CDF804B05FFA82F9E3705F
:10E340000135042D04F10504D1D118EE100A029E06
:10E35000CDF80C90FBF71AFB9C499D4A4868024097
:10E3600042F440324A600FB9019B5BB9994C482096
:10E37000FBF70CFB204602214CF098FAA26842F011
:10E380000102A2609148934A4168BAF8264641F4D6
:10E3900000014160516821F480515160916B21F47A
:10E3A000401141F480119163D16841F46001D16062
:10E3B000956B85F44011C1F3015101EB81011F20E0
:10E3C00000FA01FC25EA0C0C112505FA01F141EADD
:10E3D0000C019163D16841F4E011D160956BC5F3F4
:10E3E0000151C1F10401C9B201EB810188404FF034
:10E3F000100C25EA00000CFA01F108439063E4B127
:10E40000BAF82816CAF83046A1B1BAF82A26CAF8CE
:10E41000341662B1019B7048521A90FBF2F2CAF8AE
:10E4200038266BB917B0BDEC028BBDE8F08F6B4A94
:10E430001288EFE76A4A1188E7E76A4A1488DFE73B
:10E44000404603994CF032FA5F4B012003F1140966
:10E450000723F278441CE4B252B375783279A5F1FF
:10E460000A0101EB410105EB450C092D03FA01FE00
:10E4700003FA0CFB02FA01F140F28E80D8F80C206E
:10E4800022EA0E0E41EA0E01C8F80C10421E02EB01
:10E4900082021F21062801FA02FC05FA02F261D865
:10E4A000D8F8341021EA0C010A432046C8F8342079
:10E4B0000536B145CDD1D8F80820049942F4007250
:10E4C000C8F80820D8F8082042F48072C8F808205C
:10E4D000D8F80820574442F00102C8F8082097F9FC
:10E4E0002C26022039F0AAFB044600289AD0406866
:10E4F0004AF04EFC059A06214AF05CFC6068FFF782
:10E5000019FE07A8FFF7D8FD039EA368364A0793B4
:10E51000012E8CBF4FF48060002000230D9008F185
:10E520004C054FF40060089509920A934FF48072ED
:10E530000C930E904FF4003360680B9607A94FF4CC
:10E540000055CDE90F521193FFF7C8FD62681368BB
:10E5500043F001031360D8F8083043F08043C8F853
:10E5600008305FE7C11FA0F10D0201EB81014FF000
:10E570001F0E02EB82020C280EFA01FC0EFA02F0CA
:10E5800005FA01F113D8D8F8302022EA0C02114321
:10E590002046C8F830108BE7D8F8101002FA0CF2B9
:10E5A00021EA0B0B42EA0B02C8F810206EE7D8F8FC
:10E5B0002C1005FA02F221EA00010A432046C8F8AD
:10E5C0002C2075E7A4EF0508D84100200023014066
:10E5D000E030FCFF00200140803801002E7AFF1F50
:10E5E0002C7AFF1F2A7AFF1F0C420020D03B00200C
:10E5F00082B0064B002201920193019B03EB800045
:10E600000190019B186802B0704700BF502800407D
:10E6100082B0064B002201920193019B03EB800024
:10E620000190019B196002B0704700BF5028004064
:10E6300000B583B009238DF80730FAF737FA8DF863
:10E6400007009DF80730012BF7D09DF8070003B0B5
:10E650005DF804FB104B70B4DA6843780178867873
:10E660000E4CD243C2F30222C2F10405E8B2834049
:10E670000F2040FA02F23240DBB2134360181B0154
:10E6800001F01F0501224909DBB2AA4080F80033DE
:10E6900044F8212070BC704700ED00E000E100E08C
:10E6A000C27802B1D6E7037805485A09203203F050
:10E6B0001F03012101FA03F340F82230704700BF25
:10E6C00000E100E0002871D0F0B58388B3FA83F34D
:10E6D000202B0A4683B00446C3F11F0150D0344FAB
:10E6E000344D07EB81036E18C3F84426002196F8D9
:10E6F000BC6338F0C1F8A38821682F48B3FA83F3CC
:10E70000C3F11F0202F0FC0404F1804404F59C34C0
:10E7100002F003024FEA820E4FF00F0C01F13F426C
:10E72000A1680CFA0EFC21EA0C01A16002F57E0240
:10E73000A168C2F387224FF0004C02FA0EF22CFAC5
:10E7400003F30A43A260436102681C4922EA030200
:10E750000260426822EA0302426002681A430260D1
:10E76000826822EA03028260C26822EA0302C2606F
:10E770000A68374413430B6097F88436F02B01D8AE
:10E7800003B0F0BD3544F02195F8CC338DF804305A
:10E7900003224FF4807301A887F884168DF80520B2
:10E7A000ADF80630FFF756FF03B0F0BD704700BF6D
:10E7B000D03B002000EC0508003C0140083C014033
:10E7C0002DE9F041C54BC64EC64DC74C0822C3F8D3
:10E7D0008820336B82B043F00103336307464FF464
:10E7E000C052284640F2023388466946CDE90023EC
:10E7F000F9F706FC6B6AC4F8708C23F470436B6203
:10E800006B6AC4F8787C43F420436B626B6AB74947
:10E81000C4F8741C23F470236B626B6AB448C4F8A8
:10E820008C0643F420236B62736CB249C4F89016D3
:10E8300043F480437364736BAF48B049C4F89C06DB
:10E8400043F0800302257363AD4F84F89456AD4EB8
:10E85000AD4DC4F8E0164FF0A043C4F89836AB4A6B
:10E86000C4F8A87603F53463A1F5D071C4F8E45672
:10E87000C4F8AC66C4F8E836C4F8B0160123DFF873
:10E88000BCC2C4F8A4C607F51077A5F5E465A6F5E3
:10E89000A066A1F58C61C4F8EC76C4F8A056C4F863
:10E8A000586784F8973605F5A075536106F5B0767C
:10E8B000C4F81C1784F89E371946954B954AC4F83E
:10E8C0002457A7F5BC67A035C4F83067924EC4F84A
:10E8D0002C77C4F8343707F5D45703F56953C4F8D7
:10E8E00038574FF050250020DFF854E2C4F85C2779
:10E8F000ACF5687C02F5A042C4F86077C4F86467A0
:10E9000007F5A04706F5A046C4F86837C4F86C5769
:10E91000A3F5485304F28C65C4F87027C4F87867EF
:10E92000C4F89837C4F820E7C4F828C70246C4F8EA
:10E9300074772B4684F8A007402683F81C21A3F89F
:10E9400022210132042AC3E9496083F81D1183F8AA
:10E950001F01C3F8300103F12803EED10022114654
:10E960002B46402083F87423A3F87A230132042A2B
:10E97000C3E9DF0183F8751383F87713C3F88813AD
:10E9800003F12803EED14FF0A04364489A6822F0C7
:10E9900001029A60DA6842F04002DA60F9F7FEFCA0
:10E9A00094F895360022212161F317420BB142F40D
:10E9B000801294F88F16D4F8983601299A6300F0E3
:10E9C000E480DA68D4F89867D4F89C06C2F307614B
:10E9D00021F0600141F0400161F31F620021DA6023
:10E9E0003160026861F3CC22026094F89726012A14
:10E9F00000F0B88010214A48F9F74CFE4848F9F772
:10EA00002FFED4F89C0694F88D3600224FF0FF318B
:10EA1000026142618161C26153B305F11407414E45
:10EA2000114607EB83074FEA830C4FF0FF0E56F8B1
:10EA3000042F1368002BACBF00234FF09043B74264
:10EA400013601161C2F808E0F1D105F150033649B5
:10EA500063440027FF2651F8042F1568002DACBF32
:10EA600000254FF090459942156017619660F2D1EC
:10EA7000036994F88F1643F480730129036161D010
:10EA8000D4F8982629480023936100294FF0FF33DA
:10EA90006FF0804151615360516114BF0023102316
:10EAA000906143F470139069D4F8741C43F460537C
:10EAB00043F00803034393619368096843F001033B
:10EAC000936088471A4B1B4ADA6068461A4B0093DA
:10EAD000FFF7C0FD02B0BDE8F08100BF00E100E03B
:10EAE0000038024000000240D03B0020FC02002021
:10EAF000080401004000400100080050000B0050D5
:10EB00002009005040090050200B0050003C0140FB
:10EB1000C005005000100050003000506842002036
:10EB20005C42002070420020AC42002000080080BF
:10EB300000ED00E00005FA05430200010009005065
:10EB400020050050D4F89826144B03636FF08041E1
:10EB5000134D00234FF0FF309361516150605161BC
:10EB600095619EE701680F4A0F4E41F00301016075
:10EB7000802159629E62C3F80421E022C3F8082173
:10EB8000C0F24002C3F80C2134E79A6822F03E013B
:10EB900041F02A0161F307029A6012E70301810044
:10EBA00000080080A000400080002000024A136A94
:10EBB00023EA00001062704700380240F8B5764D35
:10EBC00005EB0013D3F8802C002A00F0968093F810
:10EBD000886C002283F88C2C044607013046FAF733
:10EBE000D5FE06F01F0276090123032E03FA02F375
:10EBF00000F09B80042E00F08980022E00F08180BE
:10EC0000EB19013493F8840C39F066F9E4B2064646
:10EC100010B11223C4718371EB1993F8850C39F08C
:10EC20005BF910B11323C4718371EB1993F8860C4F
:10EC300039F052F910B11423C4718371EC190A210F
:10EC400094F8872C304639F033FA94F8850C39F073
:10EC500043F994F8872C0A2139F02AFA94F8860CA3
:10EC600039F03AF90A2194F8872C39F021FAD4F8CE
:10EC7000801C4A4B99425DD0494B99424BD0494B3D
:10EC8000994261D0484B994268D0484B99426FD025
:10EC9000474B994276D03D4495F88C3C73BB012498
:10ECA0000220444A0D88B2F89261B2F89031B2F86D
:10ECB0009A71A2F898413343B2F89461A2F8960190
:10ECC0003343B2F89C613B43B2F89E7133433B43FC
:10ECD000B2F8A06105F44152134303439BB22343AE
:10ECE0000B808B8B23F400631B041B0C8B830E8225
:10ECF0000B889BB243F040030B80F8BD00242046F4
:10ED0000CFE72D4A516A0B43536279E72A4A1169CA
:10ED10000B43136174E7284A136A43F48043136278
:10ED20004FF48040FFF742FFB5E7234A116A0B43D7
:10ED3000136265E7204A536A43F4805353624FF4E9
:10ED40008050F9F7D3FEA6E71B4A136A43F4004349
:10ED500013624FF40040FFF729FF9CE7164A536AFD
:10ED600043F4005353624FF40050F9F7BFFE92E7AB
:10ED7000114A536A43F4801353624FF48010F9F739
:10ED8000B5FE88E70C4A536A43F4001353624FF40C
:10ED90000010F9F7ABFE7EE7D03B002000300140C9
:10EDA00000380040003C0040003401400050014069
:10EDB0000054014088010020003802404A4B98422C
:10EDC0002ED0B0F1804F33D0484B984237D0484BCB
:10EDD00098421ED0474B984238D0474B98423CD07F
:10EDE000464B984240D0464B98424DD0454B9842B6
:10EDF00041D0454B98424FD0444B984255D0444B5C
:10EE000098425BD0434B98425FD0434B984263D0CB
:10EE10007047424A136A43F0040313620420C5E6B4
:10EE20003E4A536A43F0010353620120F9F75EBE84
:10EE30003A4A136A43F0010313620120B6E6374AE7
:10EE4000136A43F0020313620220AFE6334A136AE7
:10EE500043F0080313620820A8E6304A136A43F01F
:10EE6000100313621020A1E62C4A136A43F020031A
:10EE7000136220209AE6294A536A43F4803353628E
:10EE80004FF48030F9F732BE244A536A43F002034C
:10EE900053620220F9F72ABE204A536A43F4003332
:10EEA00053624FF40030F9F721BE1C4A536A43F411
:10EEB000802353624FF48020F9F718BE174A136A73
:10EEC00043F040031362402070E6144A136A43F093
:10EED00080031362802069E6104A136A43F480734A
:10EEE00013624FF4807061E60000014000040040AE
:10EEF00000080040000C00400010004000140040DA
:10EF0000000401400040014000440140004801402D
:10EF100000180040001C0040002000400038024063
:10EF200010B504460068FFF749FF0D4BD3F84C2697
:10EF3000204652084FF6FF7136F0FCFF20460021B4
:10EF4000FBF7F2FF0749084A41F218532046CA501E
:10EF500001F5A851BDE810400022183136F06ABF13
:10EF6000D82A0020D03B0020CD9E010838B5124B96
:10EF7000D3F84C46054600686408FFF71FFFB4FB52
:10EF8000F1F3B3F5803F03D3012CFAD96408F6E717
:10EF9000224699B2284636F0CDFF0849084A41F288
:10EFA00014532846CA5001F5A851BDE83840002244
:10EFB000143136F03FBF00BFD82A0020D03B0020DC
:10EFC00045DA01082DE9F04FCCB2002185B00746A3
:10EFD0000846164639F074FA0021012039F070FA1B
:10EFE00038F002FF022E09D0042E44F6C01818BFD4
:10EFF0004FF49648072C06D900200BE0FF2C4FF465
:10F000001648F7D10326CD4D95F824342BB90020AE
:10F01000C5F8280405B0BDE8F08F032E0FD0C8490D
:10F020000C44002294F84304032137F099FA002895
:10F03000EDD0C44BC3F8F40CC3799A07E7D441F27E
:10F040000F53C04C95F82404E6540022032137F0F6
:10F0500087FA41F2F803E0500028D8D04FF48062DC
:10F06000B94BC4F8B03CC4F8BC2C0323C4F8C02C82
:10F0700004F5A852A4F8B43C0023137041F2FC42FA
:10F080004FF0010A24F802A041F2085204F6F841B8
:10F09000A35041F20C52C4F8C41CA35241F20E52C8
:10F0A00001F20441032EA354C4F8B88CC4F8DC3C2C
:10F0B000C4F8D03CC4F8CC3CC4F8C81CC4F8D83C54
:10F0C000C4F8D43C04F54B690ED0D4F8F4BC9BF8DA
:10F0D000040038F001FFC4F8F00C58460EF0C4FBF1
:10F0E000514648460EF0D4FB322038F013F9002E7A
:10F0F00065D141F2F80354F80380D8F80000FFF717
:10F100005DFE4046914A222136F014FF41F214532D
:10F110008F4AE25009F664013246404636F08AFED4
:10F12000D4F8F48CD8F80000FFF748FE874A4FF671
:10F13000FF71404636F0FEFE31464046FBF7F4FED6
:10F1400041F21853834AE25009F6680132464046BC
:10F1500036F070FEC5F828944FF0060A022E12D041
:10F16000D5F8280438F012FE68B10121002039F0EA
:10F17000A7F9D5F8280438F009FE0146002840F028
:10F18000A28039F09DF9384638F000FE88B101219F
:10F19000084639F095F94FF0050B4FF00008384656
:10F1A00038F0F4FD0146002840F09680012039F047
:10F1B00087F9042ED4D0052038F0ACF8CEE7012E24
:10F1C0000AD141F2F8034146E058FFF7CFFED4F8E8
:10F1D000F40CFFF7A5FEBDE7022E0AD1D4F8F40C1B
:10F1E0000EF031FB41F2F8034146E058FFF7BEFE56
:10F1F000B0E7032E5FD141F210534FF0000A04F83C
:10F2000003A051465448DFF858B140224FF0A7FC04
:10F210008DF80FA0DFF84CA19DF80F30072B0AD90D
:10F220004E4801210EF034FB41F2F8034146E0580C
:10F23000FFF79CFE8EE79DF80F3003EB43030BEBCB
:10F24000C30393F845307BB39DF80F3003EB4303C2
:10F250000BEBC3039B6C3BB39DF80F20384B13445F
:10F2600093F8430400B30022032137F079F90190A9
:10F27000D0B10EF0E8FA9DF80F309AF80010019A1C
:10F2800003EB43030BEBC30305EBC1009B6CC0F81E
:10F290002C34D379DB0748BF012301F1010148BFBA
:10F2A00080F830348AF800109DF80F300133DBB25B
:10F2B0008DF80F30B0E7042E7FF44CAFD4F8F40C87
:10F2C0000EF0C1FA7DE7D5F8280438F057FD014665
:10F2D000384638F05FFD4CE7384638F04FFD95F87A
:10F2E0007A3401468BB9242803D14FF0010385F805
:10F2F0007A34012E04D13846019138F04BFD019942
:10F30000D5F8280438F046FD49E7012B06D14D28F1
:10F310000CBF0223002385F87A34EAE7022B06D1DA
:10F320003C280CBF0323002385F87A34E1E7032B44
:10F3300026D10A2818D985F87A84DAE7C84C002043
:10F34000D82A0020D03B0020D4EF050840420F000F
:10F350001DD90108E99D0108F450002080480020D3
:10F3600014000010E0500020042385F86D0485F897
:10F370006C8485F86F8485F86E0485F87A34B8E774
:10F38000042B09D195F86E3485F87B04434085F849
:10F390006E3485F87AB4ACE7052BAAD195F86C34B5
:10F3A00095F86D9495F86E044B4509D25A1C2B4480
:10F3B000484085F86E0485F86C2483F8701498E74B
:10F3C0008842B8D195F87B3485F87AA4F42B90D193
:10F3D000B9F1000F8DD12421384685F87A9438F0A0
:10F3E000D9FC4D21384638F0D5FC3E21384638F05E
:10F3F000D1FC4946384638F0CDFCF421384638F087
:10F40000C9FCF421384638F0C5FC032E1BD0D4F8D3
:10F41000F40C437901689D080223AB40DB439BB2A7
:10F420000B828D892B408B81007920210EF0FAF917
:10F43000D4F8F40C4A46494636F0FCFCD4F8F43CC7
:10F440001868FFF7BBFC41F2F8050022605911462D
:10F4500036F0F0FC63591868FFF7B0FC0120D9E5DD
:10F46000224A936803F00C03042B10B421D0082B1C
:10F4700022D01F4B03601D4C1E4AA168C1F303112B
:10F48000114491F8A411CB404360A168C1F38221DB
:10F49000114491F8A41123FA01F18160A1685DF88B
:10F4A000044BC1F342310A4492F8A421D340C36013
:10F4B0007047114B0360DEE754685168526863027D
:10F4C000C2F388124CBF0C4B094B01F03F01B3FB58
:10F4D000F1F303FB02F3054A5268C2F30142013221
:10F4E0005200B3FBF2F30360C5E700BF00380240EF
:10F4F0000024F4008801002000127A002DE9F04F6A
:10F500009C4CD4F898365A69D2078BB002D50BB010
:10F51000BDE8F08F5A699B6912EA030AF7D0CAF373
:10F5200007431AF4002F009340F0DD81009B5D0734
:10F5300000F10C811AF0020F1EBFD4F89836022297
:10F540005A61BAF1000F5FFA8AF5C0F21C821AF410
:10F55000006FCAF3072740F0C3802E0708D5864BFB
:10F560008648D3F8C0319847D4F8983608225A61B3
:10F57000ED0620D4F80676D4B90632D4009BDA061C
:10F5800009D57D4B7D48D3F8D0319847D4F89836CB
:10F590004FF480125A61009B9B06B8D5764B774892
:10F5A000D3F8D4319847D4F898364FF400125A6102
:10F5B0000BB0BDE8F08FD4F898369A6922F01002AB
:10F5C0009A611A6AC2F34340022802F00F0100F068
:10F5D0001882062800F0F6819A6942F010029A61BA
:10F5E000C8E7D4F89C36D4F8A4169A680868C2F321
:10F5F0004102022A08BF03224FF0000514BF65F341
:10F600000A0062F30A0008605A6842F480725A6085
:10F6100006A8FFF725FFD4F89826D4F89C06D368EF
:10F620005749079D6FF38D23D3608068C0F3410075
:10F63000014491F80414032900F0D881514952483B
:10F640000126294484F88E6681424FF04006A4F8D2
:10F65000906600F21F820E2161F38D234FF400515A
:10F66000D36051618AE7D4F89C26444853684FF030
:10F67000000823F0010341465360F9F70BF894F8B2
:10F680008D66414656B1414BFF2203EB860653F887
:10F69000045FD86BAA609E428260F8D1D4F89C3691
:10F6A00036484FF0FF329A614FF00112DA610B22B7
:10F6B00062F3070162F30708C3F8148019611A683E
:10F6C0006FF30A121A60F8F78FFED4F898262A4BC7
:10F6D0002A48D3F8C4314FF48051516198474BE721
:10F6E000254B94F89E27D3F8C831244800218DF883
:10F6F00017108DF817209847D4F89C16D4F8982640
:10F7000094F8963688684FF400615161002B3FF4FD
:10F7100024AFC3077FF521AF94F8A137012B7FF405
:10F720001CAF9DF81730032B7FF417AFD4F8983730
:10F7300017491A6842F001021A601A6842F003027F
:10F740001A600B6943F006030B6106E7D4F89C26A8
:10F750009369D26913401FFA83FBBBF1000F3FF49A
:10F76000E9AEDFF81880CDF80CA045464FF000094F
:10F770001AE000BFD03B0020880100205C4200203E
:10F7800000EC0508401E1BFF3F420F0070420020A6
:10F7900000ED00E05FEA5B0B09F1010908F10408E4
:10F7A00005F1280500F00B811BF0010FF2D0D4F811
:10F7B0009C165FFA89F708694A6B04EB8703FA40E5
:10F7C000D3F8A436D2019B68D2B202431A40D007C4
:10F7D000D3B216D54B6BD8F81820012000FA09F0E7
:10F7E00023EA00034B63BF4BBF48D3F8B831012174
:10F7F00091603946984794F88F66012E00F02E816B
:10F8000001231A0742BFD8F8182008239360DE06A8
:10F8100042BFD8F8182010239360580642BFD8F88A
:10F82000182040239360990742BFD8F8182002237C
:10F8300093601A06AED5D5E94C60D5F82431D8F8D6
:10F8400018C0311A8B42DCF8182028BF0B4603334E
:10F8500092B2B2EB930F9DD9D4F89C26323704EBC9
:10F860008703CDE9019890469946B04238D2BEB39D
:10F87000D5F8241194F88F36D5F82821371AB942D3
:10F8800028BF394601F1030E4FEA9E0E83B98FB2AD
:10F890000337BF10D9F894A60AD0013352F8040BED
:10F8A000CAF800009F42F8D1D5E94C60D5F828216C
:10F8B000DCF8183008440A44B042C5F82821C5F8DD
:10F8C00034010AD195F81C11D8F83420012707FA21
:10F8D00001F122EA0102C8F834209BB29E45C4D34C
:10F8E000DDE9019856E7D4F89C369D69DB691D4037
:10F8F0002D0C3FF41BAE04F28C66DFF8E8B1B04685
:10F90000B146002708E06D0807F1010706F104067B
:10F9100008F128083FF40AAEEB07F4D5F9B204EB7E
:10F920008102D4F89C36D2F8E02692685B691A40CE
:10F93000D007D3B218D594F88F06726D0123984280
:10F94000936007D11269D8F87C33C2F312029B1A74
:10F95000C8F88C33DBF8B4314846984794F88F36B2
:10F96000012B00F0898001239A0742BF726D0223A8
:10F9700093601B07C7D5DBF8BC3148469847736DC9
:10F9800008229A60BFE794F896363BB1D4F89827DE
:10F99000136823F0030161F307031360D4F89C2676
:10F9A00050495368D1F8CC114F4823F001035360FC
:10F9B0008847D4F898364FF000425A61C7E5DDF821
:10F9C0000CA0B7E501EB8101D4F85C5704EBC10151
:10F9D0002E68D1F8180AC4F8586CC2F30A1202440F
:10F9E0002868C4F85C0CC1F8182AF5E500214FF42A
:10F9F000007084F88E160921A4F8900661F38D2317
:10FA00002CE647F6F07010423FF4E6AD01EB8100C2
:10FA1000C2F30A1204EBC00002F1030C5FEAAC0C63
:10FA2000D0F80C5AD4F85CE74FEA810818BF0020E0
:10FA300006D00130DEF8006045F8046B8445F8D14B
:10FA4000414404EBC101D1F80C5AD1F8180A15440D
:10FA50000244C1F80C5AC1F8182ABDE5B9F1000FEB
:10FA60007FF4CEAE94F89D37042B7FF4C9AE1E48C8
:10FA7000F8F7BAFC3346C4E6002F7FF474AF94F86D
:10FA80009D27052A7FF46FAF48460193F8F7ACFC39
:10FA9000019B69E71548A5F57401A1F51051814254
:10FAA00003D80D2161F38D23D8E51149114829446C
:10FAB000814203D20C2161F38D23CFE50E48A5F1DD
:10FAC0008C71A1F54341814203D80B2161F38D2351
:10FAD000C4E50A490A482944814213D20A2161F344
:10FAE0008D23BBE5880100205C420020DFC81000A8
:10FAF0002013FBFE20D61300FF69180000D3CEFEB2
:10FB000040771B00134914482944814203D209213C
:10FB100061F38D23A2E51148A5F1B771A1F5585104
:10FB2000814203D2082161F38D2397E50C490D48EA
:10FB30002944814203D2072161F38D238EE50A49CE
:10FB40000A482944814234BF0621052161F38D23EF
:10FB500084E500BFC05BB3FEC091210040AC27002C
:10FB6000C01D6AFE40E13300803C36FEE09C41004F
:10FB70000D4B93F8962612F0010F0C4A03D0012387
:10FB800082F87C34704792F87C2462B9D3F8D4268A
:10FB90004AB193F88C26104493F88D2683F88C068E
:10FBA000114483F88D167047D82A0020C84C0020D5
:10FBB000044B93F9CC08012806BF022283F8CC2815
:10FBC00000207047E0190020124AD2F88004B0B13A
:10FBD000D2F884349BB188420FD88B4234BF0023C3
:10FBE0000123ABB10C4BC2F88814D3F8D03899423A
:10FBF0001CBF142382F88C34DAE70023F1E7A1F567
:10FC00009C53083BB3F57A7F2CBF00230123E8E720
:10FC1000704700BFC84C0020E019002007B5002342
:10FC20000DF10602ADF806300DF054FB70B1094934
:10FC3000BDF80620B1F8D418074B9142A3F88E24E2
:10FC40001CBF142283F89024FFF7B2FF03B05DF8C5
:10FC500004FB00BFE0190020C84C002013B5044687
:10FC6000262001911BF0BAFE019948B9054BD3F843
:10FC700038392BB1204602B0BDE81040F9F736B84C
:10FC800002B010BDE0190020B1FA81F14909492004
:10FC9000E4E7F7B5C24C94F9CC3801330E4600F0D6
:10FCA0007C81D4F83839002B00F0B880BD4D022794
:10FCB000D4F8380938F06AF8002800F0AF80D4F89A
:10FCC000380938F05BF8D4F840395A1C2B44C4F892
:10FCD000402983F8910494F83C39012B08D0022B79
:10FCE00015D05BB90F280CD1012384F83C39DFE72C
:10FCF000A0F17203012B07D9762805D0002384F8E0
:10FD00003C39C4F84039D3E784F83C79D0E7102A6D
:10FD1000CED1A5490023012211F8010F013203447D
:10FD20000E2ADBB2F8D1002284F83C29C4F840291D
:10FD300095F89F249A42BBD195F8A034002BB7D1F7
:10FD400095F89234732B5FD0762B1CD0722B65D133
:10FD500095F8942495F8933494F9CC1853EA022337
:10FD60005CD0C5F880340029B5F89534C5F88434E2
:10FD700054DC95F8AE24012384F8CC38002A4DD108
:10FD800085F8AE344AE095F8942495F8933453EA14
:10FD9000022343D0D5F8A42495F8961495F89A0434
:10FDA000C4F8D03893421CBF142285F88C2495F8EF
:10FDB0009524C5F8A43442EA0122B5F8A814A4F8A1
:10FDC000D42891421CBF142185F8901495F89714FB
:10FDD00084F8CD1895F8981484F8CE1895F89914ED
:10FDE000A5F8A82441EA0021A5F8AA14D5F888149A
:10FDF00009B9C5F88834B5F88E340BB9A5F88E2446
:10FE0000022384F8CC3809E095F8982495F89734C3
:10FE100043EA02231AB20BB1A5F8AC2494F9CC380A
:10FE2000022B39D011DCDAB2012A18D9D4F82439DE
:10FE30001BB1D4F8D838002B76D15C495C481F221E
:10FE400003B0BDE8F0404EF0C8BE032BEED1554DD7
:10FE5000584AD5F8B034F31A9342E7DD14E0514D17
:10FE60005549D5F8B024B21A8A42DFDD2BB9722089
:10FE7000F8F768FFC5F8B064D8E7D5F8B4345A1C71
:10FE8000D907C5F8B42403D47620F8F75BFFF1E76F
:10FE90007320F8F757FFEDE7424DD5F88814E9B124
:10FEA00095F88C34D3B1D4F8D038994216D094F860
:10FEB000CD38DA0703D489B24620FFF7CFFE95F894
:10FEC0008C34013B85F88C3406F59226032306F525
:10FED000787684F8CC38C5F8B064A7E7B5F88E1406
:10FEE000B4F8D43889B195F8902472B18B420CD013
:10FEF00094F8CD38DB0702D45020FFF7AFFE95F819
:10FF00009034013B85F89034DEE7012284F8CC2858
:10FF1000A5F88E34D4F8D028C5F88824002385F8B5
:10FF2000903485F88C3481E7244B254DD3F8D47672
:10FF30002A2385F8E0310DF1070220230DF1060197
:10FF4000384685F8E1310DF05CFA30B19DF80610C5
:10FF50009DF8076051EA06033CD1552385F8E2314C
:10FF6000462385F8E331D4F8D0281648202385F8B5
:10FF7000E431002A3BD014493FF090F8094B134874
:10FF8000B3F8AA34002B36D0B4F8D42810499A42DA
:10FF90000CBF20222A223FF081F803B0F0BD00BF41
:10FFA000E0190020C84C0020595100209477060821
:10FFB00068030020400D030040420F00D82A0020B3
:10FFC000880100206D03002058F20608710300200C
:10FFD000AE77060838460DF0F9F9314685F8E201AA
:10FFE00038460DF0DFF9037885F8E331BBE70449C3
:10FFF0003FF054F8C2E703493FF050F8CDE700BFA7
:020000040801F1
:10000000B6770608B577060810B50E4C40F0080222
:1000100084F8032294F9F820022A06DD420704D569
:1000200083071CBF012384F8003105210648F8F737
:1000300021FE062184F80402BDE810400248F8F7CA
:10004000FFBD00BF880100208703002010B5F8F72E
:10005000A7FDA8B31B4C94F9F830012B30DD59B340
:10006000022B2DD094F800319BB971B1802305216A
:10007000154884F80932F8F7FDFD062184F80A02D4
:10008000BDE810401048F8F7DBBDBDE81040042083
:10009000BAE7002914BF0020042094F8FB301A07A7
:1000A00048BF40F002005B0701D411B108B940F02D
:1000B0000100BDE81040A7E7022BD3D10420ECE7F4
:1000C00010BD00BF880100208D030020F8B5224C30
:1000D00004F20B27030A84F810020546062138466D
:1000E00084F80F32F8F7C6FD94F8FB3084F811025B
:1000F000DB072AD4B4F8FC20AA4226D1174DD4F845
:100100000B32C5F8B834C3B285F8BE3441F26F7112
:100110004FF6FF738A4218BF0123134405F5976613
:10012000C3F307220621304685F8BC2485F8BD3488
:10013000F8F7A0FD072185F8BE043046F8F780FDEA
:10014000052104F21220F8F77BFDBDE8F8400448D1
:100150000721F8F775BD00BF88010020C84C0020BA
:100160009303002008B5F8F71BFD48B1A1F59C5397
:10017000083BB3F57A7F03D2BDE808400846A5E7FF
:1001800008BD2DE9F74F704DD5F85036002B3CD007
:100190006E4E6F4C06F1F807D5F8500637F0F6FDB5
:1001A000B0BBB5F87426092A0CD9B5F876166423C5
:1001B0004B43B3FBF2F3452B40F3B281A5F8740631
:1001C000A5F8760694F8F934012B00F0D781022BBC
:1001D00000F0F28133B95F480521F8F731FD0123C2
:1001E00084F8F93495F88236D5F83864002B00F09D
:1001F000ED81D5F88436F31A782B40F2E781D5F8F3
:100200008806F9F71DF9C4F8FC6403B0BDE8F08F67
:10021000D5F8500637F0B2FD94F8BF348046052B70
:10022000BAD8DFE803F00309161C3745AA28B3D172
:10023000012384F8BF34AFE755281BBFB5F87836E3
:1002400001330223A5F8783618BF002384F8BF34A1
:10025000A2E7032384F8C00484F8BF349CE7132882
:1002600084F8C104C4F8DC0408DDB5F87A3601333B
:10027000A5F87A36002384F8BF348DE718B9052332
:1002800084F8BF3488E70023C4F8E034042384F8FA
:10029000BF3481E7D4F8E034E218013382F8C204B5
:1002A000D4F8DC24C4F8E03493427FF475AFE6E779
:1002B000D4F8DC34284803F102094FFA89F1F8F741
:1002C000D9FC804594F8C0A440F0218126201BF081
:1002D00085FB58B1002385F88236B5F876360133B0
:1002E000A5F87636002384F8BF3455E795F88236B2
:1002F00053451AD1002385F882360AF1FF33102BBB
:1003000000F2FF80DFE813F02A0092009200E7007D
:100310009200FD00FD00FD002A00FD00FD00FD0033
:10032000FD00FD00FD00FD002A00BAF1090F02D01A
:10033000BAF1110F01D1012BDCD0B5F87E360133B3
:10034000A5F87E36D9E700BFD82A00208801002012
:10035000C84C00209A03002088510020B9F1060FF4
:1003600064DDBAF1010F00F0A280BAF1090F0CBFF1
:100370000223032394F8C51494F8C60494F8C42403
:1003800094F9C2A494F9C4E494F8C38486F8F830CC
:1003900040EA012001B2900786F8F9A086F8FBE058
:1003A0000091A6F8FC1006D512F00C0F14BF012224
:1003B000002286F80021032B15D1B9F1090F35DD94
:1003C00094F9C824082AA8BF082222EAE27286F813
:1003D00010214FF0000C4FFA8CF18A420CF1010C05
:1003E00067DC94F8C7848A4A4FF0000CD2F8D8181A
:1003F0000191934661461FFA88F801988142894627
:100400005FDB92F8191D86F8FAC023290ED103EBA1
:10041000830303EB83030EEB8303A2F81C3D009BD5
:10042000A2F81EADA2F8203DA2F822CD79497A4863
:100430000A224EF06CFB10B1002384F8EE34754BA9
:100440003A681A607A685A603A891A8194F8EE34E8
:1004500043BB96F8003195F88C2684F8F024002BE5
:1004600014BF0223012384F8EE3496F8FB3095F88C
:100470008E0684F8F40413F001031CBFB2FA82F371
:100480005B0995F88D2684F8F124D9B2B5F8902649
:1004900084F8EF14A4F8F22413B10AB1A4F8F624F6
:1004A00084F8F8140DF070FF0DF06EFF15E7534659
:1004B00060E705EB4108214491F8CA14A8F8C0167A
:1004C00089E70BEB49090131B9F8DC9849B2C1451C
:1004D00008BF8C4691E7B9F1040FA7DD94F8C22458
:1004E00094F8C33443EA022359041AB204D5C3F37F
:1004F0000D03A6F8FE3099E7002AF8DBA6F8FC30D9
:1005000094E7B5F880360133A5F88036E5E61AF0B1
:10051000010F02BFB5F87C360133A5F87C36E1E661
:100520003E4BD3F81822B3F81C12012A1DD141F218
:100530005632914203D14FF0FF32C3F81822D3F85C
:100540001822D5F8500602EB820202EB820201EB80
:10055000420189B2A3F81C1203681B699847002363
:10056000A5F87436A5F876362CE60132E7D1B1F558
:10057000965F04BF0122C3F81822E0E7274E96F9E0
:10058000F870002F3FF42EAE022F11D14FF48040AF
:10059000FFF79CFD84F8F97496F9F830012B7FF78A
:1005A00021AE96F8FB30C3F3400386F8003119E61C
:1005B000032384F8F934EFE7184BB3F8FE30002B2F
:1005C0003FF410AE032384F8F9340BE6104B93F894
:1005D000F02893F8F1389A4204D0F8F761FFC4F894
:1005E000FC6412E6D4F8FC34F31AB3F57A7FBFF456
:1005F0000CAED5F88436F61A952E7FF606AE08486E
:100600000521F8F71DFB03B0BDE8F04FF8F748BF30
:10061000E0190020AC510020800200208801002059
:100620009A03002010B5114C94F8963623B9104B5C
:100630004FF480225A6110BD0E4A136823F006035E
:1006400013604AF0DDF994F89636002BEFD0D4F819
:100650009C369B68DB07EAD5D4F89827136823F00B
:10066000030161F307031360E1E700BFD03B002003
:10067000003C014010ED00E008B501210320FDF72A
:10068000C7FF72B645F010FC2DE9F04FCB4CCC4DB6
:100690008DB000270090A4F67F5805F5A16A54F8A4
:1006A0000B0C002800F0FE8037F070FB0646002897
:1006B00000F0CF81D8F8383444F8073CE026002316
:1006C000A4F10B0B04F8033C06FB078654F80B0C53
:1006D00037F05CFB002800F0E58054F80B0C37F095
:1006E0004DFB14F8023C5A1E81460B2A0DD8DFE858
:1006F00012F020003B004700540083009A00E20003
:10070000130131013C016F01850124280DD0009AAD
:1007100042B9AC4A92F87224824240F075810122BB
:1007200004F8032C0D2BD1D184E0012304F8023C02
:10073000CCE700234D28C4F8C53084F8CD3084F8C8
:10074000CE3004D0582808D004F8023CBEE702227C
:1007500004F8022C84F8C430B8E7032304F8023C00
:10076000022384F8C430B1E704233C2804F8023C97
:100770000BD0B9F13E0F0CD0002304F8023CA5E7E2
:100780000A233C2804F8023CF3D1002304F8013C7E
:100790009CE7012304F8013C98E7D4F8C5305A1CC3
:1007A0003344C4F8C52083F87F0D94F8CD00022AA5
:1007B00089EA000184F8CD1088D12378C02BDBD8DA
:1007C0006278FF2A08D1052BD6D9012384F8C430DA
:1007D000072304F8023C79E7A4F8C12000229342E1
:1007E000C4F8C93014BF0523062384F8C320C4F815
:1007F000C52004F8023C69E7D4F8C5305A1C3344DC
:10080000C4F8C52083F87F0D94F8CD00D4F8C93022
:1008100089EA00019A4284F8CD107FF457AF06238D
:1008200004F8023C52E794F8CD308342A4D10D2362
:1008300004F8023C14F801CCBCF1000F40F0EA804F
:10084000614B08940FCB04AE86E80F00D4F8C93092
:10085000D4F8D100ADF82CC023440993B4F8C130CA
:10086000ADF8283094F8C3308DF82A3001238DF884
:100870002E30324603AB08A9CDF80CC02FF08EFF06
:1008800048B1049B059394F8C420504B049331461F
:10089000584626F0F7FB039E002304F8023C002E86
:1008A00040F0CF800137032F04F1E0047FF4F7AE6E
:1008B0000DB0BDE8F08FD4F8C520531C3244C4F805
:1008C000C53082F87F0D94F8CD2001934240014657
:1008D00094F8CE0084F8CD203EF098FC019B84F87B
:1008E000CE00072B7FF4F2AEB4F80530C02B3FF6F4
:1008F00043AFB4F80320A4F8C120A27884F8C32041
:1009000000229342C4F8C93014BF08230923C4F855
:10091000C52004F8023CD9E6014694F8CE003EF02A
:1009200075FC94F8CD3084F8CE0089EA030384F88E
:10093000CD30D4F8C5305A1C3344C4F8C52083F8F0
:100940007F9DD4F8C9309A427FF4C0AE092304F8E1
:10095000023CBBE694F8CD30434084F8CD3094F8A7
:10096000CE3083427FF408AF59E7D4F8C520531C3A
:100970003244C4F8C53082F87F0D014694F8CE00A9
:1009800001933EF043FC019B84F8CE00052B7FF4DD
:100990009DAEB4F80120B4F80330A4F8C120227849
:1009A00084F8C32000229342C4F8C93014BF0B233B
:1009B0000C23C4F8C52004F8023C87E65738002011
:1009C000C84C0020D03B002008F00508E4010120BD
:1009D000014694F8CE003EF019FCD4F8C53084F8F6
:1009E000CE005A1C3344C4F8C52083F87F9DD4F848
:1009F000C9309A427FF46AAE0C23A5E694F8CE3053
:100A000083427FF4B9AE12E7232804BF022204F820
:100A1000032C87E6BCF1010F4FF0000602D004F86A
:100A2000026C3FE7D4F8C93008942344099308A81E
:100A3000B4F8C130CDE90A66ADF8283023F0AAF940
:100A4000EDE754F80B0C2DF0C1FE54F80B0CB04739
:100A500028E714F8033C002B3FF424AFD8F83824DF
:100A600054F8071C521A632A7FF61CAF012B31D0B1
:100A7000022B7FF417AF54F80B3CC5F80035C5F8CE
:100A80000435C5F80C35402385F81035124B85F830
:100A900011050122C3F840A313F8C93C88F8D026F9
:100AA0000E4AC5F80825003B0D4A0E48C5F854A566
:100AB00018BF012382F8AC3B3BF08CFE4FF4005092
:100AC0002FF032FD08483BF07BFE85F8586585F82D
:100AD0005965E7E6FFF7D0FDD03B0020C93A04088E
:100AE00014000010BB770608F17706080023038086
:100AF00083708380C3800372704700BF054A064934
:100B0000137809780133DBB29942137004BF0023D4
:100B10001370704780640020C40B0010F8B56B4C54
:100B200063687BB16A4B1B6893F82E3053B1694BF5
:100B3000227AA3FB0013012A4FEA93132BD0022A37
:100B400007D002B1F8BD644B9842FBD90123237250
:100B5000F8BDE26864329A4235D8237804EB031377
:100B600093F82020FF2A05D05C490132012083F848
:100B700020200870FFF7C2FF594B1B780122092B78
:100B80002272DFD1B4F8A230564A01339BB2A4F8E6
:100B9000A2305380F8BD544D21785148E3608C2336
:100BA00003FB015300789A700023A37704F1140526
:100BB0000A22022309282561E2772372C2D1494B18
:100BC00001311980F8BDA27FE37F9A42BAD104F1C6
:100BD000130004F11C05002310F8012F08215340D5
:100BE0005A0013F0800F08BF5B0082F0070214BFA9
:100BF000D3B2DBB20139F3D18542EDD1627F9A42A3
:100C000030D12678E57E237FB4F81700B4F8192098
:100C100094F815C004EB061743EA0523A57D87F871
:100C2000201040BA52BA81B292B245EA0C202B4D44
:100C300079621BB294F91410BA62032E4FF00102CC
:100C40007884BB8587F821102A7008D8244A127846
:100C50000C2A26D00D2A02D1224B23F81610FFF7BA
:100C60004DFF73E7237804EB031393F82020FF2A4A
:100C700005D01A490132012083F820200870FFF7BF
:100C80003DFF174B1B780122092B22727FF45AAFCC
:100C9000B4F8A030134A01339BB2A4F8A03093807B
:100CA000F8BD1249124A897E0E4803EB830303EB19
:100CB000830349089B0093FBF1F382FB0312DB17CC
:100CC000C3EBA20320F81630C9E700BF8064002000
:100CD0005C090010D34D62103F4B4C00A80300206C
:100CE000F9260020FC260020F8320020142F0020D6
:100CF00067666666084B997FDA7F91420BD010B425
:100D00009A7F1C69511CD2B2C0B2C9B29977A05463
:100D10005DF8044B7047704780640020FD2870B573
:100D200022D0F02804D0EF2822D00224204670BD23
:100D3000114D0320052641282E444FF0000405F1F3
:100D4000010580F080030DD0042B0BD9FFF7E6FFDF
:100D50002044B542C4B2E9D015F8010B412880F017
:100D60008003F1D10420F3E7044D0B200426E2E7D1
:100D7000034D0C200626DEE770F505086CF5050826
:100D800078F505080E4B0F4AD3F8A430B2F90400E9
:100D90005B0707D400EB8000400080B200F5C8700C
:100DA00080B27047084B094A9B6B323382FB0312B7
:100DB000D817C0EBA20080B200F5C87080B27047AF
:100DC00080640020C40B00105C37002067666666F4
:100DD0000C4AD2F8BC3030B41C68D2F8B4505D6014
:100DE00019810025611C19609D812070D2F8BC30EA
:100DF000D2F8B4101A685A604FF6F67230BC196017
:100E00009A817047806400200E4B30B4D3F8602282
:100E1000C3F8642203F5A07503F5147403F1C00050
:100E200003F5A8710132C3E92E54C3E9500030BC68
:100E3000C3E99411C3F86022C3F8B000C3F8B4103A
:100E4000704700BF8064002000B583B00268084B83
:100E50008188CDF801203222D3F86832ADF8051030
:100E60008DF800206846984703B05DF804FB00BF8A
:100E7000806400205E2810B511D05D2805D00D4B90
:100E8000BDE81040D3F86C3218470A4CD4F86C32E5
:100E90009847D4F86C323D20BDE810401847054C07
:100EA0005D20D4F86C329847D4F86C323E20BDE80F
:100EB000104018478064002030B401234FF40075BF
:100EC00015244FF4167140F2D93203800023458077
:100ED0008471018130BC4281838083817047094BDA
:100EE000B3F87222B3F87032801A9B1AC00090FBDC
:100EF000F3F00628A8BF062020EAE070C0F19600B3
:100F0000C0B2704780640020094B03EB4002B2F886
:100F10008A12084A527802EAD122520707D0D3F83F
:100F20000023511CC3F80013134483F804037047D3
:100F300080640020A803002010B5154A416892F88B
:100F40003F3303F00303032B1FD1B2F84033CBB17F
:100F5000B2F94233B2F948230A2492FBF4F29B1A05
:100F60001B0103F5B95314334FF4B472B3FBF2F31E
:100F7000C3F1080303F00F0360330B7043680022D2
:100F80005A7010BD05230B70F8E72D230B70F5E7A1
:100F900080640020436872221A70436873225A707A
:100FA000436874229A7043680022DA7070470F4BCE
:100FB0004268B3F948330A2193FBF1F31B0110B5E2
:100FC00003F5B9530A4C4FF4B4711433B3FBF1F386
:100FD00003F00F03E118E35813604B6853600B7A7A
:100FE0001372436800225A7210BD00BF8064002053
:100FF0007EF50508084B93F8513333B942F210736C
:101000005843064B90FBF3F07047242358434FF4AA
:101010007A7390FBF3F070478064002040D20600A2
:10102000054B93F851332BB94FF4A4735843642301
:1010300090FBF3F0704700BF80640020831E00F136
:101040007402EA2123F8021F9342FBD143F64913AD
:101050004385CD2383804E23C380CE230381232366
:10106000A0F87230704700BFE8B91D48B0F8B4333B
:1010700003F001034BBB30B490F8B8438CB1194A6C
:1010800002F1F00552F8041B490441BF90F8A41482
:1010900000EB8101D1F83C1445F823100133A34241
:1010A000F0D130BC70470E48B0F8B423032A4FEAA1
:1010B00052030BD90A68A0F8B43302F5C332A03248
:1010C00003F001030A60002BD5D070470B6803F5CD
:1010D000C333A03348F205020B60A0F8B423704775
:1010E000806400203C6800202DE9F04100283AD1BE
:1010F0002D4A92F8B80380B32C4A2D4B92F804E0A5
:1011000092F905C092F90680CEF1FF07AEF17F0695
:10111000FFB2F6B203EB800003F1F002002403E01B
:10112000834202F1040218D053F8041B8904F7D556
:10113000E1B2A1EB0C0181EAE175A5EBE175012DAE
:101140000DDC71B1414514BF394631468342D1703F
:1011500004F1010402F10402E6D1BDE8F0810821A6
:10116000F4E77146F2E7114B1A79F02A09D802F137
:101170000F000D4A18710B6803F582431A330B6098
:10118000B7E7094A93F9054092F8BA037F258442EC
:101190001D71987905DB4042C0B2987120445871A6
:1011A000E9E7002CFADAF6E780640020A8030020C3
:1011B0003C680020F0B5364E78B196F82C35002BFF
:1011C00046D0344A013BDBB286F82C351378DC0775
:1011D00041D4314B0A681A440A6096F8B8434CB3BC
:1011E0002E4B2C4F03EB840403F1F001002503E0A8
:1011F0009C4201F104011DD053F8042BC2F30320DB
:101200000628F5D13878C00715D596F82C0596F83C
:10121000BBE300EB050CBCFBFEF00EFB10C001288D
:10122000CCBF0020012058B99C4205F1010501F115
:101230000401E1D1F0BDE84300F001000028F3D043
:10124000C2F3834206EB8202D2F83C240A60EBE749
:1012500096F8BB33B5E7124A124BB2F90620124892
:10126000A2F57A74642202FB04F283FB0234D317E2
:10127000C3EBA41303EB4303C3EB031380FB030291
:10128000DB17C3EB62130533084A92FBF3F3A1E7C4
:10129000806400206E310020400D03003C68002077
:1012A0005C400020D34D62101F85EB5140420F007F
:1012B000F0B4534C002868D194F82D05002856D07E
:1012C000504BD3ED007AB3EE097AF4EEC77AF1EE23
:1012D00010FA4EDCBBEE097AF4EEC77AF1EE10FAA2
:1012E0004CBF08270027D3ED017AB3EE097AF4EE5C
:1012F000C77AF1EE10FA3EDD47F0010794F8B853D3
:10130000ADB3414ADFF80CC102EB850502F1F000F4
:1013100014E094F94165B142ACBF0221002194F977
:101320004265B3421CDB41F004010F421CBFDCF8F4
:1013300038300360954200F1040018D052F8043BA5
:10134000D903F7D594F9406503F00F01B142C3F317
:101350000313DEDC94F94265B3424FF00101E2DA97
:1013600094F94365B342D8BF41F00801DDE7F0BC12
:1013700070470427B7E7BBEE097AF4EEC77AF1EEBF
:1013800010FA48BF47F00207B8E794F82E356BB360
:1013900004F5A663D3ED007A93ED017A1B4D0A683C
:1013A00094F82D05F0EEE77AB0EEC77AF4EEC77A3E
:1013B000F1EE10FAB8BFF0EE477AFDEEE77A80F072
:1013C000010017EE903A193B03EB4303C3EB031301
:1013D00085FB0365DB17C3EBE51305330C4DB5FB4C
:1013E000F3F31A440A6084F82D0567E70B6894F854
:1013F0002D0503F5433303F5A0730B605EE700BFD3
:1014000080640020B06900203C680020353AFC442C
:1014100040420F006CF50508F0B40B4F97F8B86325
:1014200086B107F56F72054607F2AC47002352F804
:10143000044B35EA040004BF086847F82300013371
:10144000B342F4D1F0BC70478064002030B42A4B22
:1014500060B92A48027D3ABB93F8A5342849203365
:1014600001EB830130BC4FF4A060D5E793F844252D
:1014700062BB224893F84545057DA54293BF0424ED
:101480000134012283F8452592BF83F8444583F84F
:10149000454583F844250A6802F5C32202F5207207
:1014A0000A60027D002AD7D0D3F8A4209106D3D5B4
:1014B00093F83F2393F8441592070CD5A1B993F8FC
:1014C000A7340F49203301EB8301CBE7013A0B48E6
:1014D00083F84425DFE70029BED193F8A6340849F4
:1014E000203301EB8301BDE793F8A3340449203393
:1014F00001EB8301B6E700BF80640020BC3F002001
:101500003C68002010B41E4A48B91E4C92F84605AB
:101510000B6823440B6098B15DF8044B704792F858
:10152000473503B3012B16D092F846050B68164CCD
:1015300080F00100234482F846050B600028EBD1BF
:1015400092F8A33411495DF8044B203301EB830179
:101550004FF4407060E792F846050D4C80F00100B2
:1015600082F84605D4E70B685DF8044B03F5742355
:1015700003F5107301200B6082F84605704700BF29
:101580008064002040420F0048E801003C680020D1
:1015900020A107003C4AA0B992F848356BB192F8F7
:1015A00049158A081341DB070AD501F00101032A16
:1015B00006D8DFE802F05048403892F8513553BB66
:1015C000704792F84905013000F00F0082F8490594
:1015D00038B192F84835086800F5C330A03008608B
:1015E000DCE792F8793282F84805002B44D127488D
:1015F000C07818B143F0040382F8483524480078D5
:10160000C00730D592F850050028E4D043F0080315
:1016100082F84835DFE792F85E351E4901EB830119
:101620004FF40030F8E61B4B03F13002002914BFE1
:1016300019461146F4E7184B03F1180200290CBFB4
:1016400019461146ECE7134B03F10802002914BFB9
:1016500019461146E4E70F4B03F11802002914BFA5
:1016600019461146DCE7D2F84C050028CAD043F0F1
:10167000010382F84835C5E792F84735002BB6D00C
:10168000022382F84835B2E78064002070310020E0
:101690006E31002098F50508A8F50508024B0146B3
:1016A000D3F8600536F076BB806400202DE9F04168
:1016B000FD2984B0044600F0DE80F02900F0BD80F2
:1016C000EF2900F031814AB10346861803AD0020AE
:1016D00003F8010B9E4205F8010BF9D19A4B0B2040
:1016E00003F1090501E013F8010F814200F0C88001
:1016F000AB42F8D14B1E832B00F29380DFE813F04E
:101700003201390143014E01BD01840058016301DA
:101710006F01910091007501750175018B018B01BD
:101720008B016F019100910096019D019100910044
:101730009100910091009100910091009100910021
:101740009100910091009100910091009100910011
:101750009100910091009100910091009100910001
:1017600091009100910091009100910091009100F1
:1017700091009100910091009100910091009100E1
:10178000B3019100910091009100910091009100AE
:1017900091009100910091009100910091009100C1
:1017A00091009100910091009100910091009100B1
:1017B00091009100910091009100910091009100A1
:1017C0009100910091009100910091009100910091
:1017D0009100910091009100910091009100910081
:1017E0009100910091009100910091009100910071
:1017F0009100910091009100910091009100910061
:10180000910091001F011F01504BB3F87C12002979
:1018100000F06581019225F0ADF8019A80B2ADF833
:101820000C003AB1224403AB13F8011B04F8011B6E
:10183000A242F9D104B0BDE8F081454F03214FF039
:101840000508B844002501370CE0FFF767FA0646A3
:1018500060193246FFF72AFF70194745C5B2E9D033
:1018600017F8011B412981F08003084601D0042BA1
:10187000EBD80426ECE7374F0B214FF00408E0E7E4
:10188000324BD3F8A40080060CD4002AD2D02244D4
:1018900003AB13F8011B04F8011B9442F9D104B007
:1018A000BDE8F08193F83F03870742D52A4D287D94
:1018B000052834BF02260326142917D97C39C8B25B
:1018C0000628E2D80629E0D801A050F821F000BF90
:1018D000B71A0108B71A0108A11A01088B180108E4
:1018E000C71A0108C11A0108CD1A01080929CCD963
:1018F0000A390A29C9D801A757F821F0871A01081F
:10190000D31A01088B1801088B1801088B180108DD
:101910008B1801088B1801088B1801088B18010817
:10192000991A0108B71A01080C4F0C214FF006084C
:1019300087E7094B0B29187DA7D10126CAE0084B80
:101940005B6B03936DE700BFD0F505088064002052
:1019500070F505086CF50508BC3F002078F5050812
:101960005C3700200192FFF70DFA019AADF80C00E8
:1019700057E76B4BD3ED037AFDEEE77A17EE903A1B
:10198000ADF80C304DE7674B93F87705B3F8641565
:10199000002840F0AA80ADF80C1042E76149B1F888
:1019A000643591F89015B3FBF1F3ADF80C3038E7DE
:1019B0005D4B1B78DE0700F19D805A4BB3F87C32FB
:1019C000ADF80C302DE7574B5849B3F9483381FB3C
:1019D0000301DB17C3EBA103ADF80C3021E7514B3A
:1019E000B3F8A235ADF80C301BE7514BDFED516A6F
:1019F000D3ED027A0C39C9B203EB810393ED167A69
:101A000067EEA67A67EE877AFDEEE77A17EE903AF0
:101A1000ADF80C3005E7434B03EB4101B1F8263339
:101A200003EB83035B00ADF80C30FAE63E4B1B780A
:101A300003F00103ADF80C30F3E63A4BB3F8A01510
:101A4000CD055ABFCB4303F00103032311F0440F2C
:101A500018BF042311F0020F18BF072311F4806F81
:101A600018BF0923ACE70192FFF78CF9324B019ABA
:101A7000DB6B43EAC0400390D3E62A4BD3F894359E
:101A8000ADF80C30CDE62B8A03EB830303EB830325
:101A90009B00ADF80C30F8E6EB89ADF80C30F4E6BD
:101AA000EB89264903EBC3039B00A1FB03135B09EE
:101AB000ADF80C30E9E6B3F84033ADF80C30E4E6AD
:101AC0006B680393E1E62B680393DEE6AB68039350
:101AD000DBE6F6B28DF80C608DF80D00D5E6D3F894
:101AE0009C0580F3100080B299E693F89035B1FB25
:101AF000F3F150E701921CF02DFD094B019AD3ED53
:101B0000037AFCEEE77A17EE903A9BB200287FF456
:101B100057AF0B49096811F0100F18BF00234FE7AA
:101B2000B0690020806400206E3100206766666620
:101B3000C40B001000007A445C3700201F85EB5175
:101B4000F03E002070B5214D95F8A435EA181C46EA
:101B500092F8A8258AB11E4E09225C1CA6FB04132C
:101B60005B0803EBC303E31AE918DCB291F8A8158C
:101B700009B1013AF1D185F8A44502681549561C0E
:101B800006600C2616700268561C06600026167049
:101B90000268561C066003EB430603EB86031470D1
:101BA00019440D2240F036FA95F8A415084B4A1C4A
:101BB000A3FB02035B08294403EBC3030120D31AF0
:101BC00081F8A80585F8A43570BD00BF80640020A9
:101BD000398EE338346A0020084B93F8513307EE0E
:101BE000900A4BB9F8EEE77A9FED057A9FED050A6A
:101BF000A7EE870A4AF04EBC704700BF8064002001
:101C00006766E63F00000042032811D8DFE800F0D5
:101C10000A0C0206074BD3F830067047064B1B78B8
:101C2000DB0701D435F0F8BA024BD3F82C06704725
:101C300000207047806400206E3100202DE9F041C3
:101C40002A4C2B4AD4F89435B4F85876B4F89C65ED
:101C500082FB0352DB17C3EBA2031FFA83F847454D
:101C600082B00D4603D1B4F85A36B34233D002687D
:101C70000190511C34230160137002680023511C31
:101C800001601370414640F00DFA0198314640F072
:101C900009FA019847F6FF7140F004FA019847F6F7
:101CA000FF7140F0FFF9019847F6FF7140F0FAF933
:101CB000019847F6FF7140F0F5F901980221FAF713
:101CC00089FA0120A4F85886A4F85A66C4F85C562C
:101CD00002B0BDE8F081D4F85C36064ACB1A9342D4
:101CE000C5D8002002B0BDE8F08100BF80640020AC
:101CF0006766666680841E00026810B57F21541CEA
:101D00000460117002680024511C01600E211470DF
:101D1000FAF760FA012010BD2DE9F043744B1F68FB
:101D200083B0002F56D0FF238DF803308DF802309A
:101D3000002877D16F4B93F86026002A4DD093F896
:101D4000B853002D46D06C4A93F866166B489368DA
:101D500092F8078000294FF0000103F0010C14BF36
:101D60004FF00F0E8E4600F1F0020B460F4612E0C8
:101D7000984554D3BCF1000F51D174461E2601334F
:101D8000DBB216809770D4700131A94222D0062BA5
:101D900002F104021ED050F8044B2404F4D5002BA9
:101DA000E6D174467826EAE7012203EB8202B168A5
:101DB000D2F83C240192CA077BD593F86636002BF3
:101DC00014BF0F23002301A94FF400408DF8073002
:101DD000FFF722FB03B0BDE8F083474EB3F862265D
:101DE00041F228618A42DFD941F24F618A4262D9C9
:101DF00041F276618A4260D941F29D618A4261D99D
:101E000041F2C5618A426ED941F2EB618A426CD9D6
:101E100041F212718A4294BF0B220D22C5E70024C1
:101E20002646ACE7344E0DF102020C4638460DF161
:101E300003010BF0E6FAF11D38460BF0DFFA06F16C
:101E4000080138460BF0D4FA9DF803909DF8028003
:101E50004946424638460BF051FAB568F179254BB0
:101E600005F0010505EB410505EB091593F8602622
:101E7000A3F8620605EB0825ADB202BBB3F86426F1
:101E8000AA4221D0A3F864560F22206893F8665620
:101E900000F54331013AD2B201F5A07185F001009D
:101EA00083F86026216083F86606002A7FF447AF36
:101EB00093E7FF2387E7022277E7032275E7A3F87A
:101EC0006456E2E7042270E7216893F86606A3F8F7
:101ED000642601F5433202F5A07280F00101226010
:101EE00083F866167AE706225FE70A225DE700BFFD
:101EF000AC31002080640020A80300203C68002052
:101F00002DE9F041694F6A4DD7F8008084B004464E
:101F100040460E460BF028FC85F86706B8F1000F26
:101F20000AD00DF1090202A940460BF06AFA002816
:101F300040F08D8095F867060023ADF808308DF8E5
:101F40000A301A46431EDBB20021FF20FD2B8DF81C
:101F50000C20ADF80E108DF80B0003D9002004B052
:101F6000BDE8F0819DF80830042B00F09580052B2A
:101F700000F09880032B00F09780022B00F08B80FC
:101F8000012B08BF042100F087809DF809303868D4
:101F90009DF80A10013B0DF10E028DF809300BF08F
:101FA00099F995F86736032B73D0042B0CD1414A6D
:101FB0009DF80A000121002301E012F8011F81426F
:101FC0006DD20133082BF8D1D5F86826029B3A4F21
:101FD0009A420DF108084FD023680D22591C216048
:101FE0001A7023680022591C21601A7023689DF81A
:101FF0000820591C21601A7023689DF80920591C7B
:1020000021601A7023689DF80C20591C21601A70F9
:1020100023689DF80A20591C21601A70BDF80E1023
:10202000204640F03FF823689DF80B20591C2160A2
:1020300020461A700721FAF7CDF898E8030087E8E0
:1020400003000120C5F8706604B0BDE8F08101A965
:1020500040460BF0CDF900283FF46CAF40460DF13F
:102060000A010BF0CBF900283FF464AF019B95F80F
:10207000670603F0010265E77A68D8F804309A42EF
:10208000AAD1D5F870360D4AF31A93427FF666AF9F
:10209000A2E70B4A8CE703218DF8081075E78DF84D
:1020A0000A3091E70121F7E70221F5E7AC31002082
:1020B000806400204BEC0508E86A002080841E0044
:1020C00043EC05082DE9F04FC24B1B68804613F026
:1020D000800083B000F07181BF4B93F83F0310F094
:1020E000020000F06A81DFF810B39BF81430052B72
:1020F00040F26881DBF80030B84D0093002BB8BF88
:102100005B42A5FB0342B648B649920D00FB023381
:10211000C3EB03139B0085FB034502EB8202DC1734
:1021200002EB8202C4EBA55400FB043304EB8204EF
:10213000A4B281FB0321DB17C3EBA111BCB10025C5
:10214000A94F2E46A7FB0432D20802EB8203A4EB70
:102150004303E8B2A4469BB280008340BCF1090F60
:1021600094B246EA030605F10105EBD8340489B2BE
:10217000B9B100259C4F2E46A7FB0132D20802EBD5
:102180008203A1EB4303E8B28C469BB280008340FC
:10219000BCF1090F91B246EA030605F10105EBD83F
:1021A0003443DBF804E08D4D8D4E8E498EEAEE709F
:1021B000A0EBEE70A5FB0032920D06FB0200C0EB17
:1021C0000010830085FB035002EB8202DD1702EB57
:1021D0008202C5EBA05506FB053305EB8205ADB2C7
:1021E00081FB0321DB17C3EBA111C5B10020DFF890
:1021F000F8C10646ACFB0532D20802EB8203A5EB20
:102200004303C7B2A9469BB2BF00BB40B9F1090F57
:1022100095B246EA030600F10100EBD8350489B215
:10222000C1B10020DFF8C0C10646ACFB0132D208C4
:1022300002EB8203A1EB4303C7B289469BB2BF0006
:10224000BB40B9F1090F91B246EA030600F1010063
:10225000EBD83543DBF80830634A0193002B18466E
:10226000B8BF5842A2FB0030604E6149030AA6FB8A
:102270000363DB0901FB03F1C1EBD00189B2B9B102
:10228000002691463746A9FB0132D20802EB8203B1
:10229000A1EB4303F0B28C469BB280008340BCF1BB
:1022A000090F91B247EA030706F10106EBD8B9B26C
:1022B000BBF81070DFB10026DFF82CA1B446AAFBF2
:1022C0000732D20802EB8203A7EB43035FFA86F9D9
:1022D00038469BB24FEA890903FA09F3092897B2F5
:1022E0004CEA030C06F10106E9D81FFA8CF7BBF89B
:1022F00012303D4AA2FB0306F608632E28BF632670
:10230000092B63D9002093468146ABFB0632D208E5
:1023100002EB8203A6EB43035FFA80FAB4469BB25A
:102320004FEA8A0A03FA0AF3BCF1090F96B249EAA6
:10233000030900F10100E8D85FFA89F9009B019ACE
:10234000002BCCBF392338231616BEF1000F26F020
:102350007F0635DD274A3343964543F00206C8BF62
:1023600043F00606D8F800301622581CC8F80000C2
:102370001A70D8F800300022581CC8F800001A70F3
:1023800040463FF08FFE214640463FF073FE29460F
:1023900040463FF06FFE404639463FF083FED8F896
:1023A00000305A1CC8F8002083F80090D8F800309C
:1023B0005A1CC8F8002001201E7003B0BDE8F08F41
:1023C0001E43CFE7002003B0BDE8F08F4FF00009B7
:1023D000B4E700BFF03E0020806400206BCA5F6B52
:1023E000806967FFD34D6210CDCCCCCCC55A7C0A36
:1023F000A0860100FFC99A3BBC3F00202DE9F047B1
:10240000AB4B1B68064613F0800084B000F09E8042
:10241000A84B93F83F0310F0020000F09780A64FFE
:10242000397D052940F29780632900F292800024CB
:10243000DFF898C289B22546ACFB0132D20802EB24
:102440008203A1EB4303E0B28E469BB2800083403F
:10245000BEF1090F91B245EA030504F10104EBD87E
:10246000EDB2BB68954A82FB0312D917C1EB62310A
:1024700089B2002900F018814FF0000CDFF84CE21F
:102480006446AEFB0132D20802EB8203A1EB4303A8
:102490005FFA8CF088469BB280008340B8F1090F48
:1024A00091B244EA03040CF1010CEAD8E4B2FB89CE
:1024B00083494FF4F36707FB03F7A1FB0737C7F323
:1024C0008F1742F20F739F4249D8CFB10020DFF837
:1024D000FCE18446AEFB0732D20802EB8203A7EB95
:1024E0004303C1B2B8469BB289008B40B8F1090FD3
:1024F00097B24CEA030C00F10100EBD81FFA8CF7FD
:10250000704BD3E9002313433ED14FF0FF383368BB
:102510001722591C31601A7033680022581C306031
:1025200039461A7030463FF0BDFD414630463FF017
:10253000A1FD33685A1C32601D7033685A1C32602A
:1025400030461C700621F9F745FE012004B0BDE8B5
:10255000F087992585E7002004B0BDE8F0870021C9
:10256000DFF868C10F46ACFB0302D20802EB820021
:10257000A3EB40039BB28B400431102947EA0307C9
:1025800093B2F0D1BFB2BBE701A83CF04FFE9DF87B
:102590000810002900F08A804FF0000CDFF82CE1D1
:1025A000E046AEFB0132D20802EB8203A1EB43030B
:1025B0005FFA8CF089469BB280008340B9F1090F25
:1025C00091B248EA03080CF1010CEAD84FEA082856
:1025D0009DF80910E1B10020DFF8F0E08446AEFB81
:1025E0000132D20802EB8203A1EB43035FFA80F9C8
:1025F0008A469BB24FEA890903FA09F3BAF1090F37
:1026000091B24CEA030C00F10100E8D848EA0C084A
:102610009DF80A104FEA0828E1B10020DFF8ACE08D
:102620008446AEFB0132D20802EB8203A1EB4303E6
:102630005FFA80F98A469BB24FEA890903FA09F3E7
:10264000BAF1090F91B24CEA030C00F10100E8D88D
:1026500048EA0C08BDF80C301B49632BA1FB032191
:102660004FEA08184FEA51117FF651AF0020DFF80A
:102670005CE08446AEFB0132D20802EB8203A1EBA0
:1026800043035FFA80F98A469BB24FEA890903FA4D
:1026900009F3BAF1090F91B24CEA030C00F1010001
:1026A000E8D848EA0C0832E70C4600E788468FE78E
:1026B000F03E002080640020BC3F002089B5F81463
:1026C000D34D6210F86A00201F85EB51CDCCCCCCE5
:1026D00008B5A0F10103B3FA83F302284FEA5313BC
:1026E00001D0184608BD0F201BF0A6FE28B9054BE7
:1026F0001B7803F00103184608BDBDE808400F2011
:1027000019F06CB96E31002038B5802200F18004D8
:10271000002105464CF023FA0021204638224CF0D7
:102720001EFA0C49002351F8232044F823200133DA
:102730000E2BF8D108491E2205F1C0004CF0AEF96D
:1027400006490B2205F1E4004CF0A8F9032385F8B3
:10275000EF3038BD98F50508DCF50508FCF50508EF
:10276000034B0449B3F90C30406801223CF096BC9D
:10277000A8030020AF77060837B504462A4800EBC7
:102780004303B3F8525305F00F0049B1022804F196
:1027900001011DD8002814BF9C239B2323700C46E5
:1027A0000AB3C5F30315FFF72FFA3C21012D1F4B88
:1027B000B0FBF3F3B3FBF1F201FB123315D0022DA2
:1027C00023D01B49204603B0BDE830403CF066BC36
:1027D000032801BF174B1B7803F00103653B0CBFB7
:1027E000DBB22023DAE71546DDE7642542F21071FB
:1027F000B0FBF1F1B1FBF5F005FB101000900E49B4
:1028000020463CF04BFC03B030BD0A250B49B0FB21
:10281000F1F1B1FBF5F005FB1010009008492046DE
:102820003CF03CFCEFE700BF8064002040420F001A
:10283000F67706086E31002000780608A0860100B1
:102840000F780608037840680122053B114693E79C
:1028500006494068B1F86425D1F8943504495343DA
:1028600042F2107293FBF2F23CF018BC806400203C
:102870001E780608044A05495378127840680133E7
:1028800001323CF00BBC00BF043B0020237806085B
:1028900037B51C4C4568D4F8A42012F0200F02F084
:1028A000040328D094F83F23910724D5B4F9A20556
:1028B000FEF7B6FB6421002890FBF1F301FB130146
:1028C0004FF00A0091FBF0F194F85103B4BF762267
:1028D00075220029B8BF494200280CBF99209F20CB
:1028E000002BCDE90010B8BF5B42074928463CF0F9
:1028F000D5FB03B030BD002BD8D12D222A70426801
:102900005370F6E780640020297806080B4B406876
:10291000B3F948330A2293FBF2F31A0102F5B952D4
:102920004FF4B4711432B2FBF1F2C2F1080202F0BA
:102930000F02034960323CF0B1BB00BF806400204D
:102940003778060837B5194B456893F84725B3F82B
:102950006415022A04461AD093F89005B1FBF0F0F2
:10296000FEF7BDFA2870B1F57A7F606811DB0A23A3
:10297000062405310094B1FBF3F10130B1FBF3F211
:1029800003FB12130A493CF089FB03B030BD9720CA
:10299000E8E764230624B1FBF3F2009403FB12136F
:1029A000013004493CF07AFBEFE700BF806400206F
:1029B0003E780608DCEF0608034A0449D2F89C2555
:1029C000406807233CF06ABB806400204678060814
:1029D00007B5114A406892F88236B2F88016012B8A
:1029E00009D1009192F883360C497B223CF056FBCA
:1029F00003B05DF804FB0A234B4340F2FF32B3FB04
:102A0000F2F39BB2092B064928BF09237B2203B0AE
:102A10005DF804EB3CF042BB806400204C78060873
:102A20005678060813B51F49D1F8A42012F02002E9
:102A300004461AD01C4B1A7812F0010215D091F8F6
:102A40003F2312F0020210D0184BDB89632B20D9F0
:102A500064205843FEF7CEFA00281ADDD1F89435E9
:102A60004FF47A725A4392FBF0F291F85133606856
:102A7000002B02F1FF3442F20E710CBF7E237D2346
:102A80008C4208D800930A4907233CF007FB02B0A8
:102A900010BD0022E9E70749072202B0BDE8104057
:102AA0003CF0FCBA806400206E310020BC3F002066
:102AB0005C7806086578060813B50D4A446892F8F4
:102AC0008B160C4B89B19889FEF794FA92F8512332
:102AD0000949002A0CBF9D229E22034600922046EF
:102AE00070223CF0DBFA02B010BDD889ECE700BFE1
:102AF00080640020BC3F0020CA78060830B5124A26
:102B0000124B92F8A62340681C7D85B0AAB10A2119
:102B10005A8AB2FBF1F5B5FBF1F301FB13539BB2FB
:102B200002930B496423B2FBF3F21F23CDE9004269
:102B30001E223CF0B3FA05B030BD064900941F23B5
:102B40001E223CF0ABFAF6E780640020BC3F002078
:102B50006F7806087D7806080C4B40685B680C4966
:102B6000002B4FF0980210B40270BFBF2D224270AC
:102B70005B420224A8BF0124B3FBF1F2204401FB15
:102B800012335DF8044B03493CF088BABC3F002087
:102B900080969800857806080C4B40681B680C49A5
:102BA000002B4FF0890210B40270BFBF2D2242707B
:102BB0005B420224A8BF0124B3FBF1F2204401FBD5
:102BC00012335DF8044B03493CF068BABC3F002067
:102BD00080969800857806080A4B93ED000A10B598
:102BE000F2EE047A20EE270A044649F053FC0A2349
:102BF000054990FBF3F203FB12036068BDE8104047
:102C00003CF04CBA106B00208D7806080D4B1B6809
:102C10001B0137B514D50C4C4568D4F8943693F99C
:102C20000100FEF7D9FF94F851230849002A0CBF90
:102C30000D220E220346009228467A223CF02EFAFC
:102C400003B030BDF03E0020806400209878060874
:102C5000044B1B78DB0703D4034940683CF01EBAE1
:102C6000704700BF6E310020A178060807B5094AF9
:102C70000949B2F906300193B2F904300093B2F970
:102C800002304068B2F900203CF008FA03B05DF869
:102C900004FB00BFFC260020AA78060813B5094BE8
:102CA000D3F894359A24002BB8BF5B42642100947A
:102CB000B3FBF1F2406801FB123303493CF0EEF93B
:102CC00002B010BD80640020BE78060837B50A4CFB
:102CD0004568B4F99806FEF77FFF94F85123074939
:102CE000002A0CBF0D220E220346009228467A22AB
:102CF0003CF0D4F903B030BD80640020C9780608E8
:102D000037B5104A456892F89035B2F86415B1FBB2
:102D1000F3F192F84735022B044611D00846FEF72E
:102D2000DEF82870606864230624B1FBF3F2009497
:102D300003FB1213013004493CF0B0F903B030BD7D
:102D40009720EEE780640020DCEF060837B50378B3
:102D5000114A1A2B0CBFB2F94653B2F944530A2157
:102D60001A2B95FBF1F408BF152201FB145118BF73
:102D70001422002DB4BF2D2320230029B8BF4942BF
:102D8000002CB8BF644201910094044940683CF0B3
:102D900085F903B030BD00BF80640020D2780608FA
:102DA00037B51E494468D1F8A42012F0200F02F074
:102DB000040329D091F83F23920725D5D1F89C062A
:102DC000FEF72EF97F220A2390FBF3F309302270DD
:102DD000BCBF2D22627091F85113B4BF02200120B4
:102DE000002BB8BF5B4200294FF00A050CBF0F2132
:102DF0000C210091B3FBF5F2094905FB1233204485
:102E00003CF04CF903B030BD002BD7D17F222270AB
:102E100042682D21517042689370F3E7806400206E
:102E20002B780608084BD3F8A026002A0BDD074BA9
:102E300003EB8203D3F898202AB1054B05491B699F
:102E400040683CF02BB97047806400206CF50508A1
:102E5000A8030020E078060807B59378019353781B
:102E6000009313780A4603493CF018F903B05DF863
:102E700004FB00BFE8780608024B03491A68406863
:102E80001432E9E744400020F7780608024B034972
:102E90001A6840680832DFE744400020FB780608E3
:102EA000024B03491A6840680E32D5E744400020BF
:102EB000FF78060837B5044608461546FEF7B0F811
:102EC00002460DB104F8015B1A4B93F85133002B05
:102ED0000BBF4FF4A5514FF47A717E207D200CBFBB
:102EE0000F230C23914206DD1349204603B0BDE8B1
:102EF00030403CF0D3B864235A43B2FBF1F1B1F552
:102F00007A7FB1FBF3F20DDB0A230090B1FBF3F102
:102F10002046B1FBF3F503FB151308493CF0BEF85E
:102F200003B030BD009003FB1213204604493CF06F
:102F3000B5F8F5E780640020417806083E78060879
:102F4000DCEF060810B40D49446891F83F3303F0F4
:102F50000303032B06D12046B1F840135DF8044B60
:102F60001122A7E71123237043682D225A7043686A
:102F700000229A705DF8044B704700BF8064002007
:102F8000094A406892F83F3303F00303032B06D14C
:102F9000D2F8A41664237122B1FBF3F18AE7034946
:102FA0002D2371223CF07AB8806400200379060852
:102FB00038B5224D4468B5F8A0355A0505D52046E8
:102FC0001F49BDE838404BF0EEBD180505D5204639
:102FD0001C49BDE838404BF0E6BD590605D52046F2
:102FE0001949BDE838404BF0DEBDDA0705D520466B
:102FF0001649BDE838404BF0D6BD9B0705D52046A5
:103000001349BDE838404BF0CEBD252018F0E6FC52
:1030100028B120460F49BDE838404BF0C4BD95F8B3
:10302000A8362BB120460C49BDE838404BF0BBBD5B
:1030300020460A49BDE838404BF0B5BD8064002009
:10304000087906080D790608127906081779060826
:103050001C79060821790608267906082B790608C6
:10306000074B93ED1A7AD3ED1B7AB4EEE77AF1EEC3
:1030700010FA03DD034940684BF095BD704700BF6F
:10308000C40B0010997F060810B50C46A0B9184A69
:10309000184892F8A91623680344236001B110BDB3
:1030A00092F8A33414492033BDE8104001EB8301AA
:1030B0004FF48060FEF7B0B912F020FB32280ADD31
:1030C00023680B4A03F5742303F510730121236071
:1030D00082F8A91610BD064A92F8A916142881F0A4
:1030E0000101CCBF0548064882F8A916D3E700BF06
:1030F0008064002040420F003C68002020A10700AF
:1031000048E8010010B5044620F058FE0349034684
:1031100004226068BDE810403BF0C0BFAF770608EE
:10312000F0B52B4B2B4E1C68317887B007462046F4
:103130000AF04CF97178054620460AF033F900226E
:103140000592B2788DF8132003466CB1039005A95F
:1031500020460AF04DF9327A039B2AB10DF1130192
:1031600020460AF04BF9039B9DF81310ECB1E1B136
:10317000194A1268914218DC184A02EB8102D2F80F
:10318000AC460393262018F029FC0599039B70B9DF
:1031900011F0010F14BF502200228907786808D56A
:1031A0000F493BF07BFF07B0F0BD0E4CE9E744222E
:1031B000F3E732B1CDE900420B492A463BF06EFFFE
:1031C000F1E70A4900942A463BF068FFEBE700BFAD
:1031D000AC31002064310020B8220020806400203F
:1031E000307906084C8106083879060844790608C3
:1031F000F8B50446274B4178827893F86D0323781D
:103200000138302B244B4FEA8000034423480BBF86
:1032100093F8205193F8225193F8216193F8236198
:1032200030F9153030F9160040F2CF75AB42A8BF27
:103230002B46B3F57A7FB8BF4FF47A73A8424FF4A8
:103240007A77A8BF2846A3F57A73B842C3EB031375
:10325000B3FBF7F3C3F10E03B8BF3846DBB24FF050
:10326000030CB3FBFCFC0CEB4C0EA3EB0E03A0F524
:103270007A706244C0EBC0000833B0FBF7F7394402
:10328000DBB2D2B2C9B22046F9F742FD0023237364
:10329000F8BD00BF806400206CF505085C4000208C
:1032A0002DE9F04790F8029090F8018009F10207AB
:1032B00004460026FFB2002508EB060A032E18D1AB
:1032C000022D08F1030118BF09EB0502C9B207BFBF
:1032D0000B233A461623D2B22046F9F719FD0135E1
:1032E000052DEBD10136072EE5D100232373BDE870
:1032F000F087022DF3D117233A465FFA8AF1204670
:10330000F9F706FDEBE770B504466FF00205A27809
:10331000617852FA85F207391323D2B2C9B2204636
:10332000F9F7F6FCA2786178EEB232440731132344
:10333000D2B2C9B220460135F9F7EAFC042DE6D134
:103340006178A27806390323C9B22046F9F7E0FC78
:103350006178A27806310223C9B22046F9F7D8FC79
:103360000023237370BD2DE9F8432B4A054692F8DC
:103370005D1392F86B03B2F9444392F85C33002872
:1033800001EB810114BF4FF0FF300120490044439D
:10339000C1F1000803EB830344454FEA430303DB19
:1033A0008C42A8BF0C46A046B2F946235C42424379
:1033B000A24203DB9A42A8BF1A4614461BB1192247
:1033C000544394FBF3F4293C4FEA88066FF003075B
:1033D0004FF00909002E3346B8BF06F13F03C4EB96
:1033E000A313512B0FD893FBF9F101EBC1029B1AE8
:1033F000AA780A446978803B3944DBB2D2B2C9B2B8
:103400002846F9F785FC0137052FA6EB0806E1D120
:1034100000232B73BDE8F8838064002010B50446B8
:1034200012F0A8F9642202FB00F3C3F38F23632B8D
:1034300060680449BDE8104028BF632301223BF0C7
:103440002DBE00BF7F7806081E4A9FED1F7AD2F876
:103450009C15B2F84C33406807EE901AF8EEE76A14
:1034600007EE903AF8EEE77A67EE877AF4EEE76ACD
:10347000F1EE10FA02D815493BF010BE8B4202DA89
:1034800013493BF00BBE5B1A07EE903A02F22C6335
:10349000B8EEE77AD3ED007A0E4AF8EE677A3C216F
:1034A00067EE277A87EEA67AFDEEC77A17EE903A96
:1034B000B3FBF2F3B3FBF1F201FB123306493BF02D
:1034C000EDBD00BF80640020CDCCCC3D4D79060819
:1034D0005379060840420F00F6770608244A002375
:1034E0004361D2F8601341F45C5130B541F02C01D6
:1034F0000124C2F860134471D2F8581304FA03F59A
:103500000133112B41EA0501F8D14FF4206321F476
:10351000F031C2F85813C38040F601230381154BE4
:103520000360142303718023037642F6140303829D
:103530004FF6FF73438303F58C03C36140F201230D
:10354000038400230C4A80F8223080F8333080F85E
:1035500044305023A0F856306FF07E43C0E9162364
:103560004FF0A063036640F61833A0F8643030BD16
:103570008064002098086400C4FF00FFF8B5194D6E
:103580000646002418F05EFE882705F1740C2B789F
:103590007168A342214402DC00230B70F8BDF8B12E
:1035A000D5ED1C7AFDEEE77A0CEB840317EE90EA7A
:1035B000D3ED007AFDEEE77A17EE902AD5ED257A65
:1035C000FDEEE77AA2EB0E0217EE903AD200A3EBE3
:1035D0000E0392FBF3F3C3F188030B700134D6E7BB
:1035E0000F70FBE7C40B00101F4AB2F87C32D2F810
:1035F0009C2513B50446D3B19A1A9A42A8BF1A461D
:1036000022EAE27207EE902A0B22B3FBF2F300EEFD
:10361000103AF8EEE77AB8EEC00A87EE800A48F072
:10362000F3FEFCEEC07ACDED017A9DF804306268BD
:103630008A211170012261689342ACBF8B208D20DA
:10364000885401320C2AF6D162688F2111735A1EF8
:10365000092A9FBF62689B188E225A7063680022F5
:103660005A7302B010BD00BF8064002010B504463C
:10367000132018F0B3F908B30BF088FE30B9606876
:103680000F49BDE8104010223BF008BD0D4B6068AB
:1036900093F8D226012A0BD1D3F8D826D3F8DC36FA
:1036A0009A4205D3BDE81040074910223BF0F6BC12
:1036B000BDE81040054910223BF0F0BC10BD00BF32
:1036C00059790608806400205D79060889F80608A3
:1036D00070B52D4D0A24B5F9442392FBF4F484EA25
:1036E000E473A3EBE4739BB25A2B064605D90A3266
:1036F000CCBFB4236FF0B3031C1B95F8503533B91E
:10370000224B1B78DB0729D418F0FEFD30BB95F85F
:10371000E436B32B02D818F0F7FDF8B9B5F9461323
:103720000A2391FBF3F304B9C3B1002BB8BF5B428A
:1037300084EAE4709BB2A0EBE470B3EB400F7268D4
:1037400013DAB0EB430F10DA092908DD002CCCBFE7
:103750006E2362231370736800225A7070BD002CB0
:10376000CCBF6A2366231370F5E7834205DD092980
:10377000CCBF602368231370EDE7002CCCBF6C2313
:1037800064231370E7E700BF806400206E310020DF
:1037900030B585B0054601A83BF048FD044618B990
:1037A0002870204605B030BD044A0123B2F9E8264E
:1037B00001A928463BF08EFDF3E700BF806400209E
:1037C0004068E5E773B50D4D0091044616460023A9
:1037D00002460221286836F0C7FC094B00932246B6
:1037E00028680023142136F0BFFC286800960023C7
:1037F0002246162136F0B8FC02B070BDEC3A00202B
:10380000C9AD06082DE9F04F04468BB0E8B1A94BCD
:103810001868037A9C422246A8BF1A469C42B8BF49
:103820000132A3EB020303EBD373B4BF01210021E8
:10383000C3F3470449B1A04B009322460023022161
:10384000651C36F091FCEDB22C46DFF8B8829B4F38
:10385000DFF8B4920026454617F8013BD8F860130C
:1038600001229A400A4230D0172B2ED8DFE813F0FD
:10387000180034004D0077009000B300C700DB0053
:10388000EF00FE0010015B004E012D008801A50134
:10389000BA01C501A000D501FA0105021802EE0126
:1038A0000DF1080A5046FFF773FF18B984495046D6
:1038B0003BF0F4FB7F48CDF800A0006800232246CF
:1038C000022136F051FC0134E4B20136182EC3D186
:1038D00020460BB0BDE8F08FB5F85223002312F05C
:1038E0000F02194618BF012202A8FEF745FFB5F8DE
:1038F000523303F00F02734B03EB82032046D3F8DD
:10390000481102AAFFF75EFFDDE7B5F85423012353
:1039100012F00F0218BF1A46002102A8FEF72CFF72
:10392000B5F85433E5E7D5F84006FDF779FB95F88F
:10393000511300290CBF0F210C210A23009190FB89
:10394000F3F0614990FBF3F203FB120302A83BF092
:10395000A5FB5E4902AA2046FFF734FFB3E75C4BA4
:103960001B681B06B1D5B5F93406FDF743FB95F886
:1039700051335849002B02460CBF9D239E2302A8B9
:103980003BF08CFB544902AA2046FFF71BFF9AE745
:103990004F4B1B68180698D5B5F9441602A80022AB
:1039A000FFF788FA4D4902AA2046FFF70BFF8AE786
:1039B000474B1B68190688D5D5F8A416642302A8BE
:1039C000B1FBF3F10022FFF775FA454902AA204640
:1039D000FFF7F8FE77E7B5F93616642391FBF3F2AB
:1039E00003FB1213062100911BB23E4902A83BF0D3
:1039F00055FB3D4902AA2046FFF7E4FE63E7B5F810
:103A000038166423B1FBF3F203FB12130621009175
:103A10009BB2344902A83BF041FB344902AA20463C
:103A2000FFF7D0FE4FE7B5F864156423B1FBF3F25E
:103A300003FB1213062100919BB22A4902A83BF016
:103A40002DFB2B4902AA2046FFF7BCFE3BE702A94B
:103A500095F83C06F8F740FC264902A84BF087F899
:103A6000254902AA2046FFF7ADFE2CE795F87A32E9
:103A7000002B3FF42AAFB5F93A2616499A2302A83B
:103A80003BF00CFB1D4902AA2046FFF79BFE1AE7FC
:103A900095F87A32002B3FF418AFD5F89C250D49E4
:103AA000072302A83BF0FAFA154902AA2046FFF7BD
:103AB00089FE08E7EC3A0020617906089CF60508C3
:103AC000717906086CF505083E78060878790608CD
:103AD000F03E002041780608857906088F790608AF
:103AE0009C790608DCEF0608AC790608B879060868
:103AF000BC790608E5790608C4790608CD79060878
:103B0000D979060880640020717A060895F8D236C3
:103B1000002B3FF4DAAE032B3FF4D7AE0BF036FCAC
:103B200095F8D236012B23D128B3F6F75DFF8246F4
:103B300042F0D0FB834642F00FFA6423800A03FB75
:103B400000F2BAF80210BAF80430591ADBF804305F
:103B500001FB03339B0A6249B2FBF3F202A892B263
:103B60003BF09CFA5F4902AA2046FFF72BFEAAE62B
:103B7000002840F0B3805C4902A83BF08FFAF1E7DF
:103B8000D5F8A4309A077FF5A0AE584B93ED060AFE
:103B9000F2EE047A20EE270A48F07CFC0A2354490E
:103BA00090FBF3F203FB120302A83BF077FA5149B2
:103BB00002AA2046FFF706FE85E6B5F94C06FEF799
:103BC0000BF895F851334C49002B02460CBF0D23DE
:103BD0000E2302A83BF062FA484902AA2046FFF7EA
:103BE000F1FD70E602A9D5F85006F8F775FB4449D7
:103BF00002AA2046FFF7E6FD65E6B5F854264149DE
:103C000002A83BF04BFA404902A84AF0B0FF3F49F6
:103C100002AA2046FFF7D6FD55E63D4B1B689B00E8
:103C20007FF553AE3B4BB3F898204AB13A4902A80E
:103C30003BF034FA394902AA2046FFF7C3FD42E6B9
:103C4000374A36492046FFF7BDFD3CE6B5F9562612
:103C5000344902A83BF022FA334902AA2046FFF772
:103C6000B1FD30E602A9D5F8EC06F8F735FB2F498F
:103C700002AA2046FFF7A6FD25E63C21D5F8F0363E
:103C8000B3FBF1F302A8B3FBF1F201FB12332849B5
:103C90003BF004FA274902AA2046FFF793FD12E6FB
:103CA00095F85133D5F8F42673B940F249617E2373
:103CB000B2FBF1F202A810493BF0F0F902AA494622
:103CC0002046FFF77FFDFEE54FF47A717D23B2FBBE
:103CD000F1F202A808493BF0E1F9EFE7FFDE00BF8F
:103CE000E2790608ED790608E7790608B06A00204F
:103CF0008D780608F679060841780608027A0608E3
:103D00000F7A0608B9F00608E57906081B7A060856
:103D1000F03E0020C40B0010247A0608297A060819
:103D2000327A0608E47806083B7A0608487A0608DC
:103D3000567A06085F7A060838B5044602214FF421
:103D4000FA7032220123E17040F203150021E08075
:103D5000A5802281A3722170102032F08BFB60704D
:103D600038BD00BF08B507F081F9054B1B689B0300
:103D700000D408BD33F050FABDE808400AF02EBA6E
:103D8000F03E0020104B186810B5D8B10F4C2178C8
:103D900041B1627809F0B2FAA38883421ABFA080C9
:103DA00001210021E2885AB141F288339342B8BF21
:103DB00013469A4204D0E380BDE8104039F004BCB9
:103DC0000029F9D110BD00BFAC31002064310020C2
:103DD00010B401440446002014F8013B0822584066
:103DE000430010F0800F08BF400083F0070314BFAA
:103DF000D8B2C0B2013AF3D18C42EDD15DF8044B98
:103E0000704700BF30B54FF4806085B02CF0A0F84B
:103E100040B3154C90F9040094F8FC36134A002B7B
:103E200018BF08234FF4E1310125CDE9015300917A
:103E300000234FF480612CF0E8F8FF236060003825
:103E400018BF012084F8203084F8303084F84030E6
:103E500084F8503084F8603084F8703084F8803012
:103E600084F8903005B030BD80640020F50C010866
:103E7000364B1B6813F000635FD02DE9F04F344BD5
:103E80001F78B84254D3FF2859D1324B1B78002BEE
:103E90004BD0DFF8D4A00022CAF80027CAF80427C4
:103EA000CAF80827AAF80C27002F4BD00AF12003E4
:103EB0001046144611461546164603EB071BB94635
:103EC000B3F802C09F8993F8008093F901E0614440
:103ED0003A444645D3E901C738BF464610337545D5
:103EE000B8BF75469B4509B212B264443844E7D165
:103EF00091FBF9F192FBF9F28AF800678AF8015711
:103F0000CAF80447CAF80807134BAAF802171B7827
:103F10001049AAF80C27092B4FF0000208BF0F4BDD
:103F20000A7004BF9AF80027DA800D48BDE8F08FC8
:103F30000C4A02EB0010BDE8F08F184670470020D5
:103F4000BDE8F08F3A463946DEE700BFF03E00207C
:103F5000C40B0010A8030020F9260020FC26002036
:103F6000806B0020A0640020806400200268F8B507
:103F70003A4E3B4CB6F99836511C01607E211170C7
:103F80000168054603EBC30384FB0302481CDC17EE
:103F9000002328600B70FF20C4EB6204FFF768FF6A
:103FA0002034304BA4B200284DD01B78B0F90C104F
:103FB0002BBB2D4BA1F57A729A4246D82B48B0FB09
:103FC000F1F189B228463EF047F896F87735B6F811
:103FD000641583B196F89035B1FBF3F128463EF0B5
:103FE0003BF8214628463EF037F828460821F8F7E6
:103FF000F1F80120F8BD28463EF02EF8F1E71C4B01
:104000001F78002FD5D01B48002300EB830201331B
:104010009289BB421144F8DB174B9FED186A9B7ED7
:1040200007EE103A07EE901AB8EEC77AF8EE676A14
:10403000C6EE077A67EEA67AFCEEE77A17EE901ADC
:10404000B1FBF7F1B5E71B7813B94EF69C21B9E740
:10405000074B1F78002FF8D00146D4E7806400207A
:1040600067666666600900101783930300879303F1
:10407000C40B0010600C0010142F002000004843F7
:104080002DE9F04FAF4C89B094F84785054633F0E1
:10409000C3F8D4F81037D4F8586323F40013C4F8E5
:1040A0001037F307074649D5002017F097FC002882
:1040B00041D0D4F84C25002A3DD0900104D5B2F16E
:1040C000007F18BF02F17E42D4F818179FED9E7A48
:1040D0007B1A07EE903AF8EE677AF4EEC77AF1EEC3
:1040E00010FA05DCD4F81C0701238340134212D1D7
:1040F00011B91923C4F81C37D4F81C37C4F8187741
:10410000012001331A2B28BF002300FA03F11142CA
:10411000F7D0C4F81C37D4F81C278C4B8C4968683E
:1041200003EB8203D3F858213AF0B8FF02236B73F4
:1041300009B0BDE8F08F0023C4F81837D4F8203751
:104140007BB3844B1B78D9072BD4D4F824379FED4D
:10415000827A686803F5921303F57863DB1B07EE38
:10416000903AF8EE677A67EE877AFDEEE77AB8EE76
:10417000E77A17EE903AF1EE0C7AB4EEE77AF1EEC8
:1041800010FA05DB75493AF089FF01236B73CFE71D
:104190000A21B3FBF1F201FB123371493AF07EFFC1
:1041A000F3E7B2050FD56F4BDB7863B16E496868F2
:1041B0003AF074FF03236B73D4F8103743F4001301
:1041C000C4F81037B4E7B30609D594F8503533B1C5
:1041D000664968683AF062FF01236B73A8E77705C8
:1041E00036D594F82837012B32D1D4F8A43068683A
:1041F0009E0729D5B4F93A37B4F94623D21A6FF499
:1042000063739A421BDB40F28D339A421ADC0A2315
:1042100092FBF3F256493AF041FF1FF0CFFD554BA8
:104220001B6893F865300A3B23EAE3739842ACDBE2
:10423000D4F8103743F40013C4F81037A5E76FF033
:104240005902E7E75A22E5E74B493AF027FFE4E74E
:10425000B00412D511F052FA94F8503383420CD9BD
:10426000464968683AF01AFF02236B73D4F8103796
:1042700043F40013C4F810375AE7310408D5404B13
:10428000B4F9A423B3F90C309A4201DD3D49E8E7C3
:10429000720407D511F01AFAB4F8A233834201D997
:1042A0003949DEE7330704D5B8F1020F01D13749A8
:1042B0007DE737050FD5274B1B78D8070BD51AF0AC
:1042C000E1F840B194F83F33D90704D594F8753735
:1042D0000BB92F49C5E7F20414D51E4B1B78DB0739
:1042E00010D51AF0CFF868B194F83F33DF0709D43E
:1042F000D4F83036A3F53713A3F5D863002B01DAD1
:104300002449AEE7B4F8A035580601D52249A8E7FC
:10431000310645D5B4F9980694F86A3398423FDBE4
:10432000FDF75AFC94F851236E681C49002A0CBF13
:104330000D220E220346009230467A223AF0AEFE5B
:1043400092E700BF806400200024F4486CF5050863
:1043500087A406086E310020ACC52737807A06088E
:104360008B7A060870310020987A0608A27A06082F
:10437000AD7A060844400020B77A0608BE7A0608DF
:10438000A80300203F7A0608C77A0608D47A0608F0
:10439000DE7A0608E97A0608F47A0608FD7A060845
:1043A000604B1B681A016DD573066BD55E4B93F895
:1043B000009004AAC9F1090676080023934620213B
:1043C0009E421AD10BEB060058494FF0000A4AF002
:1043D000EAFB03365246914501D90B2E11D908ABA1
:1043E0001E44002306F8103CBAF1000F4AD0504991
:1043F00068685A463AF052FE36E702F8011B01336C
:10440000DEE7D7B238460392FFF732FD494B039AF5
:1044100093F800C031371CF0010CFFB230D0B4F972
:1044200066E3BEF1FF3F2BD08189642311FB03F1CA
:10443000414B9B7E5B0891FBF3F39E45B4BF3B462B
:10444000522394F9641311F1800F04D090F901E024
:104450008E45A8BF5423BCF1000F08D0B4F96813EF
:10446000B1F1FF3F03D040688842A8BF43239F4279
:104470000BF8063018BF0AF1010A01320136AAE72B
:104480003B46DEE7D4F858335A0704D5B8F1010F9C
:1044900001D12A49E5E6DF050DD5264A1278D6076F
:1044A00009D5274A92F82520012A04D1254A1278F5
:1044B0000AB92549D5E6D8030CD51E4A1278D1078A
:1044C00008D5B4F84C232AB1D4F89C158A4201DCF3
:1044D0001E49C6E69A0718D5164A94F84715127869
:1044E00002F003020A4310D1B4F88212B4F8642532
:1044F00094F89005B2FBF0F2914206D9144968682D
:104500003AF0CCFD01236B7312E6DB067FF510AEAB
:1045100094F87837002B3FF40BAE0E4968683AF0F8
:10452000BDFD32E6F03E0020C40B00100E790608F7
:1045300087A406086E310020142F00200C7B06088B
:10454000E43B0020740A0010187B0608247B060850
:104550002D7B0608397B060810B5184CA379CBB122
:10456000A37EDFED176A07EE903AF8EEE77A154B77
:1045700086EEA77AC0B203EB8000B0F8A83007EE51
:10458000903AF8EEE77A67EE277AFDEEE77A17EED3
:10459000900A10BD0C4B1B6813F000630BD0C0B227
:1045A000FFF766FC8089642310FB03F0A37E5B08A1
:1045B00090FBF3F0EDE71846EBE700BF142F002067
:1045C00000004843C40B0010F03E002008B5FFF780
:1045D000C3FF3C2390FBF3F008BD00BF2DE9F84377
:1045E0004A4C427894F8793702F00F05C3B9EDB917
:1045F0002B46002184F87C17EB1AD9B20E290BD870
:10460000234493F8781539B102F0F002802A4AD099
:10461000902A5FD0A02A0DD000273846BDE8F88345
:104620000021AB4284F87C17F6D8E5E784F8795787
:104630002B46DEE7412966D081F08003042B62D946
:104640000846FCF76BFB031D0246DBB2304884F8DA
:104650007C3765F05F0584F87D57FDF727F894F8FF
:104660007C77002FD8D0BE1E16F0FF0024D1FF2586
:10467000A946022756B1DFF89C80464418F8011B72
:10468000D4F8A00733F086FB4645F7D1D4F8A0074D
:10469000494633F07FFBD4F8A007294633F07AFB74
:1046A0003846BDE8F88365F07F050427022684F8C4
:1046B0007D5784F87C773046164A4FF6FF711044D8
:1046C00012F8015B491B904289B2F9D15FFA81F976
:1046D0000D0ACFE7412914D081F08003042B10D9B3
:1046E0000846FCF71BFB65F06F050627042684F8D7
:1046F0007F0784F87D5784F87E1784F87C773046EE
:10470000DAE70420EFE7082304229FE78064002013
:10471000FE6B0020FC6B00202DE9F047C31DDFF885
:10472000348182B003F4FC7300AFD8F8BC60ADEB09
:10473000030DC7F800D03268D8F8B43068449A4204
:104740000C4698F8A43778606D4658D0591C0DF186
:10475000010203F00F0388F8A4178DF800303A60C7
:10476000A0EB0209D6E900125FFA89F9521A09F1A1
:1047700007035FFA82FA03F4FC73CA45ADEB030D3D
:1047800055D2524668464AF089F93368534433603B
:104790005246694638463DF03DFCD8F8BC20D8F872
:1047A000B4303068117A7060C21A4A40D2B2834283
:1047B000336088F8A52709D00133336013F8011C52
:1047C000984282EA0102F7D188F8A5273B68591C74
:1047D00039601A70D7E90032D21A012A08DD0021A7
:1047E0005A1C3A601970D7E90032D21A012AF7DC54
:1047F0002846A04700200837BD46BDE8F087B6F937
:104800000C20591C03F00F0343F01003002A2A4622
:10481000B8BF43F0200302F8023B88F8A417691CD4
:104820003960D6E900135B1A3A606B7098E74A4624
:1048300068464AF033F933684B4433604A46694668
:1048400038463DF0E7FB2846A04701200837BD4623
:10485000BDE8F087806400202DE9F04F7A4C83B0EA
:10486000D4F8BC50D5E900535B1B002B00AF834646
:104870000D46164628DD002384F8A637FCF7C4FA57
:1048800000200BEB05030BF1010AC4E92AA39BF8F6
:104890000050D4F8B8806909012940F09D8005F0E6
:1048A0000F0915F0100514D150B194F8A827013262
:1048B00002F00F024A4500F0988084F8A657284677
:1048C0000C37BD46BDE8F08F94F8A6070028D8D174
:1048D000D4E70BF10203C4F8A8300BF103029BF8F4
:1048E0000130D4F8B000C4F8A8209BF80250C8F8F2
:1048F0000000C218C8F804206B4084F8A737D4E938
:104900002AA34FF0000C84F8A617A8F80850A8F8BE
:104910000CC0A3EB0A03DDB2121AEB1D5FFA82FB97
:1049200003F4FC73AB45ADEB030D6BD25A46514615
:1049300068464AF0B3F80AEB0B035A46404669460C
:10494000C4F8A8303DF066FBD4F8B030D8F80000C9
:1049500094F8A7278342C8E900300AD00133C8F889
:10496000003013F8011C984282EA0102F6D184F863
:10497000A727D4F8A8301B78934239D1B8F908306A
:10498000FA2B54D0D8F80020D4F8B030D4F8B810AE
:10499000D4F86402C8E90032D4F8BC20D4F8B430AA
:1049A00053600025158195813B1D84F8A6577D60D5
:1049B0002BF0F4FE01303FD07B680BB1002098470C
:1049C000D4F8BC30D4F8B420196801200C37C3E9FE
:1049D0000021BD46BDE8F08F00210846FCF7F8F93C
:1049E00001200C37BD46BDE8F08FD8E9000290E702
:1049F00000230120B8F9081084F8A637FCF7E8F97D
:104A000001205DE72A46514668464AF047F80AEB1E
:104A1000050340462A466946C4F8A8303DF0FAFA34
:104A200000200C3784F8A897BD46BDE8F08F002E13
:104A3000A8D005233370A5E7D4F8BC201368022161
:104A4000581C10601970B7E7806400200B4B93F876
:104A50007A2212B1B3F888254AB9B3F94833084A23
:104A6000D81782FB0323C0EBA30000B27047D3F832
:104A70009C0590FBF2F000B2704700BF80640020FC
:104A800067666666F8B5184CC6B205463146D4F876
:104A9000AC0733F07FF994F8B017D4F8AC07C5F33E
:104AA00007274E40394684F8B06733F073F994F81D
:104AB000B017D4F8AC07C5F307464F40314684F829
:104AC000B07733F067F994F8B017D4F8AC072D0E2F
:104AD0004E40294684F8B06733F05CF994F8B0177B
:104AE0004D4084F8B057F8BD8064002070B50C4D7F
:104AF000C6B231460446D5F8AC0733F04BF995F809
:104B0000B017D5F8AC07240A4E40214685F8B067A7
:104B100033F040F995F8B0174C4085F8B04770BDB8
:104B20008064002038B50B4C002305462421D4F8BE
:104B3000AC0784F8B03733F02DF9D4F8AC07542122
:104B400033F028F9D4F8AC072946BDE8384033F0F3
:104B500021B900BF806400202DE9F043DFF85093B5
:104B60002DED028B99F8B14783B00E461546002C07
:104B700000F0DF81013C89F8B147C64F9FEDC68A3E
:104B8000DFF830833378002B00F08C8099F8B14740
:104B9000002C40F0878035B132F03EFB2B68C01A04
:104BA000002880F2D58399F8B247002C40F07A8330
:104BB00099F8B307062840F27F81B8494B7E0A7EF8
:104BC0009A4200F0A78151F8144F99F8B42734F8AD
:104BD0001340144401300133A4B2C0B2DBB2B4F5C7
:104BE000C06F89F8B3074B7100F07C817CD8B4F5B5
:104BF000806F00F0268224D8B4F5067F4FD8B4F534
:104C0000007F54D3A4F50073182B48D8DFE813F0C5
:104C1000E401DB01DB01DB01DB01DB01DB01DB01AB
:104C2000DB014700470047004700470047004700B7
:104C3000C301A801A801A801A801A801A801A80111
:104C4000A801B4F5846F00F0E38140F2E280B4F58E
:104C5000A06F00F065826FF4A06C04EB0C03072BCF
:104C60001DD8601EC0B2FFF703F9C0B1B0F90C3017
:104C70008B4AADF80140917ED9F8682203EB83039B
:104C800003EB830349089B0093FBF1F31021CDF85C
:104C900003308DF800106846904700233370002DD4
:104CA0007FF470AF03B0BDEC028BBDE8F083B4F5C8
:104CB000807F00F0FE81B4F5887FF0D1B9F9A2358C
:104CC000CDF80330012210238DF800308DF801302B
:104CD0008DF80220D9F8683268460024984734706D
:104CE000002D7FF44FAFDDE7B4F5046F00F0A8822C
:104CF00065D8B4F5006F00F085821AD9B4F5026F5B
:104D000000F0F281B4F5036FC9D199F83F339807E9
:104D1000C5D5644BD9F86822D9894FF4F36303FBF6
:104D200001F3A7FB03135B091020CDF803303021FA
:104D300091E2B4F5E26F00F03882B4F5E46F1FD170
:104D4000594B93ED180AD3ED027A20EE270A00247E
:104D500020EE080A47F09EFB102320228DF8003039
:104D60000723CDF803008DF802308DF80120D9F823
:104D70006832684698473470002D7FF403AF91E79E
:104D8000B4F5E06F8BD1484B93ED160AD3ED027A60
:104D900020EE270A002420EE080A47F07BFB1022B1
:104DA0000723CDF803008DF802308DF80020D9F8E4
:104DB00068328DF80140684698473470DCE740F669
:104DC00078339C4248D8B4F5376F00F2E381B4F5EC
:104DD000116F00F08181B4F5376F7FF460AFFF2071
:104DE000FFF746F800283FF45AAF90F90130CDF8AC
:104DF0000330102170220B238DF802308DF8001043
:104E0000D9F868328DF8012068460024984734703C
:104E100066E740F201439C4200F02C82B4F5826FB9
:104E20007FF43DAFD9F8A430980600F14A821F4BB9
:104E30001B681C0640F1A1820024102304228DF877
:104E400000308DF801308DF803408DF804408DF866
:104E500005408DF80640BCE145F230239C4200F04D
:104E6000858145F240239C427FF419AFB9F9443360
:104E7000CDF803301021402252238DF802308DF8F6
:104E80000010D9F868328DF8012068460024984750
:104E9000347025E71F85EB510000C842A8030020AD
:104EA000142F0020BC3F0020C40B0010F03E002057
:104EB00080640020C5B3A2910130CB49C0B291F803
:104EC000212091F8203093421FD0531CDBB25200B6
:104ED000CC69C649A45A89F8B307B4F5C06F4B71C1
:104EE0007FF484AED9F89C35CDF80330102200242D
:104EF00006238DF802308DF80020D9F868328DF83D
:104F0000014068469847347036E7002281F8212036
:104F10000123DDE7B64A99F8B43712784C760133AD
:104F2000DBB20132934289F8B43700F0B781012037
:104F3000C5E700283FF421AE0378303B012B3FF654
:104F40001CAE013009F2B1720621FFF785FC99F819
:104F5000B13789F8B207002B3FF40FAE34700CE67E
:104F6000A4F11100C0B2FEF783FF00283FF497AE12
:104F7000B0F90230CDF8033010238DF80030ADF8D1
:104F80000140D9F868326846984700233370002DF5
:104F90007FF4F8AD86E699F87725B9F86435002AEC
:104FA00040F0D08110220221CDF803308DF800208E
:104FB000D9F868328DF801208DF802106846002477
:104FC000984734708CE6601EC0B2FEF751FF00288F
:104FD0003FF465AE4368CDE7D9F894358549D9F8F3
:104FE000682281FB0301DB17C3EBA103002410211E
:104FF000CDF8033002238DF800108DF801408DF8B4
:105000000230684690473470002D7FF4BBAD49E60E
:1050100099F83F339A077FF542AEB9F84033CDF89F
:1050200003301021202204238DF802308DF8001067
:10503000D9F868328DF8012068460024984734700A
:105040004EE699F8B5370133DAB2042A1EBF42F2B0
:10505000107389F8B5275343D9F84C2502BF0123B3
:1050600089F8B53742F21073002A00F02881023324
:10507000614A1278D007B9F8A02548BF0433D10798
:1050800048BF0A33940748BF1433D00548BF2833BC
:10509000510748BF6433540648BF03F57A631021B3
:1050A00000240422CDF803308DF800108DF8014063
:1050B0008FE0D9F89C36CDF803301022002401236C
:1050C0008DF802308DF80020D9F868328DF8014053
:1050D0006846984734704FE699F89035002B40F0B9
:1050E0002C81102209215FE799F83F339B077FF558
:1050F000D6AD424AD9F868329268CDF80320102222
:1051000020218DF8002008228DF801108DF8022052
:105110006846002498473470002D7FF433ADC1E514
:10512000FF20FEF7A5FE00283FF4B9ADB0F90C3022
:105130003349D9F86822897E03EB830303EB8303A9
:105140001020490800249B0093FBF1F305218DF802
:105150000000CDF803308DF801408DF8021068464C
:1051600090473470002D7FF40DAD9BE5B9F94633BF
:10517000CDF803301021302252238DF802308DF803
:105180000010D9F868328DF801206846002498474D
:105190003470A5E5A4F17100C0B2FEF769FE0028E5
:1051A0003FF47DAD90F90130E4E6114B93ED170A21
:1051B000D3ED027A20EE270A002420EE080A47F0F9
:1051C00069F91023CDF8030007228DF800308DF81F
:1051D0000130D9F868328DF802206846984734705B
:1051E000002D7FF4CFAC5DE5A8030020C4030020B0
:1051F000C40B0010676666666E310020BC3F00205D
:10520000142F002099F83F2391077FF548AD13F044
:10521000010F7E4B00F0A2805A6882EAE273A3EB92
:10522000E27303EB5303A7FB0313DB08002AACBFB5
:1052300043F0004343F0404310210024082231E7AB
:10524000B9F94833D9F8682203EB83035B001020D7
:10525000CDF80330402108238DF800008DF80110AF
:105260008DF802306846002490473470002D7FF49A
:1052700089AC17E5B9F99836CDF803301021012231
:1052800004238DF802308DF80010D9F868328DF8BB
:105290000120684600249847347021E589F8B44716
:1052A00001200CE65A490620FFF736FA002389F858
:1052B000B207337003B0BDEC028BBDE8F08301335D
:1052C000D6E6524A99F83F13538A643BC3EB4370C6
:1052D000C3EBC00388FB03401844DB17C3EB202358
:1052E0000933092BA8BF092323EAE37303EB8303E4
:1052F00011F0020F03EB830314BF4FF47A70002008
:105300009B00C90748BF00F5FA60117DD9F86822F3
:105310009BB203440B44042010218DF80200CDF809
:1053200003308DF800108DF8011068460024904776
:105330003470002D7FF426ACB4E4B9F86425B2FBD8
:10534000F3F3CEE699F89025002A57D1134629E6C3
:10535000347003B0BDEC028BBDE8F0831A6882EABA
:10536000E273A3EBE27303EB5303A7FB0313DB0826
:10537000002AB8BF43F080435EE799F87635002BEA
:105380003FF48DAC99F8B637032B3AD8DFE803F039
:105390002C221302D9F8B827537A907AD17A03F1E4
:1053A000407303EB0023002203EB014389F8B62787
:1053B00010220421F8E5174A11688A7D087C897A51
:1053C000120402EB00220A44591C89F8B61702EBBA
:1053D0000363EDE70F4A11684A7DC87B497A1204DE
:1053E00002EB00220A44EFE70A4A11680A7D887B33
:1053F000097A120402EB00220A44E5E7B3FBF2F358
:10540000D0E55A1C89F8B6271B06D1E7BC3F00201F
:10541000490E01084440002030B5A0F17D03012B66
:10542000044683B00D46104608D9214632F0B2FC3E
:1054300015B1288804442C8003B030BD7D21019231
:1054400032F0A8FC019884F0200132F0A3FCEFE7D1
:1054500030B50F4B85B0D3F8BC2700230446C51DDB
:10546000ADF80E3014F8010B01920DF10E01FFF7AB
:10547000D3FFA542019AF5D10DF10E0010F022FFE5
:10548000019A9DF80E000021FFF7C6FF05B030BD60
:1054900080640020044AD2F8C03743F4DF2343F489
:1054A0008063C2F8C037704780640020013070B557
:1054B000094EC4B203E038F039FA013448B9E5B214
:1054C000152D21463046F6D9162D04BF034B93F80F
:1054D000C457284670BD00BF406C00208064002087
:1054E00000B1D7E7044AD2F8C03723F4DF2323F40E
:1054F0008063C2F8C03770478064002070B5114CDB
:1055000084B00546D4F8C8070E462AF0F5FC94F896
:10551000702594F87135003A18BF01220BB142F0A2
:105520000802CDE9016200234FF4964195F900008D
:1055300000911A4608212AF068FDC4F8C80704B093
:1055400070BD00BF8064002010B5064C03E0D4F8A5
:10555000C80732F013FCD4F8C80732F017FC002853
:10556000F5D110BD8064002010B50D4CD4F8CC37B7
:105570001B791E3B012B0DD9D4F8C8070121383007
:10558000FFF7BCFF0023C4F8D03784F8D437BDE858
:105590001040D9E7D4F8C807012132F0E7FBF1E762
:1055A0008064002070B50A4E0546D6F86C325E2045
:1055B0000C469847D6F86C3228469847E0B2FBF77D
:1055C00059FCC4F30720BDE87040FBF753BC00BF93
:1055D0008064002003682DE9F041002B3D4D3E4FD3
:1055E0003E4EB8BF5B42A5FB0321890D07FB013787
:1055F000C7EB0717BF0096F8723585FB0725FA172A
:105600000446C2EBA555002B57D101EB810101EBFC
:10561000810105EB810109B2DFF8BC801320FFF79F
:10562000C1FF2F4908FB057581FB0531ED17C5EB5F
:10563000A11109B21B20FFF7B5FF2368254D002BF0
:10564000B4BF53214E212320FFF7ACFF636896F8C7
:10565000722583EAE376A6EBE376A5FB0631890D96
:1056600008FB0168C8EB08184FEA880885FB083575
:105670004FEAE873C3EBA5552ABB01EB810101EBAF
:10568000810105EB810109B21220FFF78BFF124B5C
:10569000134903FB058581FB0531ED17C5EBA1110E
:1056A00009B21A20FFF77EFF6368002BBDE8F041C6
:1056B000B4BF57214521222074E7C1EB011105EB4E
:1056C000810109B2A8E7C1EB011105EB810109B223
:1056D000DAE700BF6BCA5F6B806967FF80640020F8
:1056E000D34D62100B2815D810B401EB41030A4CBE
:1056F00001EB83032344184490F8B43593421EBF52
:105700000919002380F8B4255DF8044B18BF81F80F
:10571000A8357047704700BF80640020F0B5464C44
:1057200094F8D537012B83B0054650D994F8D607A5
:105730004249434E94F8D777421CA1FB02C118445A
:1057400006EB800001F4FE7606EB9101521AD0F8C8
:10575000C06184F8D6272FB1D4F8D81704F2DC72D0
:1057600091420DD06EB9374A0133A2FB031222F0E9
:10577000010101EB52029B1A84F8D53703B0F0BD4A
:10578000314E94F8F03793B9304B019348F2A501AC
:10579000123B15226F46A4F8F417009384F8F627FD
:1057A00029463846B04758B994F8D537DBE76F46F5
:1057B00038460FF069FF29463846B0470028F3D035
:1057C00094F8F01759B138460FF0D8FEECE71C4AB0
:1057D00002EB8302D2F8C061002EC4D0D1E7009E54
:1057E0001B4A964214D9013A013E41F2210512F8B2
:1057F000013F81EA0321082311F4004F85EA4100AB
:105800000ABF490081B289B2013BF5D19642EED17F
:1058100038463CF047FC0F49009D6D1A152DA8BF76
:1058200015252A4601F1180049F038F994F8D537C2
:1058300084F8215897E700BF80640020CDCCCCCC01
:105840006CF50508ABAAAAAA451B0108896C0020C3
:10585000776C0020746C002070B50B4E054606F680
:10586000260139F093FC2C686C6006F62401641A5A
:10587000402CA8BF40242960224606F6640049F067
:105880000DF986F8A44870BD8064002030B50C4B3B
:105890000C4AC3F8242883B0C822014603F66405E5
:1058A00003F6290483F8282868463A22CDE9004502
:1058B0003CF0B0FB6846FFF7CFFF03B030BD00BF40
:1058C00080640020C83E7BEA044BD3F88C3530EA74
:1058D000030314BF01200020704700BF8064002034
:1058E000BC4A38B50820002382F82130FFF7ECFFCE
:1058F00048B1D3694FF4806402204FF482611C8068
:1059000082F8210059804FF40020FFF7DDFF48B1F5
:1059100092F82130D1695C1C40F2014082F82140AC
:1059200021F81300AC4991F87932002B5ED191F83F
:105930007A32002B40F028814FF40070FFF7C4FF4B
:1059400048B192F82130D0695D1C4FF4046482F8AC
:10595000215020F81340D1F8A410880700F1CA8024
:10596000490700F1A6809D4B1B681B065DD492F889
:10597000213082F820304FF48030002382F821302B
:105980005376FFF7A1FF28B1536901204FF404714A
:10599000507619804FF40040FFF796FF38B1537EE0
:1059A00051695C1C4FF40070547621F813004FF4D9
:1059B0000030FFF789FF38B1537E51695C1C4FF40A
:1059C000A060547621F813004FF48020FFF77CFF8D
:1059D00038B1537E51695C1C4FF43760547621F81E
:1059E0001300537E13760023537638BD0120FFF752
:1059F0006BFF00289BD04FF48030FFF765FF48B95C
:105A000092F82130D0695D1C4FF4047482F8215063
:105A100020F8134092F82130D0695D1C4FF41164D6
:105A200082F8215020F8134081E74FF40050FFF72F
:105A30004BFF48B192F82130D1695C1C4FF40360F0
:105A400082F8214021F813004FF48050FFF73CFF0B
:105A500070B192F82130D069591C1D46C9B24FF47B
:105A60000064023320F8154082F8213020F81140FC
:105A70004FF48040FFF728FF48B192F82130D169F8
:105A80005C1C4FF4846082F8214021F813004FF42D
:105A90008060FFF719FF00283FF469AF92F82130CA
:105AA000D1695C1C4FF4026082F8214021F8130098
:105AB0005DE74FF48060FFF707FF48B192F82130AF
:105AC000D1695C1C4FF4807082F8214021F81300EA
:105AD0004FF40060FFF7F8FE00283FF444AF92F85F
:105AE0002130D1695C1C4FF4887082F8214021F884
:105AF000130038E78020FFF7E7FE48B192F8213025
:105B0000D0695D1C45F2302482F8215020F8134002
:105B10004FF48070FFF7D8FE48B192F82130D06979
:105B20005D1C45F2402482F8215020F813401020DB
:105B3000FFF7CAFE48B192F82130D0695D1C4FF4DE
:105B4000E06482F8215020F813402020FFF7BCFECB
:105B500048B192F82130D0695D1C4FF4E26482F8BC
:105B6000215020F813404020FFF7AEFE00283FF4FC
:105B7000F7AE92F82130D0695D1C4FF4E46482F8EE
:105B8000215020F81340EBE60220FFF79DFE00288D
:105B90003FF4D2AE4FF40040FFF796FE48B992F8BA
:105BA0002130D0695D1C4FF4007482F8215020F838
:105BB00013400420FFF788FE00283FF4BDAE92F8A2
:105BC0002130D0695D1C4FF4C06482F8215020F868
:105BD0001340B1E6A803002080640020F03E0020BE
:105BE00003685A0607D513F4057F04D007298CBF34
:105BF00000200120704703F48253B3F5825F03BF96
:105C0000C81FB0FA80F040090020704770B5BD4C45
:105C100094F8A538012B84B000F04E8194F8B108B7
:105C2000FCF756FD94F8B238834205461FD0002891
:105C300000F0D780D4F8CC37CBB194F8712593F924
:105C40000400002A18BF08224FF4964100230325C0
:105C5000CDE9015200911A4608212AF0D6F9C4F87C
:105C6000C80720B1FFF780FC012384F8B23894F80C
:105C7000B338012B00F0C280D4F8BC683EB1A24B0F
:105C800030465978FFF7ACFF002840F0F38094F8D5
:105C9000C108FCF71DFD94F8C0388342054622D0A8
:105CA000002800F0F780F6B1337A002B00F019815C
:105CB000964A02EB8303D3F8DC3194F8702596F909
:105CC00004000093003A18BF012202210023CDE90D
:105CD00001121A4610212AF098F9C4F8AC0710B145
:105CE000012384F8C038D4F8C4683EB1864B3046EE
:105CF0005978FFF775FF002840F0AC8094F8D00881
:105D0000FCF7E6FC94F8C8388342054623D0002807
:105D100000F0C980FEB1337A002B00F0E5807B4AA9
:105D200002EB8303D3F8DC3194F8702596F9040074
:105D30000093003A18BF012202210023CDE901128D
:105D40001A464FF400712AF060F9C4F8CC0810B17B
:105D5000012384F8C83894F8D108FCF7B9FC94F80A
:105D6000D2388342054630D088B3694BD4F8D46822
:105D70004FF47A72C3F8F4243EB34FF480524021BA
:105D800030462AF0D1F80546F8B994F8703596F9FE
:105D90000400002B14BF0921082103224FF4E13332
:105DA000CDE9012100932A462B464FF480512AF079
:105DB0002CF9C4F8D80840B10123C4F8A00784F82E
:105DC000795784F8DC5884F8D23804B070BDD4F820
:105DD000D8082AF091F8C4F8D85884F8D25804B0FA
:105DE00070BDD4F8C8072AF087F894F8B338C4F81F
:105DF000C857012B84F8B2587FF43EAF94F8B4082A
:105E0000FCF766FC0546002871D0D4F8BC37002B9F
:105E10007FF432AFD4F8B828002A3FF42DAF94F8BD
:105E2000715594F8701592F90400002D14BF0822E2
:105E30000022002908BF42F0010203254FF461410E
:105E4000CDE9015200911A4620212AF0DEF8C4F86B
:105E5000BC0711E794F8C838002B7FF47CAFD4F866
:105E6000AC38002B3FF477AF0122C4F8CC3884F86B
:105E7000C82870E794F8C038002B7FF434AFD4F80A
:105E8000AC38002B3FF42FAF0122C4F8AC3784F8B4
:105E9000C02828E7D4F8AC072AF02EF8C4F8AC578D
:105EA00084F8C0581FE7D4F8CC082AF025F8C4F8C5
:105EB000CC5884F8C8584EE7D4F8A858124B284656
:105EC0005978FFF78DFE28B3D4F86035002B7FF4A6
:105ED000A5AED4F8AC38002B3FF4A0AEC4F86035C2
:105EE0009CE64FF49643E8E64FF461431CE7D4F890
:105EF000BC0700283FF4C0AE29F0FEFFC4F8BC5731
:105F0000BAE600BF80640020C43B00206CF50508A1
:105F1000A803002094F8B008FCF7DAFB0646D8B1D5
:105F2000D4F86035002B7FF479AE002D3FF476AEC7
:105F300094F8702595F90400B2FA82F252094FF4F0
:105F400016510225CDE9015200911A4604212AF08A
:105F50005CF8C4F8600561E6D4F8600500283FF4F9
:105F60005DAE29F0C9FFC4F8606557E670B5B04C66
:105F700094F8A538002B00F01F81082029F0E8FFD5
:105F8000C4F8CC0700283BD0082129F0D7FF002611
:105F90000346A849A84884F8B138C4F8E46834F046
:105FA000BFF841F208530122A348A4F8E83884F866
:105FB000EC2809F085F931462B22A04848F0CFFDA6
:105FC00048F67C607D25E02331462B22A4F8F408B6
:105FD0009B4884F8F73884F81F5948F0C0FD48F60C
:105FE0007C21A0224EF27B0384F84B5984F84E6941
:105FF00084F8F759A4F8201984F82329A4F84C3917
:1060000094F8B338002B00F0C180102029F0A0FFD5
:106010001021C4F8BC0829F091FF8A4B84F8C1080C
:106020003A2140F23B1094F8792218809F254AF2D9
:106030001E40197100219D7198601973002A40F06B
:106040008C8094F87A32002B5ED1D4F8A4307E4D47
:10605000580748BFD4F8C027286844BF42F40272EA
:10606000C4F8C027990741BFD4F8C02742F4601292
:1060700042F0C002C4F8C0271A0748BFD4F8C0379E
:10608000C0F3C01044BF43F48073C4F8C037FFF7B7
:1060900027FA0020FFF70AFA03464FF4007084F84D
:1060A000C43729F055FF4FF40071C4F8C40829F033
:1060B00045FFD4F8F83984F8D008002B14BF012329
:1060C000002384F8FC3926D1D4F86C2A0023C4F8C4
:1060D000683A002A51D0012284F8F03784F8702AF7
:1060E0004FF4805029F034FF4FF48051C4F8D408A5
:1060F00029F024FF002384F8D10884F8D238FAF775
:1061000083FEBDE8704081E5D4F8C03743F0040356
:10611000C4F8C03799E7D4F8A420002312F0020293
:1061200084F8FD3984F8FE396AD194F8793223B1C4
:106130000120FFF7C9FB00285CD194F87A32002BCC
:1061400053D1A3182868042183F8001A030602F12A
:1061500001015ED484F8041AB6E7D4F8C03794F885
:106160007A2243F00201C4F8C017002A3FF46DAF51
:1061700043F03603C4F8C03767E7D4F8743A7BB30A
:10618000012384F8703A84F8F037A9E7202029F039
:10619000DFFEC4F8B80800283FF437AF202129F00B
:1061A000CDFE2A4BC4F8683284F8B408FFF798FB98
:1061B000012384F8B33828E7042029F0C9FEC4F885
:1061C000A80800283FF4D9AE042129F0B7FE204AE0
:1061D00084F8B0080123C4F86C2284F8A538CCE612
:1061E00084F8703A84F8F0377AE70620FFF76CFB02
:1061F0000028A6D0A318022183F8001A0132A0E7D4
:106200004FF46070FFF760FB78B1012284F8002A38
:106210008BE74FF45850FFF757FB00289AD06318CC
:106220000820911C83F8000A94E702467DE700BF2E
:106230008064002088F70508606D0020746D0020E0
:10624000A06D0020943F0020F03E00205154010832
:106250009D16010810B5094B0022D3F8001303F571
:106260004173914201D1002010BD13F8014B8442CB
:1062700001D00132F5E70120F6E700BF806400207D
:10628000F0B404780A4E049F650906EB850604F015
:106290001F04012505FA04F4D6F8105704972C4280
:1062A0008068F0BC18BF43F0800333F05DBF00BFCF
:1062B000806400201B4B2DE9F04103EB81038EB07D
:1062C000D3F86C7206460D4647B3174B03EB4103F8
:1062D0001C22B3F88A42002319460DEB02000693F4
:1062E00004F01F0848F03BFCC4F3441401228DF86D
:1062F000085006AD8DF81420CDE903568DF80980BD
:106300008DF80A4002A8B8479DF8142000232AB14E
:1063100000952246414602A8FFF7B2FF0EB0BDE845
:10632000F08100BF6CF50508806400202DE9F04F76
:10633000194E90F801808578DFF86090DFF860B042
:1063400085B00446371D4FF4FA6A16F9013B002B5D
:1063500018DB39F91320A2F57A724FF47A730AFB2D
:1063600002F292FBF3F202ABA2F57A72594618469A
:1063700038F094FE02AB00932A46002341462046A3
:10638000FFF77EFF0135BE42EDB2DED1002323735D
:1063900005B0BDE8F08F00BF276800205C400020FA
:1063A000457F06082DE9FF47314B477893F8B02326
:1063B00093F8B183436885781E2AA8BF1E22022A5B
:1063C000B8BF0222B8F1100FA8BF4FF01008B8F103
:1063D000020F4FF00B01B8BF4FF0020804461970CE
:1063E000D6B25FFA88F90121501E4FF0170C88428F
:1063F000636826DC13440B2103F8011C6168002349
:106400008B546268009239462A4620463E44FFF784
:1064100037FF013E4FF0010AF6B208F1FF33534552
:1064200013DC05EB090263680093013A0023D2B242
:1064300039462046FFF724FF0023237304B0BDE84C
:10644000F08703F801C00131D1E705EB0A02D2B2AF
:106450001623394620460392F6F75AFC039A162370
:1064600031462046F6F754FC0AF1010AD5E700BF91
:10647000806400202DE9F04F184F91F8018091F8C9
:106480000290DFF85CA0DFF85CB085B006460C46F1
:1064900000253B78AB4204DC0023237305B0BDE844
:1064A000F08F2846B04702AB504502465946A8BF78
:1064B0005246184638F0F2FD04AB1844002109EBAF
:1064C000050202AB00F8081CD2B2009320460B462E
:1064D0004146FFF7D5FE0135DBE700BFC40B0010D6
:1064E0009F860100B9F0060801460148C2E700BFD7
:1064F000CD45010801460148BCE700BF59450108E8
:10650000F8B5324ED6F8A4500022A807C6F80023EA
:1065100005D50320FAF7F8FC2A20FAF7F5FC2C4FF2
:10652000002417F8010B0134FAF7EEFC2E2CF8D1F9
:10653000A90617D50E20FAF7E7FC0D20FAF7E4FCC0
:106540001820FAF7E1FC1720FAF7DEFC1F20FAF713
:10655000DBFC1E20FAF7D8FC2F20FAF7D5FC3A20F6
:10656000FAF7D2FC1B4C23681A011AD41A4B9B79F8
:10657000EBB996F8783A43B3184B194F1C680121D0
:10658000204633F0E3FD204633F014FE0025D6F814
:1065900000339D4212D320460021BDE8F84033F07D
:1065A000D5BD2320FAF7B0FC23681B01DED52420DB
:1065B000FAF7AAFC3320FAF7A7FCDAE717F8011B71
:1065C0002046FFF777FE0135E1E7F8BD8064002043
:1065D000C4F80508F03E0020142F0020EC3A0020FB
:1065E00084670020074B032883F86C0303D8064A0E
:1065F000012308B9537083E7013803FA00F05070A3
:10660000F9E700BF80640020A803002070B53F4B6D
:106610003F4C1B783F4D03F00103286884F8793A1A
:106620000023C4F81037C4F8143703681B6B92B00A
:10663000002B64D00121984784F87A0A0021286849
:1066400033F084FD286803685B6C0BB10221984726
:1066500028680AAE33F0AEFDF4F722FC2E4A2F492B
:10666000304638F01BFD00960023062214212868CE
:1066700033F07AFD2A4B0093082200230721286873
:1066800033F072FD274B0093092200230B21286869
:1066900033F06AFD244B0093286800230A220B2163
:1066A00002AE33F061FD3046FDF772F830B1286874
:1066B000009600230C22052133F056FD30F0ACFD8E
:1066C00094F86C3300F5741000F51060032BC4F8D7
:1066D0007C0A03D8154901229BB94A7094F87A3A8A
:1066E00084F8783A0023C4F80033FFF709FF2868DC
:1066F00033F020FD012384F8803A12B070BD1846B3
:106700009AE7013B02FA03F34B70E7E76E31002092
:1067100080640020EC3A0020437B0608497B060891
:106720004D7B06085A7B0608657B0608A8030020F7
:106730002DE9F04FCE4C94F8513591B0054613B188
:10674000012384F87837D4F8842ACA4F0523B2FB92
:10675000F3F303EB8303D31A386802933E4640F009
:10676000858394F8803A93B933F0EAFC68B93868C5
:1067700033F0F2FC002384F87837D4F8843A0133FC
:10678000C4F8843A11B0BDE8F08FFFF73FFFBA4F6D
:1067900094F8792A3B7803F001039A4257D0002BF2
:1067A00000F01481002384F8883A84F8893AC4F808
:1067B0004036A4F84436C4F83036C4F83836A4F865
:1067C0004C36C4F8503694F88236AC4AC4F83426B5
:1067D000012B4FF063020CBF6423632384F83C2633
:1067E000A74AA4F85436002114233068A4F856367A
:1067F000916133F0DFFC94F8AE33012B06D0022B0D
:1068000040F0E1803B789A0700F1DD80F4F748FB27
:1068100094F8AF339FED9B7A07EE903AF8EEE77A63
:1068200067EE877AFDEEE77A17EE908A964B009333
:106830003068002307220C2133F096FC08EB050397
:10684000C4F87C3A3B7803F0010384F8793A3B784A
:1068500013F0010300F0F88094F88B268B4B002A8C
:1068600000F0DB80B3F90C30B4F934269A42B8BF9B
:10687000A4F83436B4F93626B4F964359A42C8BF60
:10688000A4F836366422D4F8943593FBF2F3B4F9C5
:106890003A261BB29A42B8BFA4F83A360EF02EFF41
:1068A00094F83C36D4F840268342D4F89C3688BF0E
:1068B00084F83C069A42B8BFC4F84036744BD3ED16
:1068C000007A13ED127AB4EEE77A603BF1EE10FA3B
:1068D00048BFC3ED067A0EF0F9FEB4F8542603B2B1
:1068E0009A426C4BB4F95626B3F90C30C8BFA4F8E1
:1068F00054069A42C8BFA4F8563694F83F3303F0C2
:106900000303032B07D1B4F84033B4F944269A4269
:10691000B8BFA4F84436604B1B6813F0006309D07D
:10692000D4F89426B4F94C1692F901209142B8BFDC
:10693000A4F84C26594A91799446002977D05848B2
:10694000002310F89C2B1946914269DBB3FBF2F24D
:10695000C82353439CF81A20B3FBF2F3D4F8502613
:106960009A42B8BFC4F85036D4F88C3AD4F82C26E2
:10697000EB1A1A44C4F82C26D4F830261344C4F871
:1069800030363068C4F88C5A03685B6C0BB1022156
:106990009847D4F87C3A002B00F0C580EB1A002B06
:1069A000306880F2B7803F4AB2F9061040F2D663F1
:1069B000994203DCB2F902209A4201DDC4F87C5A04
:1069C00033F0CEFBD6E6DFF8E4802FE7D4F860336F
:1069D000002B3FF437AF94F88A3A002B7FF432AFA4
:1069E000D4F84C3513F0600F08D02A4BB4F8B42219
:1069F0005B7803EAD2235B077FF424AF012384F89A
:106A0000883A294B2B44C4F87C3AB4F86435A4F88E
:106A10003836002384F88B3A14E7B3F90E3023E7B5
:106A200000EB810E0131BEF80CE073448CE7002BC3
:106A300094D0D4F89436927E9B89642113FB01F3A1
:106A4000520893FBF2F389E794F8882A002A98D039
:106A5000D6F80080B8F1000F2AD098F90F20002A4C
:106A600026DD84F8883AC4F87C3AC4F8303688E7E2
:106A700080640020EC3A00206E3100200000881372
:106A8000B06A00200050C347A4780608BC3F00202D
:106A9000106B0020A8030020F03E0020142F0020DF
:106AA000C40B00105C4000200087930320A1070066
:106AB0000E2014F093FF94F8893A48B1002B3FF46C
:106AC00060AF0023404684F8893A33F073FB58E7FF
:106AD000D3B9012384F8893A05F5742303F51073BB
:106AE0004046C4F8903A33F065FB94F88B0A30B90D
:106AF000FCF788FE84F88B0A306833F05BFB94F86F
:106B00008B0AFCF77FFE3CE7D4F8903A9D42FFF4F5
:106B100038AFE1E733F04EFB0023C4F87C3A84F849
:106B2000883AC4F830368E4B1A6812F0006F9946D6
:106B300004D0FF20FDF79CF9C4F89406D4F8A4B063
:106B40001BF0020F27D0874BB4F8DE225B7803EAF4
:106B5000D223D4F8602303F0070302F480421343E6
:106B600019D0814BA3F2044293ED007AD2ED007A62
:106B7000E7EE077A93ED017AE7EE077A93ED027A72
:106B80007A4BE7EE077AB1EEE77AD3ED027A67EE59
:106B9000877AC2ED007A336823B193F90F30002B66
:106BA00000F3CD800EF0AAFD94F85023D4F81037EE
:106BB0008242D4F89C068CBF43F0010A23F0010AFC
:106BC000FAF72EFAC4F810A780460EF07FFDB4F84D
:106BD000A223D4F8143782428CBF43F4804323F4B9
:106BE0008043C4F8143794F84735002B4BD12AF46E
:106BF000800323F0020394F83FA3C4F810371AF07F
:106C0000020F0DD05A4A127D042A09D994F8BC1AF1
:106C100091424BD9039317F035FC039B002845D0D4
:106C200043F48043C4F81037B4F85233039303F0AD
:106C30000F00FAF7E9FF039B4E4A1B0A5A4327D17C
:106C4000D4F8103723F02003C4F81037B4F85433C5
:106C5000039303F00F00FAF7D7FF039B454A1B0A83
:106C60005A431CD1D4F8103723F04003B4F84C0336
:106C7000D4F89C15D4F8142788421ADD23F0102389
:106C800022F0200219E04AF4800343F00203B2E745
:106C90009042D4F81037D3D343F02003D4E7824294
:106CA000D4F81037DED843F04003DFE723F4804305
:106CB000B8E743F0102342F02002B4F84E13C4F8B2
:106CC0001427642098FBF0F888453CDB3978C80726
:106CD00039D543F400431BF0200F37D03978C9076A
:106CE00034D50AF0030ABAF1030F2FD1B4F8AC136C
:106CF00061B3B4F84003884228D343F00043C4F89A
:106D00001037D9F800301B010ED594F9643313F114
:106D1000800F20D0D4F8941691F9011099421ADB13
:106D200042F00802C4F814270E2014F057FE014662
:106D3000306809B333F03EFA306833F011FA306846
:106D400033F0F8F916E523F40043C4E723F00043D9
:106D5000C4F81037D5E722F00802C4F81427E3E797
:106D6000F03E0020A8030020146F0020C40B001088
:106D7000BC3F00200087930394F87A3A002B72D02E
:106D800003689B6B0BB101229847D4F8A43094F8A8
:106D9000CE2AD6F80080C3F340139A4203D084F879
:106DA000CE3AFFF7ADFB334B3348DFF8D490B5FB59
:106DB000F0F505F0010583F864570393D4F8003328
:106DC000029A9A42B8D294F8783A23B999F8001006
:106DD0004046FFF76FFA19F8017B284B03EB870356
:106DE000D3F888B3BBF1000F39D098F8103073B9DD
:106DF0007A0904EB820207F01F01D2F81027012361
:106E00008B40134203D0039B93F864373BBB04EBE6
:106E100047031C22B3F88A520023194609A805F03B
:106E20001F0A0893C5F3441547F099FE01238DF816
:106E3000107008AFADF81C30CDE905788DF811A0C1
:106E40008DF8125004A8D8479DF81C303BB19DF82E
:106E50001D3000972A46514604A8FFF711FA029BFD
:106E600001330293AAE733F0A5F98EE70368DB68E4
:106E7000984782E4A8030020400D03006CF5050844
:106E80008467002010B5084B084C09480021FF22F8
:106E900084F8CF1A83F8652706F070FF94F856053A
:106EA000BDE8104006F06DBEA803002080640020FD
:106EB00098F505082DE9F04FC94C94F8D03A8DB0FB
:106EC000002B00F0848094F8D13A002B7FD194F805
:106ED000CF3A05460C20002B75D014F07FFD00281A
:106EE00040F02C8106F05CFF94F857650123012ED9
:106EF00084F8CF3A6ED9022E69D10023B4F8D21AA1
:106F0000B84FDFF81483DFF814E3DFF814931E465C
:106F10004FF0010C41FA03F2D2070ED457F82320A8
:106F2000AA1A02EB080070450CFA03FA05D94A4583
:106F300088BF47F8235046EA0A060133092BE9D1F6
:106F4000002E44D094F8B853002D00F0DA8094F865
:106F5000A334DFF8D082B4F8A0750297203394F8F8
:106F6000AB74A148019708EB830738F8233094F8F5
:106F7000A12494F8A01400780593FB780493BB78BF
:106F80000693203102F1200300F00102039208EB86
:106F9000830308EB810208EB850A099208934746B0
:106FA00008F1F0054FF4B479079657F8046BC6F36F
:106FB0000323042B00F2E780DFE813F04300CD0049
:106FC00039013601EB0014F009FD00288AD00DB01C
:106FD000BDE8F08F0B2014F001FD002800F0318196
:106FE000824A834B126894F85E65A3FB02131B0967
:106FF000FA2101FB13237D2B28BF00267D4F97F834
:107000006537B34203D1D4F8F83A9D42DFD37A48CA
:1070100000EB860006F0B2FE94F8560506F0B1FDCE
:1070200007EE905A9FED757A87F86567F8EE677AF4
:1070300077EE877AFCEEE77A17EE903AC4F8F83AE2
:10704000C5E7C6F3834303F1200208EB8201F00495
:1070500038F822C08A78C9783CD56948019E30F951
:1070600016B040F2DB50834500F3038103F10F00BB
:1070700000F00F00203008EB800338F820E09E7805
:10708000DB780A930A98ABF57A7B091A0BFB01F1BE
:107090000846ACEB0E0356490B90921B0BFB03F317
:1070A0000BFB02F281FB03BC81FB021B5049DB1787
:1070B000C3EB6C13D21781FB001CC1170A98C1EBFC
:1070C0006C11C2EB6B127344324401441FFA83FC0F
:1070D000D2B2C9B24FF4B4704A4BAA70844483FB55
:1070E0000C3060444FEAEC76C6EB202609FB16CC48
:1070F000BA45E970A5F800C005F104057FF455AF65
:10710000079E414F414ADFF8DC9000254FF001080F
:1071100001E057F8042F08FA05F3334214BF0120A9
:10712000002009EB850101359047092DF1D194F834
:1071300056050DB0BDE8F04F06F023BDFFF7A2FEE7
:1071400094F8CF3A002B3FF442AF94F85765012EE4
:107150003FF6D1AE3EE7029940220023114207D10B
:107160000133052B0FD02A4A32F82320002AF5D10B
:10717000C6F38550002240FA02F1C90700F1AE8043
:107180000132062AF7D1DDE9041C069A4FF4B470E7
:1071900014E00EF0B3FA00B200EB80001D4BC0EB20
:1071A00000104000A3FB003040091E3820EAE070C8
:1071B0004FF0000C00F5B4706246FF21F3048BD54C
:1071C000019E0F4B33F91630094EA3F57A7309FB74
:1071D00003F386FB03E6DB17C3EBA61318447BE738
:1071E00080640020546F00206E310020102F00209A
:1071F000D34D6210A803002098F5050800247449B7
:107200005C400020B7600BB6E0F905086910010882
:1072100004FA05081F85EB513F4B4C003E4B4C00D8
:107220009F8601003C6800201FF0A4FBB3E7039B8E
:10723000EBB1089B9A78D978B3F800C04FF4B470DA
:10724000BCE7404BDB78002B7FF4CAAE012E5BD04D
:1072500094F8586594F85435002B3FF4CFAE94F869
:107260005135002B3FF4CAAE94F85E65C6E6099B23
:10727000E0E7113303F00F03203308EB830038F805
:1072800023308678C078ABF2DC5BA3EB0C030BFBFE
:1072900003F3B61A401A0A932B4B0BFB00F00BFBBF
:1072A00006F683FB06BE83FB003BC3170B930A98CD
:1072B000254BF617C6EB6E1683FB003EC3170B98E3
:1072C000C3EB6E13C0EB6B10014432449C44D2B24A
:1072D000C9B21FFA8CFC4FF4B470FDE61B4901EBF8
:1072E00083034FF4B47093F89A3403EB430304EB35
:1072F00043031A4492F87C24203208EB820338F8C6
:1073000022C0D9789A7859E794F85D3523B1104BAB
:107310001E7816F001069DD00E4AB4F85A1594F85E
:107320005C3510680C4EB0FBF1F201FB03F301FB7E
:107330001202A6FB0313B2EB531F94F8596528BF42
:10734000002687E770310020D34D62106CF50508E8
:107350006E310020102F00201F85EB510F2A11D80D
:1073600005280BD805290DD80F4B00EB400003EB87
:1073700040000144012081F87C24704706280AD08F
:10738000072801D0002070470029FBD1064B0120BF
:1073900083F8AB2470470A29F4D8034B1944012021
:1073A00081F8A024704700BF806400202DE9F041DF
:1073B0001C4FDFF8788000F120060C4607EB8607AB
:1073C0000025204638F032FD08EB45020346B2F8AE
:1073D000AC24824220DB012D20464FF02C0109D045
:1073E000022D0FD10F4800EB860686F8BF3301202F
:1073F000BDE8F08187F8BE3347F0C8FB60B1441C9C
:107400000225DEE7A7F8BC3347F0C0FB0135441C7A
:1074100010B1032DD5D1EAE7034B002043F8260035
:10742000BDE8F081806400203C6800206CF5050810
:10743000794900202DE9F04302460D4604460AE052
:10744000062E02F1010208BF01349E0448BF01303C
:10745000202A00F0B58055F8043BC3F30326002B27
:10746000EED16E4E6E4B86F8B823E4B2012586F855
:10747000B94386F8BA03C6F8FC2A83F86657002A8F
:1074800000F0AD8000204FF00F0EF0460546074695
:10749000894659F8043BC3F3031C654503F00F0309
:1074A000B8BF6546E045A8BFE046984207F101072E
:1074B000B8BF18469E45A8BF9E469742E9DB4545A2
:1074C000C1BF45446B10013305F1FF35C7BF5BB247
:1074D00045F3470506250723704586F8435586F88A
:1074E00042355CDD70444710013701387FB240F30C
:1074F000470004EBC40304EB430303EBC303C3F3F0
:10750000460545EAC313DBB22A2B86F8400586F808
:10751000417526D8062386F8BB3301EB82030A4661
:1075200001E0934244D052F8040B4004F9D5002402
:107530000A4601E093423DD052F8040B8704F9D586
:107540000A4601E0934238D052F8040B8503F9D57E
:107550000A4601E0934225D052F8040B000415D4EA
:10756000F8E7062C234608D9E50706D401E0DC0736
:1075700002D45B10062BFADCDCB286F8BB43002A8F
:10758000CBD140F21B1406E08B420ED051F8042BF5
:10759000D203F9D5A4B2A6F8D24ABDE8F0830620FA
:1075A0000727A6E744F01004F0E744F00804F1E7E9
:1075B0000124BDE744F00204C2E744F48074C7E745
:1075C000164E174B86F8B823E4B2012586F8B94366
:1075D00086F8BA03C6F8FC2A83F8665752E704EB2C
:1075E000C40304EB430303EBC303C3F3460040EAC5
:1075F000C313DBB2062007252A2B86F8430586F83D
:10760000400586F8425586F84155AAD886F8BB034E
:1076100040F21B14BFE700BF3C68002080640020DC
:10762000A80300202DE9F04F002589B06F4B704E64
:1076300043F82050CDE9015503900C462F46AB4648
:10764000A846A9462C204FF0010A2378E9B293B14D
:107650000DF1140C002205E00CF8013B14F8013F79
:1076600001324BB1984200F089800A2AF4D10020FF
:1076700009B0BDE8F08F1A4608AB1A4402F80C9C1A
:107680000028F4D14B1E0134032B00F2AA80DFE85E
:1076900003F06548230205A838F0C8FB0F2872DC08
:1076A0008304019A02F00F0040EA885848EA030870
:1076B000029B039A4F4848EA0B2B1B0100EB820008
:1076C000DBB24BEA07371F43C0F8BC73FFF7B0FECD
:1076D000012009B0BDE8F08F9DF81420002A41D0A8
:1076E0000DF1140E8C4644490023432001E011F8AB
:1076F000010B90423AD00133072BF8D1542A38D0ED
:107700004F2A48D0422A51D0562A54D0492A5DD017
:10771000572A08BF05232DD01EF8012F002AE2D1D9
:1077200020E09DF8143005AAE3B14E2B10D0452B74
:107730002BD0532B34D0572B42D0552B4BD0442B2E
:1077400008BF052305D012F8013F5BB14E2BEED1E7
:1077500000230AFA03F348EA0308F4E705A838F01F
:1077600065FB019016F8010B01356EE7542A9B4624
:10777000C6D100230AFA03F31F43CDE708AB1A442E
:1077800002F80C9C7EE700238BE701230AFA03F33F
:1077900048EA0308D7E701230AFA03F31F43BBE7CC
:1077A0000B460AFA03F348EA0308CCE702230AFA75
:1077B00003F31F43B0E763460AFA03F31F43ABE743
:1077C00003230AFA03F348EA0308BCE704230AFA8E
:1077D00003F31F43A0E704230AFA03F348EA03086C
:1077E000B1E705A838F022FB0290BBE73C68002017
:1077F00021FA0508806400208DEE050810B5FFF71A
:1078000017FE074B40F6A84203F53060002193F8BD
:10781000554547F0A4F9034B83F8B04610BD00BFAF
:107820008064002078750020F0B55D4C5D4ED4F882
:10783000B4263368DFED5C6A5C4D3168C4F8B41679
:107840009B1A07EE903AF8EE677AB7EE007A67EE89
:10785000A67A95F83F33F4EEC77AF1EE10FA88BFB6
:10786000F0EE477A04F5D76213F0010383B0C2ED5E
:10787000007A0CD14E4AA5F840331278A5F842336D
:10788000D20730D4012384F8D83603B0F0BD01AB61
:107890006A4604F5D86104F2BC60F4F763FF44481B
:1078A0004449019B009A0078A1FB027281FB03719D
:1078B000DB17C3EB61135209C107A5F84023A5F8F4
:1078C0004233DFD595F83F333668DB0761D595F84D
:1078D0008B36394F8BBBFB890F2B30D8B868D4F867
